:020000040800F2
:1030000000500020196B0108A52401080155010892
:10301000A3240108A12401089F2401080000000046
:103020000000000000000000000000009D240108D6
:103030009B2401080000000099240108A9A80008A9
:10304000B96B0108B96B0108B96B0108B96B0108CC
:10305000B96B0108B96B0108B96B0108B96B0108BC
:10306000B96B0108658E0008B96B0108B96B0108DE
:10307000B96B0108B96B0108FDFC0008B96B0108C8
:10308000D1B70008B96B0108B96B0108B96B010829
:1030900005250108B96B0108B96B0108B96B010876
:1030A000B96B010821F90008B96B010831F9000872
:1030B00011F9000801F90008F1F80008618B000817
:1030C000638B00085D8B00085F8B0008B96B0108FB
:1030D000B96B0108F5FC0008B96B0108EDFC0008AC
:1030E000B9A80008B96B01085D4E01080000000096
:1030F00000000000000000000000000000000000D0
:0C31000000000000000000005FF808F173
:103110002DE9F04F684B694EA1B033600023736016
:1031200010F0EFF818B910F00DF90AF055F80AF0A0
:103130001DF9634A634D1378634F43F00103137025
:103140000023089309930A934FF4E0130B932B6821
:10315000387B43F480332B60AB6943F01003AB61E1
:103160002B6803F400330993089B01330893099BF0
:103170001BB9089BB3F5A06FF2D12B68514913F42A
:10318000003301D0022315E00A6842F001020A6010
:1031900008932B6803F002030993089B01330893FB
:1031A000099B1BB9089BB3F5A06FF2D12B689A0756
:1031B00039D501230A93454B45491A6842F010025C
:1031C0001A601A6822F003021A601A6842F00202BA
:1031D0001A606B686B606B686B606B6843F480634C
:1031E0006B603C4B1A68043B22F070425A603A4ACA
:1031F0001160696821F47C116960596841F00041EF
:103200005960D96821F40041D9609B681B0449BF0B
:10321000324B4FF4E01313604FF480130B930A9B6F
:10322000012B01D117E0FEE7022B18D168B10B9BEF
:10323000B3F5801F02D14FF4A01305E00B9BB3F54B
:10324000E01F02D14FF400130B930B996B680B43F3
:1032500043F4803302E06B6843F460136B602B68C7
:1032600043F080732B602968164B8C01FBD559689D
:1032700021F003015960596841F0020159606B68FF
:10328000104903F00C03082BF9D14B68DFF8548088
:1032900003F00C03042B03D0082B03D00C4B29E0C4
:1032A000136827E04B684868C3F38343C00303F106
:1032B000020319D40A4A1CE097CA000860010020E2
:1032C000DC2D002000100240B40F0020002002403E
:1032D00000127A000410014040000020001BB700DB
:1032E00000093D00EC00002049681268890348BFCE
:1032F00052085343C8F800306B68DFF83091C3F3CD
:10330000031319F80320D8F8003020ACD340C8F8D4
:1033100000303A4A3A4BDFF818B19360394B4FF01E
:10332000000AD360AB69039243F00103AB616B6A9F
:103330003548B3606B6A43F080736B62AB6943F0EE
:103340001C03AB614FF6FF7324F82C3D21468DF82A
:1033500056A00FF089FD584621460FF085FD2B48F9
:1033600021460FF081FD2A4920464B6843F0007347
:103370004B600DF095FE159B2649039AB3FBF1F3C4
:1033800025490B60254B4FF47A71C3F800A0D8F89B
:103390000030DFF89480B3FBF1F32149013B4B602F
:1033A000F02382F823300723C1F808A00B60BB6824
:1033B000DFF880A0CAF8003009F1100393E8030099
:1033C000AB6984E8030043F00803AB610823CBF842
:1033D0001030159816A90FF047FDDAF800301B07DA
:1033E00030D598F89031012B2CD80E4B98F89121BC
:1033F0009B6813F0805800F0898523E000ED00E021
:10340000003000080005FA050008014000100140E6
:103410000000014040420F00AC18002000190020BD
:1034200010E000E060010020B40F0020EC970108DC
:10343000000C014094170020B74B002283F8912123
:103440000AF03AF9642007F03CF9A022B3480021C1
:1034500015F03FFBB24A536823F4406343F07063B6
:1034600043F400635360EB69002243F00703EB6110
:10347000AB6943F4006343F00C03AB61A94B002537
:1034800003F10C01555401320C2AF7D1FF221A76B0
:103490005A769A76DA76A44BA44A29461A60A4484A
:1034A0003022DAF8008015F014FB2946C8F3801AA0
:1034B0000423A04A9E488D5C0C224A431554BAF15D
:1034C000000F06D11E2D01BFFF2503F1FF33155458
:1034D000DBB201310429ECD1974A7D791370974B07
:1034E00097491D70974B8F4AF361C0330B60964B21
:1034F00018F0200F03EBC5035B7818BF012313629C
:10350000002340F2DC51914A22F813100133082BBA
:10351000F7D10EA800211C2215F0DBFA0E2D03D0E6
:1035200005F0EF03082B02D101238DF84830C8F3D2
:1035300040038DF83E30C8F340338DF83830C8F37F
:10354000C0338DF83B3018F400638DF840A007D0ED
:1035500097F8843103F1FF3EDEF1000343EB0E03E5
:103560008DF83C30C8F300438DF84130336AB7F82A
:103570004401003318BF01238DF84230C8F30053D3
:103580008DF84330B7F8463118F4805FADF8463017
:10359000B7F85231ADF84C0018BF5F48ADF8443071
:1035A000C8F3804318BFB0F84C018DF83F30B7F82E
:1035B000503118BFADF84C00B3F5FA7FADF84A3082
:1035C00084BF0023ADF84C3097F8D431604886F8BA
:1035D0002430002386F8253043709DF8483008F0E9
:1035E0000101002BC8F3C0028DF839108DF83A2084
:1035F0000CBF0023022301B902B1013309EB830997
:10360000D9F818304FF0000AA3F1020B16330393D8
:103610004FF6FF723BF8023F934200F0A6819DF8FF
:103620003D10DDB21B0ADAB219B1A91E012940F220
:1036300098819DF8401031B14648290140584649CB
:10364000884200F08E819DF8411031B14148290136
:1036500040584149884200F084819DF83E1051B1A4
:103660003C483E4F00EB05104168B94203D1018947
:10367000012900F076819DF83B1051B13548374F54
:1036800000EB05104168B94203D10189022900F01D
:1036900068819DF83C1051B12E48314F00EB051068
:1036A0004168B94203D10189022900F05A81022BF5
:1036B00002D19DF8383003E0012B04D19DF8393058
:1036C000002B00F04E819DF8433033B19DF8483017
:1036D0001BB92B1F032B98BF04221E4B9DF83810DB
:1036E0002D015F1900293FD0D11EC9B2012909D887
:1036F0005B59B3F1804F00F0348117498B4240F0A1
:103700008D802EE1022A40F00F815A59154B9A42C2
:1037100040F0868025E100BFB40F0020481900204A
:103720000000014060010020A02B0020A611002015
:10373000A42B002010D20108610F0020D007002028
:10374000641A0020C40F00204CBE0108D00E0020D7
:10375000850100209CB801080004004000080140D9
:10376000000C014000080040012A57D19DF83F207D
:10377000DFF8508322B9BDF84A20B2F5FA7F06D9A6
:103780005A59CB4B9A4204BF032388F82730C94AC1
:10379000FF23511991F80DE088F86C3088F86D30EE
:1037A000486801F1080309894FF00009ADF8541089
:1037B00002218DF8571088F870902146C8F87C7067
:1037C0008DF856E00592049388F82890C8F82C905C
:1037D000C8F83090C8F83490C8F8689088F86E90AF
:1037E00088F86F900FF040FB049B059A9978505928
:1037F0004A4607F03EFE3846494601220CF0D2F90F
:10380000AD4BAE49C8F88030AD4BC8F88890C8F8C9
:10381000843038460A1D0CF00DFAA2E0022A4CD181
:103820005FFA8AF31C2101FB03FCA64B4FF0000852
:1038300003EB0C09012389F8703005939D4B89F83F
:1038400071A0591991F80DE001F108024868098941
:1038500089F87280ADF8541002218DF8571089F85C
:103860007A802146C9F87C70CDF818C08DF856E0F2
:1038700004920FF0F9FA8F4B049A58599178424606
:1038800007F0F7FD059B38461A4641460CF08AF9C9
:103890008D4A8C4BDDF818C0C9F8802003EB0C0171
:1038A0008A4A8031C9F88420C9F8888038460A1DC0
:1038B0000CF0C0F90AF1010A53E0032A37D19DF850
:1038C0003F30804DDFF83C823BB195F8269038467A
:1038D00008214FF6FF7200231AE0BDF84A2095F840
:1038E0002690B2F5FA7FBDF84C300BD978493846AE
:1038F000B1FBF2F2082192B207F010FE754B48F8C6
:1039000029000AE074493846B1FBF2F2012192B273
:1039100007F004FE714B48F82900C36095F8263083
:10392000013385F826301CE0012A3FF41FAF042A3A
:1039300017D1BDF84420684B624D93FBF2F2384634
:10394000BDF84630012192B295F8258007F0E6FDDA
:1039500095F8253005EB88080133C8F8500185F843
:103960002530039B9B457FF453AE96F825205C4B96
:1039700086F870215B4A002517781D70A7F11702A1
:10398000022A98461AD8F3690021585903EB050911
:1039900012F07AFA10B1336A7BBB27E0524B05EB89
:1039A000030E99E80F008EE80F0098F800301035EC
:1039B0000133C02D88F80030E5D1ECE74B4B13F80C
:1039C00037E003EBC703D3F804C088F800E0BCF18C
:1039D000000FE0D07545DEDA434A2B0103EB020904
:1039E00063440FCB013589E80F00F3E7404B1A68B9
:1039F000049312F4805F24D11DE03E4B3E4A13F83D
:103A0000370003EBC7035D681070002DEED0002374
:103A10008342EBDAC3EBC3016A18D2F800C0DFF8C7
:103A2000E8E0013341F80EC001EB0E069188B18049
:103A30009279B271ECE707F0EF03082B2F4B25D1F9
:103A400026E098F80030012BF5D92D4D05EB031336
:103A500003F110061035B542EDD055F8100C4FF0BB
:103A60007C5112F07DF84FF07C5145F8100C55F860
:103A7000140C12F075F84FF07C5145F8140C55F801
:103A80000C0C12F06DF845F80C0CE3E70E2F08D182
:103A90001A78182F42F010021A7037D107F084F903
:103AA00034E01A78192F22F010021A70F5E700BFDF
:103AB000000800409CB80108E5AE0008E0010020C5
:103AC000D1AF000860010020ADB40008BBAE000813
:103AD00000127A00F1AF000840420F00E1AF000889
:103AE00044190020D00700200C0700204CBE01081C
:103AF00094170020B0A60108F0190020B01700208C
:103B00001407002014190020F119002007F030F9E3
:103B1000049B02271B6821465D035EBFBB4B01224D
:103B20001A70BB4ABB4D13788DF8577043F00403ED
:103B300013704FF40043ADF8543014238DF8563011
:103B4000AB69B54843F00403AB610FF08DF9B34A9C
:103B5000B34B00201A6006F0B7FEB24B032693E881
:103B60000300AB6984E8030043F00803AB611598D8
:103B700016A90FF079F9AB694FF0180B43F4805395
:103B8000AB61EB68A44843F48053EB602146A0236B
:103B90004FF00408ADF854308DF857608DF856B0EA
:103BA0000FF062F940239C4821464FF0100AADF80F
:103BB00054308DF856800FF057F997482146ADF8EC
:103BC00054A08DF856A00FF04FF9EB684FF007099D
:103BD00043F48053EB60EB68214623F48053EB60A1
:103BE000914B1A8802F4415242F4457232431A80D2
:103BF0009A8B22F4006202FA0AF222FA0AF29A83FB
:103C0000A3F810901A8892B242F040021A80EB6931
:103C100043F48043EB612B6943F480432B618DF8BF
:103C20005760824E4FF420433046ADF854308DF843
:103C300056B00FF019F94FF4804330462146ADF8E5
:103C400054308DF856800FF00FF94FF480583046FD
:103C50002146ADF854808DF856A00FF005F92B6978
:103C6000734A43F480432B612B69384623F4804325
:103C70002B61138803F4415343F4457343F003036A
:103C80001380938B23F4006303FA0AF323FA0AF3F5
:103C90009383A2F8109013889BB243F040031380E3
:103CA000C6F8108006F0AAFB002801F07780438850
:103CB000002B01F073805F4F049B384600211022D7
:103CC0001E6814F006FF4FF6FF73ADF83430022380
:103CD00006F4004906F400684FF0000A1E408DF813
:103CE00036308DF837A00DD0012620A921F84C6D73
:103CF00049480DF043FB072387F800A087F801A08F
:103D0000BE70FB70B9F1000F0ED0022320A921F87C
:103D10004C3D41480DF032FB0123F2183B71BB7161
:103D200007237E71FB71D6B2B8F1000F0FD00223CA
:103D300020A921F84C3D3D480DF020FB092301222C
:103D40003B73BA73731C07227E73FA73DEB26B681F
:103D5000394843F440436B606B69DFF8DC8043F023
:103D600001036B61AB6943F40073AB610DF020F9A3
:103D7000324B012E1593324B4FF00005169394BF32
:103D80002B4680231A934FF480731B934FF4806368
:103D90001C93202321461D9340464FF40053189650
:103DA0001E93179519951F950DF0E4F8D8F800307B
:103DB000244A43F00103C8F800305368012E23F46D
:103DC000702394BF0021012123F4807343EA01236F
:103DD000536091681C4B013E0B4043F4602343F059
:103DE00002039360D36AF6B223F4700343EA0656E3
:103DF000D66201237A199178002972D0785D591C16
:103E00000928C9B2D2780F4E31D91FE0380C0020F2
:103E1000DC2D00200010024000080140E9A300084A
:103E2000E42D00201498010800300140000C0140EE
:103E300000380040CC250020080002404C240140FE
:103E4000DC25002000240140FDF7F1FFA0F10A0469
:103E5000D6F80CC004EB44044FF0070E0EFA04FE33
:103E60002CEA0E0EA2404EEA0202F2600CE0346927
:103E700000EB400C4FF0070E0EFA0CFE24EA0E0485
:103E800002FA0CF222433261062BA54C0CD85A1EC2
:103E9000666B02EB82021F23934026EA030600FAB8
:103EA00002F3334363631BE00C2B0CD8DA1F266B41
:103EB00002EB82021F23934026EA030600FA02F374
:103EC000334323630CE0A3F10D02E66A02EB8202A6
:103ED0001F23934026EA030600FA02F33343E3620A
:103EE0000B460435102D85D18D4B9A6842F48072B3
:103EF0009A609A6842F001029A609A6842F0080259
:103F00009A609968864A080731D5FAE7531E092B4B
:103F10003FF698AAD9F84C002146206058460EF08A
:103F2000A3FF4FF40063CBF810303C2006F0C9FB30
:103F300097F891319845BFF67FAADFF828B208229A
:103F40004FF40063CBF8102078200492CBF81430A3
:103F5000039306F0ABFB049A039BCBF81420782064
:103F6000CBF8103006F0A2FB08F10108E0E79368F7
:103F700043F0040393606A4B9A6812F004020392C0
:103F8000F9D19A6842F4A0029A60664BB3F85801DE
:103F9000002840F00887B3F95A21002A40F003872F
:103FA000B3F95C31002B40F0FE86DFF8BCB15D4D0B
:103FB000DBF8003000210C225B48B3F8569095F8EE
:103FC0005F7195F8696114F084FD0021142257484F
:103FD00014F07FFD564C57490023574A0B7094F854
:103FE0007831C4F87421CDF814B08846924633B1C4
:103FF0000022A4F87A2153B904F096FE07E0069354
:1040000004F0EEFE069B002800F03481F0E74B4AF6
:104010001920138823F040031B041B0C1380138802
:1040200023F038031B041B0C43F030031380138868
:104030009BB243F04003138094F87C1104F05EFEC1
:10404000012006F033FB01211A2004F057FE012065
:1040500006F02CFB15A804F01DFE9DF95630013327
:1040600003D19DF95430013303D0B4F87A319BB2B7
:104070001BB10023A4F87A31FCE02C4B304A6420B9
:104080001A60304A5A60304ADA60304A1A6106F0E3
:1040900018FB042388F800302D4B06221A702D4A95
:1040A000136843F0010313602B4B0022092F1A7091
:1040B0009B4601D91746F7E740F202320123BB4085
:1040C0001A4042BB13F0FD0F25D094F87831C4F8A4
:1040D00074A133B10022A4F87A2143B904F024FE7C
:1040E00005E0069304F07CFE069BA0B1F2E70E4BC0
:1040F0001A4A64201A601A4A5A6006F0E2FA042347
:104100008BF80030124B07225A70124A136843F0A2
:10411000020313602AE0012F28D90027C4E700BF5B
:1041200000240140B40F0020CC280020E02600200D
:1041300060010020F42600201C9801080030014096
:10414000398B0008958C0008AD89000890C1793D35
:10415000E8000020AC170020022E0020258B00086C
:104160002D8C0008000C0140E00E0020354F3B680C
:10417000990702D5344B1B689847002384F87C319B
:10418000324B4FF47A721A60314B1B689847314AB0
:104190000023137016B1022E40F0F6854FF0000A8E
:1041A0000A20012115AA8DF854A0C4F880A111F0AD
:1041B000D1F8002800F07C869DF85430482B0CD1B3
:1041C000254B264A1A60264A5A60264B0222DA708C
:1041D0003B6843F008033B6002E0504600F068BED5
:1041E00095F854310BB188F8003095F855310BB182
:1041F0001D4A137095F856310BB1164A13703B687F
:104200001A071AD50FFA89F9642799FBF7F6304691
:1042100011F052FC804607FB169000B211F04CFCE6
:10422000124911F09DFC0146404611F091FB1049E6
:1042300011F096FCC4F884011FE00023C4F8843117
:104240001BE000BFAC170020CC28002080260020F7
:10425000E0260020FE2D002078060020CD2E01084B
:10426000352C0108E8000020022E00208988883CB7
:1042700000002041012006F083FBAB4A0A26137898
:1042800043F002031370A94B08221A61A74F1920AB
:10429000FB68013E83F00803FB6006F012FA012080
:1042A00006F012FB192006F00CFA002006F00CFBB9
:1042B00016F0FF06EAD108233B619D4B1B681B07E4
:1042C00005D59C4B1B6898479B4B01221A709B4B52
:1042D00000271E68DFF89C82307B11F0EDFB9849C7
:1042E00011F03EFC08F01CFF964B1860964B1888A6
:1042F00011F0E2FB01464FF07E5011F0E5FC934BCC
:104300008F491860924B186911F02AFC914B186084
:10431000307811F0D1FB01464FF07E5011F0D4FC03
:104320008D4B014618604FF07E5011F00FFB8B4B08
:104330004FF07E5218608A4B38469A601F605F606B
:10434000884B9A601F605F6008F0EAFE06463846B8
:1043500008F074FE31460746304611F001FC39463C
:104360008246384611F0FCFB31468146504611F03A
:10437000F7FB39468346484611F0F2FB01465846A2
:1043800011F0E6FA3146C8F80000384611F0E8FBB3
:104390003146069011F0E4FB069B834639461846E9
:1043A00011F0DEFB034658461946069311F0CEFA8B
:1043B000069BC8F804001946584611F0C9FA394658
:1043C000C8F80800504611F0CBFB31460746484676
:1043D00011F0C6FB0146384611F0B8FA624E634B45
:1043E0000027C8F80C00FF2130461B221F7014F074
:1043F00070FB30464E4A5E4B1268012112F0020FEC
:1044000018BF717019701FBF032119700221B1709C
:104410003770570741BF19784E1C1E70032648BFDE
:10442000465412F00A0F0CD01A7804218154511C02
:10443000C9B205264654D11C02321970D2B20621E7
:104440008154049A11688E0641BF1A78561C1E705A
:10445000072648BF86540A0608D51A7809268654C6
:10446000961C01321E70D2B20A2686546E79082E2E
:1044700001D00E2E04D11A78571C1F700B278754B9
:104480001A7811F4803F4FF00C0E00F802E002F1B0
:1044900001071CBFDFF8D8E00232FFB21F701FBF58
:1044A0008EF80020304A4FF00E0E02F807E04A075F
:1044B00048BF1A784FF0120E41BF571C1F701027CB
:1044C00087541A7811F4806F02F10107FFB21F7050
:1044D00000F802E00ED095F814E2BEF1000F09D00A
:1044E000DFF88CE002328EF800201F4A4FF0130EE6
:1044F00002F807E08F0541BF1A78571C1F70152777
:1045000048BF8754182E37D11A7816278754571C5E
:10451000FFB24FF0170E00F807E0D71C0232D2B2FC
:104520001F70865428E000BFDC2D0020000C0140E5
:10453000AC1700207806002090060020D827002025
:1045400035FA8E3CD4270020140000208C27002050
:10455000E026002090270020EC270020DC27002008
:10456000F0270020E0270020A90E00204A27002085
:10457000A80E0020C42700200A0341BF1A78561C49
:104580001E70192648BF8654CF0541BF1A78511CAA
:1045900019701A2348BF8354002198229D4814F0B3
:1045A00098FA10F0DEF99C4A9C4BB5F84E111A604F
:1045B0009B4BB5F8960119809A4900230B808B70AC
:1045C00099490A60994A81B21370994A22F81310E6
:1045D0000133122BF9D1974F3B68DE0458BFB5F871
:1045E0009C111B07D18040F1C48095F89031062BB7
:1045F00000F2B980DFE803F004070E39547373004A
:1046000045F2F05201E042F6F8228B4B1A8010F08E
:1046100044FAA7E042F6F822874B1A8011F04CFAD0
:10462000864911F09DFA864911F090F911F084FC49
:104630000023844A42F823000133122BF9D1824A25
:10464000824940201160824A137005F00FFF002854
:1046500000F0898001234FF0070990F90000402104
:104660008DE808027B4A7C4B77E042F6F822724BD9
:1046700040201A80794A744B1A60754B10221A70C8
:1046800005F0F4FE00286ED001234FF0000890F9E9
:10469000000040218DE80801714A4FF4E1335CE0ED
:1046A00042F6F822644B40201A806E4A664B1A602C
:1046B000674B08221A7005F0D9FE002853D0012359
:1046C0004FF0000C90F9000040218DE80810664A78
:1046D0004FF4E13305F0FFFFC4F888013FE042F6F4
:1046E000F821554A062B118059494FF00C02DFF88A
:1046F000B4C1DFF8B4E15D4E5D480A700FD000230D
:1047000033708CF800308EF800301B230370594B47
:104710004FF4E1361A70584B05221A700CE0002154
:1047200031708CF800108EF8001021210170514971
:10473000524E0A70504A1370514A434B40201A603F
:1047400005F094FE78B101234FF0000E90F90000BF
:104750008DE8084033464B4A402105F0BCFF00304D
:1047600018BF012028B9082008F004FD464A364B3E
:104770001A603B68364A13F4804F1FBF1221117034
:104780004248314918BF086042F20101194099B10D
:1047900044F6206028499E04088041BF082111701A
:1047A0003B48294948BF0860D80741BF0C21117018
:1047B0003848254948BF08601178043951701906F6
:1047C00040F1B0804FF00008334EDFF8E0904146F2
:1047D00015223248DFF8D8A0C4F88C9186F8018001
:1047E000C6F80480C6F8088014F073F9A9F105032F
:1047F0004046CAF800300AF0FFFD294B02201B6832
:10480000F36005F033FE002854D1802008F0B2FC9C
:1048100080E000BFFC2A00203C110020800D002019
:10482000840D00208C2D00205C2D0020030D002025
:10483000602D002094170020E6060020CDCCCC3F50
:104840000000B044482C002090000020BD4E01081C
:10485000982B002065500108A0860100A94E010890
:10486000B94F0108954E01086D4F01087C250020C5
:104870009F250020572D0020A025002090D0030068
:10488000590D0108710D01081D4F0108ED4E010879
:104890000D4F0108FD4E010894060020F002002093
:1048A000980F0020582D00207D250020A611002003
:1048B000B406002090F805E07378D3490C2202FB7F
:1048C00003125278724504D00133DBB2042BF4D9C1
:1048D00000237370DAF8003072781B7890F90000CA
:1048E000002B4FF00C0303FB021314BF4FF0030E19
:1048F0004FF0010E00225B78CDF800E0019202211A
:1049000005F0E9FEC14B186000283FF47EAF01209E
:104910000AF072FD059B1868BD4B00F5C5721A6060
:104920000AF012FEBB4BBC4ABC4E1360BC4A80333B
:1049300013603B684FF00008DA0386F8008040F10E
:10494000C78009F079FE40F22A3CB64BDFF814B379
:104950004FF001096246184641460593CDF810C054
:1049600086F8009014F0B5F8DBF818104FF0100A34
:1049700041F00801CBF8181018218DF833100321ED
:104980008DF83210A8480CA9ADF830A00CF0F6FC58
:10499000DBF81C10A54841F00201CBF81C10A4491B
:1049A000A44E0968ABF6947BB1FBF0F13088013975
:1049B00020F45C7000FA0AF020FA0AF0308089B224
:1049C0001D20B0853185A6F81490318C21F00101AD
:1049D00001FA0AF121FA0AF13184318CB6F804E0C7
:1049E000308B21F0020120F0730000FA0AF001FA86
:1049F0000AF120FA0AF021FA0AF11FFA8EFE40F0BD
:104A0000600041EA0901A6F804E03083A6F834808A
:104A10003184318B21F0080101FA0AF121FA0AF1FF
:104A200041F008013183B6F844106FEA41416FEA62
:104A3000514189B2A6F84410DBF8A81F41EA0901E8
:104A4000CBF8A81F58460CF0B3FA059B7A49169389
:104A50008023DDF810C01A934FF4807315911B93D7
:104A600058464FF4005315A91E93CDF86480CDF835
:104A70007080CDF87480CDF87C80CDF85CA0CDF846
:104A800060C00CF077FAB3890DA89BB243F40073B1
:104A9000B381DBF8003043F00203CBF800308DF82F
:104AA00034A08DF835908DF836808DF8379010F061
:104AB000C3FB624B03991A68614B43F821200B46F4
:104AC0000133202B0393F4D10EF0F0F80EF0EEF842
:104AD0003B685B0555D5D4F8D0845A4B0420C3F805
:104AE000008005F0C3FC0421C4F8D40405F09AFC4E
:104AF000554B84F8D8040820C3F8008005F0B6FCB4
:104B0000524B0821186005F08DFC514E84F8D904F1
:104B1000002130462C2213F0DCFF8E2373704FF0FF
:104B20007C0AE0234FF07D09F37086F800A086F838
:104B30002B90484E2C220021304613F0CAFF8A23C6
:104B400073701020A023F37086F800A086F82B90D5
:104B5000C4F8DC8405F08AFC1021C4F8E00405F0F8
:104B600061FC84F8E4042020C4F8E88405F07EFCAD
:104B70002021C4F8EC0405F055FC84F8F00409F099
:104B8000EBFB354E4FF000083388322023F0400312
:104B90001B041B0C338033884FF4805A23F03803F6
:104BA0001B041B0C338033880DF154099BB243F076
:104BB000400333809F238DF834308DF835808DF895
:104BC00036808DF8378005F07CFD8DF85580DFF854
:104BD00058800DAA0423C8F814A03046494603F0B3
:104BE000C1FFC8F810A09DF856209DF8553012025C
:104BF00042EA03429DF857301A43184B9A42184B29
:104C000049D03AD830E000BFB498010814250020FC
:104C1000D40D0020D8110020001E0020390C0020E7
:104C20004C25002005030020000C014000366E01D9
:104C3000EC000020000400403404004034980108D7
:104C40003A0C0020A0170020F8170020441800207C
:104C5000C8170020FD1700200038004018BA2000B7
:104C6000040000200010024095498A420CD001F552
:104C70001A4102318A4209D01BE092498A4205D08A
:104C800001318A4207D014E0202200E080221A80FD
:104C90004FF4807202E04FF480721A805A809A8832
:104CA000198812029A604A43DA60012284F8F124DA
:104CB00004E000221A805A809A60DA60DB6813B33D
:104CC0004FEAD328C2464FF0000BC34509DA0BEB7D
:104CD00008067610F002494610220EF0EBF90F2874
:104CE00006DC0AF09BFD4FEACA23C4F8F4340AE05C
:104CF000002359F8232001324CD10133042BF8D181
:104D0000B046B246E1E73B686F4A13F4002318BF90
:104D10000123137005F0AEFC6C4B18606B79052B0A
:104D200002BF6B4B4FF4C8721A806A4B4FF47A7211
:104D30001A80694A137843F008031370674A13789E
:104D400023F00203137040F602033A6813406BB17C
:104D5000634A644B1A60644B03221A70634B01224E
:104D60001A70634A00231380624A1380624B012247
:104D70009B683B60614B1A70614A137863F07F0354
:104D8000137021B0BDE8F08F012E7FF629AA1E46D0
:104D9000FFF7FDB906F1010B5646B2E701200EF010
:104DA000B3F9FEF788BF574B00221A7000B210F01B
:104DB00083FE554910F0D4FE4F4C0646B4F95A0113
:104DC00010F07AFE504910F0CBFE0546B4F95C01B4
:104DD00010F072FE4C4910F0C3FE0446304608F055
:104DE0009FF98046304608F029F90646284608F023
:104DF00097F90746284608F021F90546204608F0AD
:104E00008FF98246204608F019F9414681465046FE
:104E100010F0A6FE41468346484610F0A1FE5146DA
:104E20000590304610F09CFE49460690304610F042
:104E300097FE39460790504610F092FE334C494693
:104E4000206007F1004010F08BFE29466060A560ED
:104E5000069810F085FE0146059810F079FD294668
:104E6000E060079810F07CFE0146584610F06EFD99
:104E70003946206106F1004010F072FE294660615B
:104E8000584610F06DFE0146079810F05FFD294668
:104E9000A061059810F064FE0146069810F058FDD8
:104EA0004146E061384610F05BFE2062FFF77DB8B6
:104EB000012E7FF695A9164B00261870FFF76EB9E4
:104EC000152020001740EF00A8180020B806002089
:104ED0005E270020FC2D0020B0170020002E0020AF
:104EE0002E11002098170020FC170020E000002061
:104EF000780E00207A0E0020B40F0020380C00201D
:104F0000DC2D00204400002035FA8E3CA82500202E
:104F1000FE2D002093492DE9F04F0A68924C02F5CE
:104F20009C4320332360914B89B01E788946DFF87B
:104F30006882C6B18E4909688A4240F2EA80013E21
:104F40001E70E6E0D8F80030072D98BF595D894BF8
:104F500088BF29461B6888489847032D0AD904EB67
:104F60004505A8800136844BF5B21A78AA421A4644
:104F7000E8D820E0D8F8002005F10E0302EB830307
:104F80009988DA880028EAD04FF47A73401A584397
:104F9000531A90FBF3F040F6C90300F57A7098427B
:104FA00005DC40F2EE239842B8BF184601E040F617
:104FB000CA0080B2D3E742F20107704B1B681F4062
:104FC000B7FA87F794F828307F0923B92FB1664BD9
:104FD00093F8293002E0012300E03B4692F800A05C
:104FE00094F82B200326B2FBF6F60F2106EB4606BB
:104FF00084F82A10961BD8F80010DFF8A0B1F6B29A
:10500000002555454DDA1BB15D4830F8150000E02C
:105010001846B1F814E0864503D8B1F816E0864585
:1050200015D2E8B203920291019310F08FF8032D8C
:10503000DFBF4FF0010E94F82AC00EFA05FE2CEAED
:105040000E0E019B0299039AD8BF84F82AE007BB91
:1050500094F874E02BF81600BEF1000F06D1022A76
:1050600017D941484FF0010E80F874E0BBF800E01A
:10507000BBF802007044BBF804E07044DFF820E1A4
:1050800080B22EF8150000B24FF0030E90FBFEF038
:1050900080B2DFF8FCE00BF1060B2EF815000135AD
:1050A000AFE794F82A203748A2F10F014A424A415B
:1050B00084F88E20344B6AB1344A1268520109D404
:1050C0000268D9689A60521AC82A1DD9012283F849
:1050D000212019E002689868DA605B68121A9A4227
:1050E00088BF294B4FF0000184F8281088BF83F84F
:1050F00021100025554507DAE8B210F027F8244BB7
:1051000023F815000135F5E794F82B30013384F8C6
:105110002B301A4E3368DB0405D51C4B1B68DF07A8
:1051200001D40FF033FAD8F80020D9F80070907A43
:10513000002837D01649137B013831F810001BB115
:10514000C0F53B60083080B200B2A0F57A70B0F5CF
:105150007A7FA8BF4FF47A7020EAE07010F0ACFCC0
:105160000C4954E0E02D0020D80C0020882D0020B0
:10517000842D002090000020982B00209417002000
:10518000DC0C0020980F00208C2D0020A40E0020A5
:10519000602D002000007A445C2D0020040D0020CA
:1051A0004E0D002033681D043AD5D4F89030924D4E
:1051B000FB1A002B34DB07F59C432033C5F89030F5
:1051C0008E4BD27A59798E4B33F8113095F8941072
:1051D0009BB293FBF2F3013101F00F0285F89420AA
:1051E0002A4482F895300346864A825C0130134493
:1051F00010289BB2F8D11BB293FBF0F000B26428E8
:10520000A8BF642020EAE07010F056FC7E4910F040
:105210005BFD7E4910F0A4FC10F08EFE7C4B1880E4
:1052200033687C4D13F4807F00F00D817A4BDFF8FA
:10523000EC919F4205D999F8022012B9012289F810
:10524000022099F80220002A00F0FD80734A95F8A8
:10525000008092F82170724A781E92464742116887
:105260004741002FC1F38063C8F38008019314BF46
:105270004FF0000B4FF0030B99F82020052A00F2A5
:10528000DC80DFE802F0034E537988A5B8F1000F07
:105290003AD0D4F8A800B4F8AC1005F084F901288D
:1052A00009D16049604A09681268C988642000FB16
:1052B0000122C9F81020019B6BB15A4A1268127979
:1052C0004AB107F04DFB032289F820204FF47A728F
:1052D000C9F81C20D0E7002F40F0AF80524AD9F81F
:1052E000101010684D4A88420AD9029207F038FB24
:1052F000029A032182F8201040F6B831D161BBE751
:10530000012182F82010B7E7019B4FF4806013B1B0
:1053100007F020FF01E007F00DFF0022C9F8102080
:105320008BE0002F49D107F01BFBA5E727B1052231
:1053300089F82020012000E03846B8F1000F0CD099
:10534000D4F8A8204FF0020BD189384A118051803F
:105350009180344909684988D180334A1168D9F865
:105360001420914202D8B8F1000F63D147F23052B5
:10537000C9F81C20032221E02A7842F002022A7098
:105380000FF004F9284AD9F81C1012680A44C9F829
:105390001820042212E0244A9FB11168D9F818207D
:1053A00091424AD9224A12781AB9DAF80020D10774
:1053B00043D42A7822F002022A70052289F820209C
:1053C0005AE71268D9F81C100A44C9F8182034E0CA
:1053D0001449154A09681268C988642000FB012233
:1053E0004FF48060C9F81020002289F8202089F845
:1053F000032007F09FFE3FE7D80C0020CC250020BB
:10540000DC2500206D0D00200000C84200C07F4454
:10541000000F0020002E0020404B4C008C2D00205F
:10542000A40E0020CC1D0020980F0020602D00202D
:105430000200002000287FF41FAFBBF1000F02D054
:10544000584605F05FFA904F07F5C470B7F84E1153
:1054500005F0A9F80197834668B907F077FA8B4BF6
:105460000022C3F800B0C3F804B0C3F808B0884BFA
:105470001A605A609A602B785A0736D53368DB0673
:1054800033D5844B1B78DF062FD4834B1B789BB11D
:10549000019B93F8E031BBF1000F15D17BB17F4B3D
:1054A0001A68D4F8B0309B1A002B08DA0FF06EF8A7
:1054B0007B4B83F8B4B018E0BBF1000F0DD1102086
:1054C00005F020FA01230EE03BB1744A4FF47A71E3
:1054D000126801FB0323C4F8B03094F8B43023B150
:1054E00005F0F8F9002384F8B430019B93F8DEA1AD
:1054F00093F8DF11B3F898E1B3F89AC10023184686
:10550000684F800837F9132001337245C4BF60F03B
:105510007F00C0B26245B8BF40F04000042BB946DE
:10552000EED194F8B5305E4A834205D192F8B63098
:10553000F92B04D8013300E0002382F8B630564B33
:1055400084F8B5001A78584F9846E2B93B68D807F6
:1055500008D5BBF1000F16D12B78D90713D50EF063
:105560005FFE10E02B785A070DD54D4B93F828308D
:105570004BB14E4BDB7833B911B10FF007F802E0B5
:10558000BBF1000FF9D094F8B630454A142BDFF880
:1055900034B140F0A98098F800301AF1000A18BF21
:1055A0004FF0010A6BB392F8B5305F2B11D12B7815
:1055B00003F0040303F0FF0113B10EF0E7FF08E06E
:1055C0000B200391029205F09DF9029A039982F84B
:1055D000B610BAF1000F14D094F8B5307D2B10D16D
:1055E0002B7803F0040303F0FF0213B10EF0CEFF9B
:1055F00007E00B20029205F085F9294B029A83F807
:10560000B6202B7803F0040303F0FF01002B6BD1CD
:1056100094F8B530224A572B10D1254B4FF47A72AB
:105620001A8033681B0601D509F0DEFF214B1B6889
:1056300013F0080358D1204A138055E03068400722
:1056400016D55A2B14D11D4B187820B119701C4B4C
:1056500001221A7048E092F8B73083F0010382F813
:10566000B7300BB10C2000E00D2005F04BF93BE00A
:105670005D2B00F016855B2B00F015855E2B23D18A
:10568000032000F011BD00BFB40F002084260020CD
:10569000841D0020B017002002000020980F002079
:1056A000D80C0020602D0020A40E00208C2D00209E
:1056B000FC2D0020AC170020A80F00208927002017
:1056C0008A270020E00E0020562B01D107F0F4FFBE
:1056D00098F80030002B00F0FD8494F8B5306F2B63
:1056E00040F0F2840EF09CFD33685B0732D594F8ED
:1056F000B730A3B12B78580711D5019BB9F9062013
:10570000B3F898319A420ADD3B6813F0010301BFF8
:10571000AC4A32211180AC4A08BF82F8B7303B68EE
:10572000D9030AD5A94B1A782AB9A94A127812B90D
:10573000A44A3221118001220BE0A54A13784BB113
:105740002B7803F0040303F0FF011BB9A14B117088
:1057500001221A70DBF8009000233B6009F17B08FE
:1057600009F1CB0A98F8002098F8013018F8010CDC
:105770009A420BD2414604F0E1FE38B118F8022CEF
:10578000012303FA02F23B6813433B6008F104086B
:10579000D045E7D1904B1B784BB1904BDFF854923A
:1057A0001A68984612F0020F40F037832FE309F190
:1057B000CA0709F589783A787B7817F8010C9A427C
:1057C00025D2394604F0BAFE08B397F804E00C215C
:1057D000BB7801FB0E41824A013B03EB43031344B8
:1057E000D1F8BC2097F803909A4277480FD0C1F8BF
:1057F000BC30002390F8E820C1F8C030012303FA40
:105800000EF322EA030381F8B89080F8E8300637F7
:105810004745D0D1734BDFF8E0A1D3F80080724B3D
:105820004FF0000B1B68029394F828300393DAF8CA
:105830000030002B00F0E28293F80090B9F1000FE5
:1058400000F0DC82DAF8042002998A1A002A0CDBC4
:1058500001F5FA72CAF8042094F8E810012202FA5D
:105860000BF221EA020284F8E820039A002A00F0F1
:10587000C5821AF8042C59780432D2B2002940F0BB
:105880007E825A4931F91210594AB2F8962102F132
:10589000C800814201DD9F7814E0C83A914202DAE3
:1058A00099784F420EE094F8E820012303FA0BF3B5
:1058B00022EA030384F8E830029B03F5FA73CAF87E
:1058C00004309BE294F8E83043FA0BF3DA0700F176
:1058D0009582002FCCBF0220012005F039F809F194
:1058E000FF32394B132A00F28182DFE812F01400F4
:1058F00023003200440061008700EC005101B60132
:10590000E90118027F02440055008700EC005101B4
:10591000BE002301880198F8001040460F44FA2F7A
:10592000A8BFFA2727EAE77788F8007004F0ECFDB3
:1059300001201EE098F8011040460F44642FA8BFD4
:10594000642727EAE77788F8017004F0DDFD02207C
:105950000FE098F8031040460F44642FA8BF642757
:1059600027EAE77788F80370D3F8EC1004F084FD99
:1059700003203946D0E198F805100D2039446429F8
:10598000A8BF642121EAE17188F8051004F052FEF5
:10599000B9F10D0F00F02A8298F804100E20394456
:1059A0006429A8BF642121EAE17188F80410B3E1F9
:1059B00098F806100520394481F3080188F806108C
:1059C000AAE100BF70270020D80C00208827002003
:1059D000892700208A270020012E0020A40E002005
:1059E000C89C0108040F0020980F0020602D0020A3
:1059F000B40F0020AC170020940D0020D3F8F03035
:105A00001A78022A22D13846049310F055F8A94991
:105A100010F05AF9049B596A05930FF099FF002181
:105A2000049010F03BFA059B48B9049AA14910462E
:105A300010F052FA049A059B10B19E4A00E0002231
:105A40005A620F20114604F0C9FD0AE099780F2030
:105A50003944C829A8BFC82121EAE171997004F02E
:105A6000E9FDB9F10F0F00F0C181934BD3F8F0902D
:105A700099F80030022B1AD1384610F01DF88D49E4
:105A800010F022F9D9F820100FF062FF002107462C
:105A900010F004FA30B93846864910F01DFA10B1FA
:105AA000844F00E00027C9F82070122057E199F8D0
:105AB000011012203944C829A8BFC82121EAE17188
:105AC00089F8011028E1D3F8F0301A78022A22D19F
:105AD000384604930FF0F0FF764910F0F5F8049B78
:105AE000196B05930FF034FF0021049010F0D6F9E4
:105AF000059B48B9049A6F49104610F0EDF9049AD5
:105B0000059B10B16B4A00E000221A631020114679
:105B100004F064FD0AE0197B10203944C829A8BFAD
:105B2000C82121EAE171197304F084FDB9F1100F65
:105B300000F05C81604BD3F8F09099F80030022BB4
:105B40001AD138460FF0B8FF5A4910F0BDF8D9F80D
:105B50002C100FF0FDFE0021074610F09FF930B920
:105B60003846544910F0B8F910B1524F00E0002700
:105B7000C9F82C701320F2E099F80B101320394467
:105B8000C829A8BFC82121EAE17189F80B10C3E038
:105B9000D3F8F0301A78022A22D1384604930FF055
:105BA0008BFF464910F090F8049BD96B05930FF0DA
:105BB000CFFE0021049010F071F9059B48B9049ABA
:105BC0003C49104610F088F9049A059B10B1394AF7
:105BD00000E00022DA631120114604F0FFFC0AE025
:105BE000997D11203944C829A8BFC82121EAE17153
:105BF000997504F01FFDB9F1110F00F0F7802E4BDD
:105C0000D3F8F09099F80030022B1AD138460FF0F3
:105C100053FF2A4910F058F8D9F838100FF098FEC1
:105C20000021074610F03AF930B93846214910F002
:105C300053F910B11F4F00E00027C9F83870142045
:105C40008DE099F8151014203944C829A8BFC8213F
:105C500021EAE17189F815105EE0D3F8F09099F827
:105C60000030022B1AD138460FF026FF114910F0F0
:105C70002BF8D9F828100FF06BFE0021074610F022
:105C80000DF930B938460B4910F026F910B1094F1B
:105C900000E00027C9F82870092060E099F8031097
:105CA00009203944C829A8BFC82121EAE17189F82F
:105CB000031031E00000C842D80C002000007A44F4
:105CC000D3F8F09099F80030022B1AD138460FF033
:105CD000F3FEBB490FF0F8FFD9F834100FF038FE8F
:105CE0000021074610F0DAF830B93846B44910F010
:105CF000F3F810B1B24F00E00027C9F834700A2061
:105D00002DE099F80D100A203944C829A8BFC821F0
:105D100021EAE17189F80D1004F08CFC66E0D3F8FB
:105D2000F09099F80030022B1DD138460FF0C4FED8
:105D3000A4490FF0C9FFD9F840100FF009FE002167
:105D4000074610F0ABF830B938469D4910F0C4F85A
:105D500010B19B4F00E00027C9F840700B20394676
:105D600004F03CFC42E099F817100B203944C82994
:105D7000A8BFC82121EAE17189F81710CCE70129F1
:105D800034D19878904B33F91230B3F5617F05DB4D
:105D900040F633029342A8BF134601E04FF461730B
:105DA000B9F10C0F22D14FF4966292FBF0F0A3F5FB
:105DB000617393FBF0F3854ADFB21378BB4215D0D1
:105DC000042F34BF3B4602231370019A09FB0323BF
:105DD0007F4A03F2AE73136007F0A4FA48463946CF
:105DE00004F028FC781CC0B204F0B2FD94F8E8205E
:105DF000012303FA0BF3134384F8E8300BF1010B92
:105E0000BBF1040F0AF10C0A7FF411ADC5E433684D
:105E1000DB0511D56F4BDB7873B1D9F800309F07E4
:105E20000AD56D4B1B8813F001070AD106F08EFDD1
:105E3000012007F08FF904E0012007F07BF901232E
:105E400000E00023D8F8002050070DD563B10120F1
:105E500007F070F9604B1B88990708D406F076FDAF
:105E6000022007F077F902E0022007F063F9D9F881
:105E7000003013F00A0F29D0D8F80030DA060BD51D
:105E8000554B1B885B070AD4042007F063F9534B7A
:105E90001B88A4F8F43002E0042007F04BF9D8F88E
:105EA00000309F0607D54C4B1B88580606D440206F
:105EB00007F050F902E0402007F03CF9D8F8003034
:105EC000590642BF454B1B88A4F8F630D9F800307C
:105ED0009A0609D4D8F800301B0540F1B2804FF47F
:105EE000807007F037F9B0E03D4BDFF8EC901B789D
:105EF00013F0020F53D03B4B1B78042B4FD9D8F82B
:105F0000003013F4007A0FD0B9F80030DF063AD42D
:105F1000102007F01FF9202007F00CF93248011D6E
:105F200009F0CCFA02232AE0B9F8007007F0100754
:105F3000BFB22FB1102007F0FDF8012784F8F8A0B8
:105F4000D8F80030580512D5D4F8FC3027495A89C2
:105F5000B1F90030002BB8BF5B42934207DAB1F9C8
:105F60000230002BB8BF5B429342C0F2F580B9F813
:105F70000030990608D5202007F0DCF8002384F8CB
:105F8000F830012700E0002794F8003193BB0E2081
:105F900004F0B8FC164B012283F800212AE0B9F87E
:105FA000003003F03003002B94D0102007F0C2F82B
:105FB000202007F0BFF8002384F8F8301DE000BF70
:105FC0000000C84200007A44602D0020AC28002068
:105FD000040F00208C2D002074180020A80F002032
:105FE000B0170020B61700200C0F0020AC0F0020C7
:105FF000D80C0020002F3FF46DAF00221446634BF5
:10600000002023F81400624B191D03F10A0721F840
:1060100014000021D15117447860B96023F81400AE
:1060200003F132075A33D151D150174413447860E9
:10603000B960586099601432002C7FF44BAF012492
:10604000DDE74FF4807007F075F8524B5A791C4623
:10605000082A01D00E2A02D1402007F06BF83368DD
:106060005A0540F18F8094F814321BB92B7813F045
:10607000040F03E0D8F8003013F4002F0AD0464B89
:1060800000221A703C200EF051FD00287AD00DF04D
:10609000F9FDF7E708F060F909B0BDE8F04F0EF040
:1060A00060BC012000E002205FFA80F8019A08F14C
:1060B000FF3382F8AC3707F08FF807F057F9404606
:1060C00004F046FCFFF710BBBAF1000F02D07E2BA4
:1060D0003FF408AB94F8B530972B05D12F4B4FF414
:1060E000C8721A80FFF700BBA72B06D12C4A137881
:1060F00043F004031370FFF7F7BA0022BB2B07929B
:1061000001D1022303E0B72B04D14FF6FE73ADF8A3
:106110001E300AE0BE2B01D1022304E0BD2B7FF428
:10612000E3AA4FF6FE73ADF81C30DBF80030BDF883
:106130001C10B3F858200A44A3F85820BDF81E10CC
:10614000B3F85A200A44A3F85A2007F0B5FA0023FE
:1061500084F8B630FFF7C8BAB9F800309B063FF5AF
:1061600013AF202006F0F6FF0E4B0F481A685B684D
:10617000011D4360026009F0A1F90C4B012783F86F
:10618000F87001E709B0BDE8F08F00BFF82D0020DE
:10619000DA0D0020B40F00209D2B00205E27002088
:1061A000B0170020B8170020140F0020D80C0020D2
:1061B000BA4B2DE9F04FB3F90610B94B91B01F68F7
:1061C00001937A8991420EDBB1F5FA6FFC79BFBF7A
:1061D0008B1A6343A2F5FA6493FBF4F4ACBFC4F1E9
:1061E0006404643400E06424AE4BAF4A1868B2F82B
:1061F00096A1054692F95E21049092B2059202930F
:10620000002240F2E630A54B4FEA420B33F9123040
:106210000393CAEB030303F2F316864203D8002B61
:10622000B8BF5B4201E04FF4FA73022A049E4FF0BC
:1062300064002FD096F811E1BEF1000F04D0734531
:10624000CCBFCEEB0303002393FBF0FCDFF8A0E20E
:106250006FF063093EF81C8009FB0C390CF1010C4E
:106260003EF91CE00FFA88FCCCEB0E0E0EFB09FE8B
:106270009EFBF0FE8D4EC64426F80BE0BE18367924
:1062800073438B4E93FBF6F364339BB2634393FBF0
:10629000F0F02DE096F812E1BEF1000F04D0734546
:1062A000CCBFCEEB0303002393FBF0F0DFF82C828E
:1062B0006FF0630C0CFB003938F910E0013038F94D
:1062C0001000002BCEEB000000FB09F999FBFCF954
:1062D0000598CEEB090909FB00F97448B8BF5B4289
:1062E000A0F80490B8794343714893FBF0F0643010
:1062F0006B784FF0640E434393FBFEF36D4E022A1E
:10630000B354EB7A6C4E00FB03F393FBFEF3B354F0
:106310006B7D664E00FB03F090FBFEF0674B9854DC
:10632000674B0FD183F802E0039B53450EDB5E4CB5
:10633000B4F89821914215DBB1F5FA6FA8BF4FF47C
:10634000FA6110E09C54039B534504DA36F80B3095
:106350005B4226F80B300132032A05F101057FF478
:1063600050AFE4E71146891A4FF47A735943C2F5E6
:10637000FA62B1FBF2F1642791FBF7F2DFF874E106
:106380006FF063033EF8120003FB021101323EF985
:10639000122003B2D21A514391FBF7F30344F38066
:1063A000484B424D1B885F063BD5474A474B1088F8
:1063B0001B88181A00B20FF07FFB45490FF0D0FB85
:1063C000074606F0ADFE8046384606F037FE074623
:1063D000B5F902000FF070FB8146B5F900000FF02F
:1063E0006BFB414682460FF0BBFB3946834648466D
:1063F0000FF0B6FB014658460FF0A8FA0FF076FDF5
:106400004146288048460FF0ABFB3946804650464F
:106410000FF0A6FB014640460FF09AFA0FF066FD1A
:1064200068802C4F3B68980740F19F8045F2072118
:10643000294B2A4D1A686B69D31A8B4240F3958019
:106440006A610BF0D9F8264BDFF8AC901A789846C1
:10645000032AB9F8003051D10A2B59D9002328203A
:1064600088F8003004F02DF90BF0C6F81D4B1888A1
:106470000BF0ACF81C4B1A68D37890FBF3F00130AA
:1064800008281A4BA8BF08201870537980B24343DC
:106490002B831379584368833AE000BF602D0020B6
:1064A000040F0020E00E0020B40F0020AC0F0020ED
:1064B0000CFEFFFF901D00206E0E0020A41D00208A
:1064C0007026002074180020CE0D0020A80F002098
:1064D00035FA8E3C94170020E02D0020600E00203D
:1064E000FC170020E425002098170020E000002081
:1064F0009A180020821800209C1700200A2B07D829
:1065000003239D4A88F80030002313702B836B838C
:1065100098F80030994A012B0CD002D3022B1BD0E3
:1065200023E02A8BB9F800309A421EDD012388F857
:1065300000300FE0B9F800106B8B8B4202DD0223B4
:1065400013700FE08E4B1B8B0133994202DD002349
:1065500013700AE0082006E06B8BB9F800200133C5
:106560009A42E3DC072004F0CDF93D68290573D594
:10657000844B834F1B68FA69C2EB030845F207227C
:10658000904569DDFB61804BB6F906B0D3F8009009
:10659000B4F84E1199F80A30ABF57A7B012B7B4E9B
:1065A00003D042D3022B20D041E0794B396A5A7B89
:1065B000784B082033F8122091FBF0F392B2C91AFD
:1065C0008B183B6293FBF0F3BA8440F6E4429BB233
:1065D0005343B9F80820C2EB13334FF47A72534394
:1065E000B9F9062093FBF2F320E06B4BB9F808A051
:1065F0001B78C6F800A05A0719D5684803F0D3FFE6
:1066000020B915F0100F18BF4FF0000B0BFB0BF368
:10661000322293FBF2F3B9F906205B445A434FF45C
:106620007A7392FBF3F3534400E000233360336842
:10663000D7E90A0103FB08F84FF47A7398FBF3F8E3
:1066400010EB080041EBE8710023C7E90A01544A46
:106650000FF092FC534B1860534E3368DB0427D580
:106660002F0622D5514B1B789D071ED5504B18780D
:1066700004281AD900224F4B0521D718951C4FF03A
:106680000A0E122AD154E9B287F801E004D0B0EB27
:10669000510F2A46EFD800E014215A18322002F890
:1066A000010CFF225A540F2000E00A2004F02AF9BE
:1066B000414D2A68002A56D0404B414F186839682E
:1066C000984681424FD83F4BDFF8049118785168C3
:1066D00008BB01201870B9F80030CB5C5BB31378AD
:1066E000013B00FA03F2D4F8D8371A4201D104F082
:1066F000EBF8354B01221A700EF07AFDB9F8003034
:10670000CBB92B681B78053B012B14D803F0B2FFE3
:106710002E4B18600FE04FF0000A83F800A0B9F884
:106720000030CB5C3BB1504604F0CEF8264B83F8EA
:1067300000A00EF05DFD2B68B9F800205B682449CD
:106740009B5CFE2B02D100230B800CE0FF2B02D1BF
:1067500004F0C0F807E0D8F800000A2505FB0303A1
:1067600001323B600A800C4D2B78580734D5194B09
:1067700008225A6164E000BFE0000020FC170020FE
:10678000600E0020E02D002098170020A4170020A4
:10679000CC250020DC250020002E00203C1100200C
:1067A000407E0500A8170020A40E0020B01700208E
:1067B000B6170020D828002010190020980F0020BC
:1067C0000819002004190020B02D0020802A002084
:1067D0000C190020000C01403268D1075CBF43F067
:1067E00001032B70A94B1B781F075EBF2B7823F08A
:1067F00001032B70D60242BF2B7823F001032B70CC
:10680000A34B1A88A34B1AB1A34A1268900702D46B
:10681000A24A128832B102221A702B7823F00103A7
:106820002B7004E02978C90758BF02221A7003F0C0
:1068300021FF9B4B1B68C01A002801DB0EF0D8FC1F
:10684000984F07F089FD3E78002E00F0AC80964B03
:106850001A689846002A00F04087D8F8000004F033
:10686000D8F8002800F039878F4B904C186804F056
:10687000CDF8092801D03F2852D14FF0000A5546E3
:106880002668DFF8649236B18948D9F8001032469C
:1068900012F06CF910B9CA4605B94D46854B09F19D
:1068A00010099945EFD3EDB1D5F800C0DAF80090A2
:1068B00023681CF803E019F80300704512D15A1C34
:1068C0007B4958B92D2B09D8DFF8E0E1CEF800203C
:1068D0004FF0200E01F803E0885403E001F803E0D4
:1068E0002260E5E723680BB1554510D072480DF0E2
:1068F000BFFA554507D855F8100B0DF0B9FA092025
:106900000DF0AEFAF5E76D480DF0B2FA00262368F7
:106910009E42A2D2664B985D0DF0A2FA0136F6E7D0
:106920002368002B40F0BF86042840F0F5866048BD
:1069300009F0D8FC00F0D1BED8F80000DFF888A13B
:1069400004F067F828B3DAF8000004F05FF8DBF829
:106950000030024693F84810A9BB24286CD10122CC
:1069600083F84820DBF80030DFF880A193F8482056
:10697000062AE1D193F8490000F05AFF8346002827
:1069800000F0B6800DF0CCF9D9F80030002283F881
:1069900048204B4B93F83530002B40F072864C3634
:1069A000982E00F09A86474BF21892F84A10012967
:1069B000F5D1DFF83891F358C9F80020424ACB46A8
:1069C00013609046B8E7012904D14D2814BF002276
:1069D0000222C5E7022904D13C2814BF0022032269
:1069E000BEE703290CD140284FF0000102D983F8FB
:1069F0004810B7E758711971D97198710422AFE73F
:106A0000042906D1997983F849004A409A710522F0
:106A1000A6E70529A6D1587919798842987906D927
:106A200050409871481C18710B441A729AE79042B2
:106A30000CBF0622002293E72B782449580791D4F3
:106A4000232ADAF8003013D1012038701648049157
:106A500003601B48039203631D480DF009FA1748B1
:106A60000DF006FA0499039A0B7843F002030B70B9
:106A7000184B1B681B78934201BF174A174B1A60CB
:106A8000174A04BF174BDA606CE700BFB01700204D
:106A90005E270020B02D0020AC170020FC2D002028
:106AA000B42D0020012E0020C828002048250020F9
:106AB00018250020F0A501087DBC010882BC010852
:106AC000600E0020FC2A002058180020002E002014
:106AD000B2BC0108A02B0020EFBEADDEF04F0020BD
:106AE0000400FA0500ED00E010A40108541800208D
:106AF000DAF8002092F849304C2B00F091845CD8F1
:106B0000332B00F0C88421D8292B00F0388409D811
:106B1000252B00F00F84272B00F01384232B40F04B
:106B2000F785F4E12D2B00F03B8407D82B2B40F0A8
:106B3000EF850DF0C7F8607100F09EBD2F2B00F0BF
:106B40001785312B00F0298500F0E2BD3E2B00F0C7
:106B5000D2801DD8372B00F0D28404D8352B00F01A
:106B60000F8200F0D5BD392B00F0F8833C2B40F0AC
:106B7000CF85DFF86C84D8F800A00DF0A3F88AF870
:106B80000000D8F8003018780BF042FC00F074BD1B
:106B9000432B00F0918406D8412B40F0B9854FF08B
:106BA000000800F07DBC442B00F02C85482B40F001
:106BB000AF8508F071FE00F05FBDD12B00F07B8344
:106BC00020D8CC2B00F01E820FD8C82B62D004D85E
:106BD0004E2B00F0328400F09BBDC92B00F04483A3
:106BE000CA2B00F0928000F093BDCE2B00F02F83D3
:106BF000C0F02483CF2B00F05982D02B00F01383F8
:106C000000F086BDD82B00F014810BD8D32B3BD0DD
:106C100027D3D42B00F08E82D62B40F079854FF00D
:106C200000087CE2F22B00F0D38212D8EF2B40F068
:106C30006F85DFF8AC83D8F800A00DF04DF8AAF806
:106C40005A00D8F800800DF047F8A8F8580000F076
:106C500013BDF32B00F0DB84FA2B00F0018300F06E
:106C600057BD2B7803F0040303F0FF08002B40F01E
:106C700003850DF027F8022884F8AC0740F2D9828A
:106C8000D34B83F8AC87D4E20DF026F8D14B1880B3
:106C900000F0F2BC92F805804FEA5808B8F1120FE4
:106CA00003D90DF03FFF00F0E7BC4FF0000AC245EA
:106CB00007D20DF011F807AB23F81A000AF1010A08
:106CC000F5E742460023434507DA07A931F81300E8
:106CD000C14921F813000133F5E7122A05D0BE4B54
:106CE000002123F812100132F7E7BC4B012283F890
:106CF000342000F0C1BC0CF0E5FF84F8E0010CF09A
:106D0000E1FF84F8DF0100F0B7BCB54B1A68984684
:106D10001278022A6FD14FF00008DFF8C4A208F100
:106D2000080BDAF8003003930CF0CCFF0EF0C0FE35
:106D3000AC490EF0C9FF039B43F82B00DAF800B012
:106D40000CF0C0FF08F10A030BEB830B0EF0B0FE52
:106D5000A5490EF0B9FFDAF80030CBF80400039330
:106D60000CF0B0FF0EF0A4FEA0490EF0ADFF08F14C
:106D70000E0B039B08F10108B8F1030F43F82B0039
:106D8000CBD1B8F1070FDAF800B01AD10CF09AFFA6
:106D90000EF08EFE93490EF097FFCBF84400DAF820
:106DA00000B00CF08FFF0EF083FE8E490EF08CFFCA
:106DB000CBF84800DAF800B00CF084FF8BF84C00F8
:106DC00012E00CF07FFFC3448BF80100DAF800B04A
:106DD0000CF078FFC3448BF80B00DAF800B00CF02D
:106DE00071FFC3448BF8150008F10108B8F10A0FD0
:106DF000C7D100F041BC4FF0000AD8F800B00CF049
:106E000061FFD3448BF80100D8F800B00CF05AFFB2
:106E1000D3448BF80B00D8F800B00CF053FFD344E8
:106E20000AF1010ABAF10A0F8BF81500E5D100F05A
:106E300023BC8046DFF8A8A108F1080BDAF800307F
:106E400003930CF049FF0EF033FE68490EF03CFF4F
:106E5000039B43F82B00DAF800B00CF03DFF08F17B
:106E60000A030BEB830B0EF023FE60490EF02CFFA0
:106E7000DAF80030CBF8040003930CF02DFF0EF08D
:106E800017FE5A490EF020FF08F10E0B039B08F184
:106E90000108B8F1030F43F82B00CBD1B8F1070F6D
:106EA000DAF800B01AD10CF017FF0EF001FE4F49CE
:106EB0000EF00AFFCBF84400DAF800B00CF00CFF3B
:106EC0000EF0F6FD49490EF0FFFECBF84800DAF867
:106ED00000B00CF001FF8BF84C0012E00CF0FCFE4F
:106EE000C3448BF80100DAF800B00CF0F5FEC3449F
:106EF0008BF80B00DAF800B00CF0EEFEC3448BF810
:106F0000150008F10108B8F10A0FC7D1B4E30CF07D
:106F1000D9FE132883463FF6C4AEDFF8C4A0DAF8E2
:106F200000800CF0CFFE002331490C2202FB03123B
:106F3000117A814220D1137808EB8B0888F87930D8
:106F40000CF0C0FE88F87A000CF0BCFE88F87B00DC
:106F50000CF0B8FE274A284B88F87C001A60DAF853
:106F60000000264B00211860793003F00BFB244B06
:106F700080F0010018707FE301331C2BD4D190E620
:106F80000CF0A0FE0B2882463FF68BAE144BD3F8D4
:106F900000800CF097FE03283FF683AE062303FB28
:106FA0000A8888F8CE000CF08DFE88F8C9000CF035
:106FB00089FE88F8CA000CF085FE88F8CB000CF03A
:106FC00081FE88F8CC000CF07DFE88F8CD0053E3FC
:106FD000B40F0020CC0D0020902C0020600E00206B
:106FE000E00E0020000020410000C84200007A446A
:106FF000349D0108F4100020C40D0020C80D0020AD
:10700000020000205379092B7FF64BAE019BD3F889
:1070100000800CF057FE019B88F80000D3F8008038
:107020000CF050FE88F801000CF04CFE019B642827
:107030001B68A8BF642018710CF044FE019B6428F3
:107040001B68A8BF642058710CF03CFE019BFF2810
:107050001B68A8BFFF2098710CF034FE019B6428C8
:10706000D3F8008028BF642088F807000CF02AFEBF
:10707000019B88F80200D3F800800CF023FE019BEE
:1070800088F80300D3F800800CF026FEDAF8003010
:10709000A8F80A005B790A2B40F2EE82D24BD3F8B3
:1070A00000800CF00FFE88F80800E5E20CF014FEFA
:1070B0006FF4AF6283189BB2C62B98BFA4F89601F9
:1070C0000CF00AFEA4F840010CF006FEA4F8420100
:1070D0000CF002FEA4F844010CF0FEFDA4F8D80167
:1070E0000CF0F0FD84F8ED010CF0ECFD0CF0EAFD85
:1070F00084F8EE010CF0E6FD84F885010CF0E2FD69
:1071000084F892010CF0DEFDB84BD3F800800CF04F
:10711000E3FD00EB80004000A8F856001EE10CF0F3
:10712000DBFDB34B23F8180008F10108B8F1080F94
:10713000F5D1A1E253790F2B7FF4B3AD0CF0C2FD72
:10714000072880463FF6ADAD029BD3F800A00CF0B7
:10715000C3FD0E2303FB08F8029BC244AAF81901E1
:10716000D3F800A00CF0B8FDC244029BAAF81B01A2
:10717000D3F800A00CF0B0FDC244029BAAF81D0198
:10718000D3F800A00CF09EFDC244029B8AF81F01B8
:10719000D3F800A00CF096FDC244029B8AF82001AF
:1071A000D3F800A00CF08EFDC244029B8AF82101A6
:1071B000D3F800A00CF086FDC244029B8AF822019D
:1071C000D3F800A00CF092FDD044C8F8230153E29C
:1071D0000CF078FD0F2880463FF663AD0CF072FD91
:1071E000C8EBC80804EB080383F8D00003F1D0080B
:1071F0000CF068FD88F801000CF064FD88F80200CE
:107200000CF060FD88F803000CF05CFD88F80400C9
:107210000CF058FD88F805000CF054FD88F80600C5
:1072200003F0C2FD28E22B785B0700F125820CF009
:1072300089F805F0D1FF06F099F81DE22B78580780
:1072400000F11A826B4B4FF4C8721A8014E22B784B
:10725000590700F11182684A137843F0040328E0CB
:107260002B785A07E5D553E20CF02CFD624B1A78C7
:1072700010B142F0020201E022F002021A700CF09A
:1072800021FD5E4BDFF8948118700CF02FFDC8F8DB
:1072900000000CF02BFDC8F804000CF01DFD584B4D
:1072A00018800CF019FD574B574A1880137843F09B
:1072B00002031370E0E10CF005FD03900CF016FDE5
:1072C00083460CF013FD82460CF010FD80460CF056
:1072D00003FD0CF001FD0CF0F5FC039BA3B94B4B37
:1072E0001020C3F800B0C3F804A005F023FF424A01
:1072F000137843F001031370B8F1000F00F0BC8164
:10730000434BC3F80080B7E1102B40F0B581414BEF
:10731000C3F800B0C3F804A0B8F1000F02D03C4B92
:10732000C3F800803B483C4B0222011D1A7008F054
:10733000C5F8A1E1A0600CF0D9FCA3681843A060D7
:107340009AE10CF0C9FCA4F858010CF0C5FCA4F8B3
:107350005A010CF0C1FCA4F85C018DE10CF0B2FC08
:1073600084F87A010CF0AEFC84F87E010CF0AAFCE3
:1073700084F87D010CF0A6FC84F87F017CE10CF020
:10738000ABFCA4F880010CF0A7FCA4F882010CF07F
:1073900099FC84F884010CF09FFCA4F886016BE151
:1073A0000CF090FC84F890010CF096FCA4F89A0183
:1073B0000CF092FCA4F896010CF08EFCA4F8980155
:1073C0000CF080FCDAF8003084F891015B79082B2E
:1073D00040F252810CF080FCA4F89C010CF07CFC83
:1073E000A4F89E0148E100BF040F0020E00E002039
:1073F000AE2800205E270020B0170020B61700201E
:10740000B4170020B21700200A0F00200C0F002034
:107410001C0F0020140F0020D00D0020B8170020F2
:107420000CF050FC84F8D6010CF04CFC84F8D70129
:107430000CF052FCA4F8D8011EE192F80580032359
:10744000B8FBF3F8B8F1120F3FF62BACDFF8DCA372
:107450004FF0000BC34580F00F810CF033FC8AF82D
:10746000A0010CF039FC40F2ED23984205DD40F616
:10747000CA039842A8BF184601E040F2EE20A0F2ED
:10748000EE20192390FBF3F00BF1010B8AF8A10118
:107490000AF1020ADEE70CF015FC84F89201EBE039
:1074A0000CF010FC04EB080308F10108B8F1080F18
:1074B00083F88801F4D1DFE00CF004FCC4F808B0D4
:1074C00060710CF013FCA3681843A0600CF0FAFB89
:1074D00084F890010CF000FCA4F858010CF0FCFBBF
:1074E000A4F85A010CF0F8FBA4F85C010CF0F4FBD2
:1074F000A4F880010CF0F0FBA4F88201BCE0537901
:107500004FF0070AB3FBFAF2C2EBC2029A1A12F06A
:10751000FF0F7FF4C6ABB3FBFAFA0AF1FF3A5FFA4A
:107520008AFABAF1FF0F00F0A7800CF0CBFB5FFAEC
:1075300080FB4FFA8BF002F061FF804600283FF499
:10754000B0AB80F800B00CF0C7FBA8F802000CF05C
:10755000B9FB88F804000CF0B5FB88F805000CF0C6
:10756000B1FB88F807000CF0ADFB88F80600D4E703
:10757000DFF8B88208F1400A0CF0AEFBA8F8A402CC
:107580000CF0A0FB88F8A6020CF09CFB08F10408A4
:1075900088F8A302D045EFD16EE00CF093FB1F28D2
:1075A00080463FF67EABD9F800305B79082B7FF43C
:1075B00078AB0CF091FB08F1880804EB880800F028
:1075C0003F00A8F806000CF087FBB8F806308001F1
:1075D00000F4FE501843A8F806000CF073FB0001FD
:1075E00088F804000CF06EFB98F8043000F00F00EF
:1075F000184388F804000CF065FB88F8050007F0D4
:107600001BF839E0764B012283F8352034E00CF08A
:1076100059FBFF2882461BD100238DF81B309DF8B3
:107620001B30052B28D89DF81B006E4A9DF81B3097
:10763000012102EBC3035B6852F83000994089B224
:10764000482206F057FD9DF81B300133DBB2E4E71A
:1076500005283FF626AB00200CF086FB0CF060FB03
:10766000D8F8000003F0CCF918B9322003F029F85B
:10767000F6E7504606F04CFD00200CF075FBFFF7D6
:1076800081B9594B985903F0BBF918B9322003F06E
:1076900018F8F6E703F048FB05F074FD534A544B25
:1076A000DA60FFF77CB90C2838D00A283FD1514D59
:1076B00051480CF0DDFB2846232111F040FA08B1B7
:1076C000401B20602368002B54D14A4800213022FF
:1076D000236011F0FEF93B781BBB484B1B689B06EF
:1076E0000FD5474B3E491B688A6B9A1A002A08DB64
:1076F000444A1278042A82BF03F5123303F5F87363
:107700008B63414B9B68002B67D04048984764E0EF
:107710000DF008FAFFF736B90C2804D13C480CF0FC
:10772000A7FB3C480DE07F2812D1FFF796B80D2843
:10773000BDD07F2809D12F4A013B00213648236064
:10774000D1540CF095FBFFF788B82F2B3FF685A896
:10775000A0F12002D2B25E2A3FF67FA813B92028FA
:107760003FF47BA85A1C2260224AD0540CF078FBCC
:10777000FFF773B85A1EA95C202901D11346A2E76E
:107780001C4A00212360D154244B254DD3F800A07E
:10779000D5F800B0DFF85C90584611F0DEF90646E7
:1077A00059463246484611F0E1F91E4A28B919F8FF
:1077B000063053445B785B0703D010359542E7D31E
:1077C00006E0954204D2701CEB684844984702E0FA
:1077D00015480CF04DFB002377E711B0BDE8F08FA2
:1077E000600E002040C00108FC2A00200400FA05B9
:1077F00000ED00E018250020B7C70108AC170020F5
:10780000E02D0020B6170020E0260020AA0F00205F
:1078100087BC010882BC0108AEBC0108F40000204E
:1078200010A40108F0A5010892BC0108B40F0020C3
:107830002DE9F0474D28A0B0044600F0418600F243
:10784000BD80302800F0A28651D8222800F08D8417
:1078500023D8032800F0068214D8012800F0F6810E
:10786000022840F0168704200CF07EFA43200CF02A
:1078700046FA4C200CF043FA46200CF040FA4C201B
:1078800000F043BE042800F0F681052840F001878F
:107890001A200CF069FA0024FDE1282800F0DE85AA
:1078A00015D8242800F0C585262840F0F286DC4C47
:1078B00006200CF059FAB4F858010CF058FAB4F854
:1078C0005A010CF054FAB4F85C0100F0AFBD2C285A
:1078D00000F0D7852E2800F043862A2840F0D9866C
:1078E00001200CF041FACE4B587900F00EBE3D2835
:1078F00000F0FA821ED8362800F018860BD83228FD
:1079000000F0FD85342840F0C48648200CF02CFAA5
:10791000002500F04CBC3A2800F0BC823B2800F067
:107920001D84382840F0B58604200CF01DFABC4CAC
:1079300000F085BD452800F0998627D8402800F042
:10794000E785422840F0A586B54C10200CF00CFAD3
:1079500060790CF0D4F9A0680CF012FA94F8900158
:107960000CF0CDF9B4F858010CF001FAB4F85A0152
:107970000CF0FDF9B4F85C010CF0F9F9B4F88001F1
:107980000CF0F5F9B4F8820100F050BD472800F082
:107990004B86C0F020864B2840F07B86A04C04200C
:1079A0000CF0E2F994F8D6010CF0A9F994F8D7019B
:1079B0000CF0A5F9B4F8D80100F038BD702800F03B
:1079C000E98200F2E080692800F0428200F2B28091
:1079D000662800F09C8100F2A280642800F0748187
:1079E000652840F056868F4C0B200CF0BDF920889E
:1079F0000CF0BDF9608880B20CF0B9F98A4B1B68B5
:107A0000C3F3C000C3F38002800040EA4200C3F326
:107A100040021043C3F3401240EAC20003F01003D7
:107A200018430CF0A4F9814B1A88636802F008012E
:107A300003F4475949EA010903F4804149EA01097D
:107A400003F4004149EA010903F4803149EA0109DC
:107A500003F4003149EA010903F4802149EA0109EC
:107A600003F4002149EA010903F4801149EA0109FC
:107A700003F0007349EA0303DFF8CC9112F0010F21
:107A800099F8009018BF4FF00208C9F3800908BFA9
:107A90004FF0000843EA090312F0020F43EA08031B
:107AA00014BF4FF0040C4FF0000C12F0040F43EA27
:107AB0000C0C14BF4FF0100E4FF0000E12F0400FE0
:107AC00014BF202700274CEA0E0E12F0100F14BF2F
:107AD0004FF4007600264EEA070712F0200F14BF7D
:107AE0004FF4806500253E4312F4807F14BF4FF4AD
:107AF00000600020354312F4007F14BF4FF40011E2
:107B00000021284312F4806F41EA000114BF4FF0B6
:107B10008063002300201943247A0346E4E06728A9
:107B200000F01D81682840F0B48510200CF01CF98D
:107B3000002484E16C2800F09E8117D86A2800F0A8
:107B4000FC836B2840F0A58505200CF00DF9384B1F
:107B500018880CF00CF9374B18880CF008F9314BE9
:107B600093F86A0000F0010000F0CFBC6E2800F02E
:107B7000958100F2C48106200CF0F6F800200CF08C
:107B8000FFF800F052BC782800F0F68018D874286E
:107B900000F02E830AD8722800F08F83732840F0FB
:107BA000788508200CF0E0F80124BFE3762800F087
:107BB000E48300F256832F200CF0D6F81E4CC5E269
:107BC000A42800F0FF8314D87B2800F06582A02849
:107BD00040F05F850C200CF0C7F8184B18680CF0CB
:107BE000CFF8174B18680CF0CBF8164B186800F05C
:107BF0004CBDF12800F0FC80FE2800F00A84F0283B
:107C000040F04785074C04200CF0AEF8236CB3F825
:107C10005A000CF0ACF8236CB3F8580000F006BC26
:107C2000B40F0020A00E0020AC1700207418002014
:107C30002A1800202C180020039D0108E8F7FF1FD8
:107C4000ECF7FF1FF0F7FF1F002E002003200CF0C1
:107C50008BF800200CF053F820460CF050F80D2063
:107C600000F053BC0CF080F801200CF048F80A201A
:107C70000CF045F8A4E306200CF076F843200CF055
:107C80003EF843200CF03BF833200CF038F8442049
:107C90000CF035F8C9E3AF4B185D01340CF02FF848
:107CA0000B2CF8D10024AC4B185D01340CF027F8F4
:107CB000082CF8D10024A94B185D01340CF01FF8F2
:107CC000072CF8D100F0E3BC07200CF04DF8E720BA
:107CD0000CF015F8A24B58790CF011F800200CF0BC
:107CE0000EF8042000F0D1BCA3420AD29D4A9D5C4C
:107CF000012202FA05F50D421CBF9A4010430133E0
:107D0000F2E70CF03DF8964B93F8AC07FDE3122038
:107D10000CF02AF8944B00241B88B3F5806F8CBFBD
:107D200008250125914B33F91400013490FBF5F03F
:107D300080B20CF01CF8032CF4D18D4CA08C0CF00C
:107D400016F8E08C0CF013F8208D0CF010F8608D14
:107D50000CF00DF8A08D0CF00AF8E08D66E3102011
:107D60000CF002F80024834B185D01340BF0C7FFC0
:107D7000102CF8D100F08BBC70200BF0F5FF002622
:107D80000E2474437A4D01362B6C2344B3F8190149
:107D90000BF0EDFF2B6C2344B3F81B010BF0E7FF56
:107DA0002B6C2344B3F81D010BF0E1FF2B6C234433
:107DB00093F81F010BF0A3FF2B6C234493F82001D1
:107DC0000BF09DFF2B6C234493F821010BF097FFE0
:107DD0002B6C234493F822010BF091FF2B6C1C4475
:107DE000D4F823010BF0CCFF082EC9D100F04FBC12
:107DF00070200BF0B9FF5A4C04F1700594F8D000D4
:107E00000BF07DFF94F8D1000BF079FF94F8D200CD
:107E10000BF075FF94F8D3000BF071FF94F8D400C9
:107E20000BF06DFF94F8D5000BF069FF073494F860
:107E3000CF000BF064FFAC42E0D100F028BC4E4B09
:107E4000185D01340BF05BFF102CF8D100F01FBC63
:107E50004A4D00242878400000F0FE000BF084FF1B
:107E60002B789C4280F01384454B33F814000BF0C0
:107E70007EFF0134F4E73E4C06200BF075FFB4F8AA
:107E80005C000BF074FFB4F85E000BF070FF3D4B2C
:107E90001888CBE204200BF067FFF5E307200BF016
:107EA00063FF394B1888FF28A8BFFF20C0B20BF032
:107EB00026FF364B186880F3100080B20BF057FF96
:107EC0002B4BB3F860000BF052FF254B93F8852144
:107ED0002F4B186822B10A23584380F3100001E0A9
:107EE00000F30F0080B2A1E21D4C02200BF03CFF1A
:107EF00094F8E0010BF003FF94F8DF0105E31C4C5C
:107F00000B200BF031FF636E254618780BF0F7FE5F
:107F1000636E002658780BF0F2FE6B6E144C3344FF
:107F2000187901360BF0EBFE032EF6D1636ED8798B
:107F30000BF0E5FE636E98780BF0E1FE636ED87887
:107F40000BF0DDFE636E58890BF011FF636E187A3B
:107F5000DBE200BFB4B90108C0B9010895B9010856
:107F6000B40F0020A90E002014000020A20F002052
:107F7000A00E0020D00E0020E40E0020982B002040
:107F8000602D0020A80F00209C170020A8170020BB
:107F9000A4170020C04C1E200BF0E6FE236C002529
:107FA0001B78022B65D1236C05F1080253F82200DF
:107FB000BA490DF0D5FD10F099FF80F30800C0B26A
:107FC0000BF09DFE236CB64903EB8503D86A0DF0D8
:107FD000C7FD10F08BFF80F30800C0B20BF08FFEDE
:107FE000236C05F10E0253F82200AE490DF0B8FDE6
:107FF00010F07CFF80F30800C0B201350BF07FFE6B
:10800000032DD0D1072D236C21D1586CA3490DF03D
:10801000A7FD10F06BFF80F30800C0B20BF06FFEFD
:10802000236C9E49986C0DF09BFD10F05FFF80F370
:108030000800C0B20BF063FE236C93F84C000DF007
:1080400037FD10F053FF80F30800C0B20BE02B4463
:1080500058780BF054FE236C2B44D87A0BF04FFE6B
:10806000236C2B44587D01350BF049FE0A2DC9D1F4
:108070000DE3236C2B4458780BF041FE236C2B440A
:10808000D87A0BF03CFE236C2B44587D01350BF065
:1080900036FE0A2DEDD1FAE23C200BF065FE0024FD
:1080A0007D4D04F108022B6C7E4953F822000DF03F
:1080B00057FD10F01BFF80B20BF059FE2B6C794975
:1080C00003EB8403D86A0DF04BFD10F00FFF80B274
:1080D0000BF04DFE2B6C04F10E0253F82200714997
:1080E0000DF03EFD10F002FF013480B20BF03FFEB8
:1080F000032CD5D1072C2B6C16D1586C69490DF087
:108100002FFD10F0F3FE80B20BF031FE2B6C6549B1
:10811000986C0DF025FD10F0E9FE80B20BF027FE03
:108120002B6C93F84C000BE0234458780BF01FFEA7
:108130002B6C2344D87A0BF01AFE2B6C2344587D09
:1081400001340BF014FE0A2CD4D1A0E214F8010F74
:10815000002800F09C820BF0D2FDF7E701200BF025
:1081600003FE4D4B1B6C1878CFE150200BF0FCFD4B
:108170000025494B0C211C6C4B4B04EB850494F8F7
:108180007920013501FB023393F838000BF0B7FD7D
:1081900094F87A000BF0B3FD94F87B000BF0AFFD80
:1081A00094F87C000BF0ABFD142DE2D16FE23A4B5A
:1081B0001C6C062303FB054494F8CE000BF09FFDD6
:1081C00094F8C9000BF09BFD94F8CA000BF097FDE2
:1081D00094F8CB000BF093FD94F8CC000BF08FFDDE
:1081E000013594F8CD000BF08AFD0C2DDFD14EE265
:1081F0004FF0000801260027274B1A7A974227DA0A
:108200000933FA5C00240C236343274D05F1300148
:10821000595C914207D12B44586B10F09EFC82466A
:108220002EB9B14605E001341C2CECD10EE080449F
:108230000CE0D1450ADA0C2303FB04535B6B13F803
:1082400009000BF05CFD09F10109F2E70137D3E702
:10825000002E00F01C825FFA88F00BF085FD0026EE
:10826000C9E70D4D0024287A0BF07EFD2B7A9C4245
:1082700080F00D820D4B0021E65C0C2202FB01F325
:10828000094800F13007DA5DB24211D1034493F896
:1082900038000BF034FD0EE0A00E0020000020415D
:1082A0000000C84200007A44049D0108A90E002085
:1082B00001311C29E1D10134D8E7CF4C16200BF055
:1082C00053FDB4F896010BF052FDB4F840010BF0E9
:1082D0004EFDB4F842010BF04AFDB4F844010BF036
:1082E00046FDB4F8D8010BF042FD94F8ED010BF017
:1082F00006FD00200BF003FD94F8EE010BF0FFFCEF
:1083000094F885010BF0FBFC94F892010BF0F7FC5C
:1083100000200BF0F4FCB94B0A201B6CB3F956306B
:1083200093FBF0F080B20BF022FD88E0E0B2013464
:108330000BF0E5FC092CF9D1A9E110200BF014FD9C
:10834000AF4BB04C187800F002000BF0D8FCAE4BED
:1083500018780BF0D4FC20680BF012FD60680BF06D
:108360000FFDAA4B18880BF002FDA94B18880BF0E3
:10837000FEFCA24BB3F8680058E00BF0A3FC0746E4
:1083800012200BF0F1FC9D4C17B9E66E256F05E04D
:10839000102F19BF00252E46666FA56F38460BF0CB
:1083A000AEFC30460BF0ECFC28460BF0E9FCE06F2D
:1083B0000BF0E6FC00200BF0DAFC00200BF0D7FC01
:1083C0000020A2E08D4D002495F880002E4680000C
:1083D0000130C0B20BF0C8FC95F880000BF08FFCA8
:1083E00096F880309C4280F052818A4D285D0BF0D7
:1083F00086FC05F11003185D0BF081FC05F12003EC
:10840000185D30350BF07BFC285D0BF078FC0134F7
:10841000E6E708200BF0A8FC00200BF0A8FC0020E9
:108420000BF0A5FC00200BF0A2FC00200BF09FFC41
:108430002DE104200BF098FC6F4B986825E194F82F
:108440007A010BF05CFC94F87E010BF058FC94F878
:108450007D010BF054FC94F87F0156E0664C072038
:108460000BF082FCB4F880010BF081FCB4F88201BF
:108470000BF07DFC94F884010BF041FCB4F886010C
:10848000D4E75D4C0C200BF06FFC94F890010BF0DE
:1084900036FCB4F89A010BF06AFCB4F896010BF0C4
:1084A00066FCB4F898010BF062FC94F891010BF0B3
:1084B00026FCB4F89C010BF05AFCB4F89E01B5E719
:1084C000554C564D2078002600EB4000C0B20BF012
:1084D0004BFC237802359E4280F0D98015F8020CBF
:1084E0000BF00DFC15F8010C013600EB800000EBE1
:1084F000800000F2EE2080B20BF039FCE9E70120A9
:108500000BF032FC3C4B93F892010BF0F8FBBEE011
:1085100008200BF029FC0024374B234493F88801F2
:1085200001340BF0ECFB082CF6D1B0E0334B324CAD
:1085300093F8C10004F12005C0EBC000C0B20BF0FD
:1085400013FC94F8F4010023354AD25C904200F009
:10855000A2800C33302BF7D10834AC42F1D196E035
:1085600040200BF001FC244C04F14005B4F8A402B7
:108570000BF0FDFB94F8A6020BF0C1FB043494F859
:10858000A3020BF0BCFBAC42F0D180E0E0200BF08A
:10859000EBFB194C04F18005B4F82602043400F01A
:1085A0003F000BF0E4FBB4F82202C0F386100BF09E
:1085B000DEFB94F8200200090BF0A1FB94F82002E6
:1085C00000F00F000BF09BFB94F821020BF097FBDF
:1085D000AC42E1D15BE0134C0D200BF0C5FB0AF07F
:1085E00031FD0BF08CFB20880BF0CAFBE0680BF030
:1085F000C7FB07F053F848E0B40F0020A00E00209E
:10860000B0170020B8170020B6170020B4170020BC
:10861000B2170020210F0020982B002054110020B9
:10862000A42B0020040000200BF060FB05468420F2
:108630000BF09AFB28460BF0A3FB244BDC6805F1FA
:108640008003A3428CBF641B802407F0E7F8284610
:10865000224669460AF02EFD05460024AC4216DA91
:108660001DF804000BF04BFB0134F7E713200BF06F
:108670007BFB0024164B185D01340BF040FB0B2CE8
:10868000F8D100200BF07CFB00200BF079FB0120DF
:1086900018E0002016E00BF032FBB4F8F6010BF006
:1086A00066FB94F8F8010BF02AFB94F8F9010BF043
:1086B00026FB94F8FB010BF022FB94F8FA010BF077
:1086C0001EFB49E720B0BDE8F08700BF0400002092
:1086D000B4B901088848F0B50368884A9C8AA4B2F6
:1086E000E1B211F0010F32D01988854C21F40061FC
:1086F0000904090C1980198889B241F48061198034
:10870000002111707F490978A9B1517819B97E49C2
:108710000978FF290FD1012151707C49097802297C
:1087200001BF198889B241F400611980217841F0B4
:108730000101198201E1217801F0FE011982724BD9
:108740001B78FF2B00F0F980FF231370F5E08E07F4
:108750003CD5BFF35F8F6D490C78E4B2012C14D186
:10876000684D2D788DB155787DB1198821F48061DF
:108770000904090C1980BFF35F8F198B1988947055
:1087800089B241F4007119801BE01C8BBFF35F8F2D
:108790000C78022C0BD15B4C247844B1547834B162
:1087A000198821F480610904090C1980BFE0097857
:1087B000032906D15349097819B15178002940F0AD
:1087C000B680998889B241F48061B5E04D075BD5E8
:1087D000012191704B49097800293AD0517800293C
:1087E00037D04A494A4D09781C88022911781ED988
:1087F00024F480642404240C1C801E8A2F68CCB2CC
:10880000F6B249B27E5419882D6889B241F40071DC
:1088100019800168A31C13700B8A0134DBB264B2A7
:108820002B558B889BB243F480638B8027E0A4B2E6
:1088300044F400741C802E681D8ACCB2EDB249B29B
:1088400075541B8A611C49B2DBB203347354147033
:1088500015E0517811B92F49097841B1198889B2C9
:1088600041F40071198013780133137007E01988FF
:1088700089B241F480711980204B0121597001683F
:108880000B88DC05FCD458E001F0400101F0FF0644
:108890001E4DF1B114781E491F8AD1F800E0E6B2EE
:1088A000FFB264B2711C0EF80470C9B22F78117057
:1088B00049B2CC1CA74201BF9C8824F480642404E4
:1088C000240C08BF9C802B788B4236D10236167060
:1088D00033E0210631D511784CB2671C1ED00E4E04
:1088E00001313668C9B2345D11701C822C7849B2EE
:1088F0008C4222D11BE000BFC82D0020640F002055
:10890000B82D0020BB2D0020B92D0020C42D002043
:10891000C02D0020BA2D0020BC2D00201249167059
:10892000097819821149097809B9297829B99988EA
:1089300021F480610904090C99800D4B92F9002003
:108940001B780C4901339A420DD100234B708B7870
:1089500033B10268938823F440731B041B0C93808B
:10896000054B00221A70F0BDB92D0020BB2D002050
:10897000C42D0020640F0020C52D0020074B984215
:1089800001D1074A03E0074B984204D1064A1388F5
:1089900001339BB213804FF0FF307047003001402D
:1089A000DA0200200038004058060020044AD3783C
:1089B00023B1012303700023D37070470370704705
:1089C000640F002010B5224C2368998A89B211F4F3
:1089D000706F1EBF1F4A0120107011F4E06F2BD082
:1089E0001A8B9A88890522F480624FEA02424FEA84
:1089F00012429A8020D41A8892051DD41A88D00574
:108A00000FD51A88D105FCD41A8892B242F40072AC
:108A10001A801A889205FCD40F4B18780AF074FB60
:108A20000AE01A8892B242F400721A809A8822F4FC
:108A300040721204120C9A802268938A23F47063A5
:108A40001B041B0C9382054B00221A7010BD00BF43
:108A5000C82D0020C62D002027280020C52D00206D
:108A6000F0B52C4D85B02B79002B51D12A4C2368C1
:108A7000002B4DD01A68294E12B1B1690A43B26178
:108A80009A889868ADF8002002228DF80320694684
:108A900004228DF802200AF0E7F9B369216843F057
:108AA0000103B3610B7D0F2003F0030203F0FC030D
:108AB00003F1804303F580339F689200904027EADA
:108AC00000000E7B9860986806FA02F202439A60F2
:108AD0000B69134A01265361029308230DEB03002F
:108AE00000278DF80D308DF80C708DF80E600CF0AD
:108AF000C1FB236801A85B7D8DF806708DF80430FA
:108B000003238DF805308DF807600CF095FB2E716E
:108B100005B0F0BD640F0020D40200200010024018
:108B20000004014008B5FFF79BFF024B4FF4805251
:108B30001A8008BD1400002092E7064A08B5138881
:108B400001339BB21380044B18780AF0DDFA002041
:108B500008BD00BFA20E002027280020BAE531E79B
:108B6000B8E52FE770B584894FF47A74FBB112B180
:108B70001578013207E0FF2505E04FF6FF76013C4E
:108B8000A4B2B4420DD00689B607F6D5ADB2858140
:108B90000589ED070DD44FF6FF75013CA4B2AC4238
:108BA000F6D1FFF7EBFE003018BF012070BD0120A9
:108BB00070BD8589ADB209B10D700131013BD5E7BA
:108BC00008B540F2E9330289920704D4013B9BB215
:108BD000002BF8D10AE040F2E93389B281810289A1
:108BE000D20706D4013B9BB2002BF8D1FFF7C6FE9B
:108BF00000E08089C0B208BD2DE9F04117468846E3
:108C0000084C094E102540F0800165613046FFF7A1
:108C1000D7FF3046414600223B46FFF7A3FF2561C0
:108C2000BDE8F0810008014000300140184A13B54A
:108C30001388044623F040031B041B0C1380138885
:108C40003B2023F038031B041B0C13801388694658
:108C50009BB243F0400313800622FFF7CDFF9DF83F
:108C600000209DF80130012043EA022323809DF873
:108C700002209DF8033043EA022363809DF804201C
:108C80009DF8053043EA0223A38002B010BD00BF67
:108C900000300140184A13B51388044623F04003FE
:108CA0001B041B0C13801388432023F038031B0480
:108CB0001B0C1380138869469BB243F0400313805A
:108CC0000622FFF799FF9DF800209DF80130012052
:108CD00043EA022323809DF802209DF8033043EAF3
:108CE000022363809DF804209DF8053043EA0223A7
:108CF000A38002B010BD00BF00300140F8B50346AC
:108D00000F46074C074E1025194665613046FFF7A0
:108D100057FF30463946FFF753FF2561F8BD00BFC6
:108D200000080140003001402B4A08B5138880211B
:108D300023F040031B041B0C138013886B2023F0CB
:108D400038031B041B0C43F03003138013889BB2C1
:108D500043F040031380FFF7D1FF962001F0B1FCF0
:108D600003216820FFF7CAFF962001F0AAFC032127
:108D70006B20FFF7C3FF012001F098FC10216A204F
:108D8000FFF7BCFF012001F091FC00216C20FFF7F0
:108D9000B5FF012001F08AFC00211920FFF7AEFF8A
:108DA000012001F083FC10211C20FFF7A7FF012008
:108DB00001F07CFC18211B20FFF7A0FF012001F02F
:108DC00075FC38200121FFF799FF012001F06EFCAE
:108DD000024B01221A7008BD00300140D802002069
:108DE0001F4A13B513886B2023F040031B041B0C90
:108DF00013801388802123F038031B041B0C43F0DD
:108E000030031380138806249BB243F04003138081
:108E1000FFF774FF962001F054FC75200DF1070157
:108E20000122FFF7E9FE9DF80730682B04D0013CD2
:108E300014F0FF04EED10EE00C200DF10701012229
:108E4000FFF7DAFE9DF80730142B04D3182B04D952
:108E5000543B062B01D9002000E0012002B010BDD8
:108E600000300140074B1B681A69074B19685869A5
:108E7000104205D011421FBF5A61044B0122DA7023
:108E8000704700BFD402002000040140640F00209E
:108E90002DE9FF47CC4C07462378002B00F0E881F2
:108EA0006268A368D31A7C2B40F2E281237BA26024
:108EB00001332373002505F12400C34EC0B205F031
:108EC0003BFA06F10E0333F915000CF0F5FDBF4B2C
:108ED000804618880CF0F0FD014640460CF0F4FE88
:108EE000BB490CF03DFE0DF001F8013500B205F074
:108EF00011FA032DDFD1302005F01EFA002005F015
:108F000009FA05F011FA357B15F003051FD141F27E
:108F10008833B2689A420BD9102005F00DFA284622
:108F200005F0F8F9212005F007FA284605F0F2F9D6
:108F3000142005F001FAB4F9140005F0EBF91C2037
:108F400005F0FAF9002005F0E5F905F0EDF9237BCD
:108F50009D4E580740F06981022005F0EDF9B6F901
:108F600016000A2390FBF3F005F0D4F9B6F91E5071
:108F70004FF0050895FBF8F5032005F0DDF9954B5A
:108F8000ADB21B7859070DD506F5D470394601F0FE
:108F90000AFB28B9D6F8003813F0100F18BF0025C7
:108FA00028B205E0D6F804389889B0FBF8F000B292
:108FB00005F0B0F9D4F80038834D9A0740F1858068
:108FC000DFF82882B5F8082898F80030642707FBF6
:108FD00002325B00B2FBF3F3B5F80A6806203601F3
:108FE000B6B246EA0326B6B2C3F303231E4305F026
:108FF000A3F930B205F08EF9B5F80A3898F80010E8
:1090000001339BB293FBF1F201FB1233A5F80A384E
:10901000D5F80C389B7B012B05D1392005F08CF954
:10902000B5F908081AE0B5F808586E235D4315260F
:1090300095FBF6F53A20AEB205F07EF9B6FBF7F5F2
:1090400028B207FB156505F065F93B2005F074F9BA
:10905000A8B2451D0A2095FBF0F000B205F05AF9C0
:10906000282005F069F9D4F810380A2093FBF0F0B5
:1090700000B205F04FF9042005F05EF9D4F8043889
:10908000514E9D894FF6FF73D6F814089842A8BF39
:109090001846ADB10028ACBF281A28460CF00CFDCC
:1090A0004D490CF05DFD064628460CF005FD0146D5
:1090B00030460CF009FE0CF019FF6428A8BF6420AC
:1090C00020EAE07000B205F025F9D4F818383E4ED9
:1090D0009B0640F19F8096F81C389F071DD51120F4
:1090E00005F02AF9B6F81E084FF4F36568433B4BC8
:1090F00090FBF3F000B205F00DF9192005F01CF912
:10910000B6F81E084543642095FBF0F595FBF0F397
:1091100000FB135000B205F0FDF894F81C38B4F8C9
:10912000205813F0020F08BF0025012005F004F9B4
:1091300028B205F0EFF8092005F0FEF8002005F050
:10914000E9F8274B94F822581A88B2F5967F0AD985
:109150001D4B1B7B03F00F03072B04D842F20F7546
:10916000954228BF1546052005F0E6F8D4F80C38DE
:109170005B7B0BB928B216E0A5F120000CF09CFC3B
:1091800018490CF0A1FD002105460CF087FE10B92E
:109190004FF07C5101E04FF03F4128460CF0D8FBE6
:1091A0000CF0A4FE00B205F0B5F894F81C28064BAC
:1091B000950703D493F82328012A19D1012384F8B1
:1091C000233809482DE000BF940F00201400002030
:1091D00000007A44002E00200000C842A086010052
:1091E000E20000206666E63FB8170020E00000209D
:1091F000D3F80C58BF4968680CF0B2FC0CF076FE4E
:10920000BC490290A8680CF0ABFC0CF06FFE039018
:1092100002A806E0B84A02AB92E8030083E8030024
:10922000184601F09BF805F07FF8227BB34B282A03
:109230001ED100221A735B684FF47A70B3FBF0F70B
:109240003C26172005F078F8B7FBF6F5B5FBF6F0ED
:1092500006FB1050000200B205F05CF8182005F083
:109260006BF806FB157000B205F054F805F05CF8D9
:1092700094F82C38A14D002B00F05D8101F0FAF933
:10928000D5F830389E4AC31A9342074640F2C6804A
:10929000002385F8363885F83838B5F80838DAB25A
:1092A0001B0A85F8522885F8533885F8482885F830
:1092B0004938D5F860286B689A1AD5F86438D97B94
:1092C0004FF47A734B439A420DD36B68C5F86038FC
:1092D00095F86838013B012B9FBF102385F836387D
:1092E000022385F83838D4F810280A20D4F8143826
:1092F00092FBF0F293FBF0F384F85028121284F8FA
:10930000512884F8543894F81C281B1284F85538D6
:1093100094F822389007794984F8833803D42D23B0
:1093200081F8843878E0D4F824987648DFF8E0C1F2
:1093300099FBF0FA0CFB0A924FF0060E042B0EFB81
:1093400002F28CBF3323322381F884386E4BD4F879
:10935000286892FBF3F196FBF0F003FB11226425E1
:1093600092FBF5F20CFB006C0EFB0CFE84F87528EA
:10937000121284F876289EFBF3F203FB12E393FBB0
:10938000F5F30AEB8A0A4FFA81F80AEB8A0A08EB2E
:109390008A0189B284F8731800EB8000090A84F806
:1093A000741800EB800051B201EB800292B284F895
:1093B0007828120A84F8792884F87A38B4F81E28B4
:1093C0001B1284F87B382423534393FBF5F5B4F840
:1093D00096380A2284F87C381B0A84F87D38B4F861
:1093E00020384FEAD979B3FBF2F303F5FA739BB255
:1093F00084F87E381B0A84F87F38B4F89838F60F62
:1094000084F87058C5F3072584F8729884F8776853
:1094100084F8715884F88538C4F8307894F89A88BC
:10942000364DB8F1000F0DD1D5F8A00801F0F1FAD2
:10943000012807D90228354E00F04F8200F080FF46
:109440000123B370D4F8A4282C4D002A73D095F8CA
:109450009A683EB140F6B731D5F8AC38FB1A8B426A
:1094600019D868E00123D5F8A00885F89A3804F0E7
:10947000E2FED5F8B038082193F9000002238DE808
:10948000480032464FF4964301F025F985F8B46858
:10949000C5F8A0084DE095F8A868CEB9D5F8A008A1
:1094A000C5F8A46885F89A6804F0C5FED5F8B03808
:1094B000082193F9000001238DE8480032464FF45B
:1094C000964301F008F9C5F8A00800F039FF30E034
:1094D000013EF6B285F8A86895F8B41895F8B53845
:1094E000C6B94A1C013385F8B42885F8B538D5F8D3
:1094F000A0081CE08096184B909E0108940F002055
:109500003F0D03008096980040420F001400002099
:10951000806967FF12F8016B01337018314685F8D6
:10952000B408D5F8A008C5F8A42885F8B53801F026
:1095300073FAC4F8AC7894F8B638C14DDBB1D5F8FD
:10954000B838C3B1D5F8BC38ABB1C5F8C0381B6862
:10955000BC4AC5F8C438D5F8C8381344187AFEF7A1
:1095600067F90AF0DDFBD5F8C8380133092B88BF4D
:109570000023C5F8C83894F8CC28B14B6568002A98
:1095800000F0E681D3F8D028002A00F0E18193F8BA
:10959000D438013B012B00F2DB81D4F8D008A84E6F
:1095A00001F037FAE0B1D6F8D00801F02FFA96F8BA
:1095B000D53807467E2BD6F804800ED102231B280F
:1095C00086F8D43809D1D6F8D00801F022FA20B9AB
:1095D0000123C6F8D88886F8DC3884F8D578DCE72B
:1095E000D6F8D82873689B1A41F6583293421ED990
:1095F000032386F8D438ABE1934A32F8130010B94C
:1096000003464FF403600133B0F5C06FDBB275D091
:109610001FD9B0F5006F7BD034D9B0F5036F41D1BD
:1096200084F8DD38D4F81838854E9F0641D494F874
:10963000DC6894F8DD38002E00F04C8162688049C7
:10964000521B012AD8D981F8DD38002381F8DC3893
:109650007EE1B0F5007F44D008D8B0F5807F00F0FF
:109660008880B0F5887F00F08480E4E7B0F5806FF3
:1096700000F09C80B0F5826F00F0EA80B0F5047FC6
:10968000D9D123E0B0F5E26F00F08380B0F5E46F4C
:1096900000F08480B0F5E06FCDD184F8DD38B4F906
:1096A0000E107FE0B0F5046F6CD0B0F5026FC2D140
:1096B000F9E096F81C389907B9D5B6F81E18242396
:1096C0004B436421123393FBF1F1FDE084F8DD3864
:1096D000D4F800385A4E9A07A9D5B6F808380A21A6
:1096E000F1E084F8DD38D4F80038554E1B059ED5DE
:1096F000D6F810180A2391FBF3F1E5E084F8DD3881
:10970000D4F800384E4E1F0591D5D6F81418DBE07A
:10971000D4F818184A4A880684F8DD3887D592F8B4
:109720001C18890783D5DF0711D5D2F828381922EC
:1097300083EAE371A1EBE37101EB5101B1FBF2F1BB
:10974000002BACBF41F0004141F040410EE0D2F8A7
:109750002438192283EAE371A1EBE37101EB510193
:10976000B1FBF2F1002BB8BF41F080414FF4006033
:1097700088E084F8DD38D4F818385E077FF557AFF5
:10978000002155E084F8DD38B4F9143064215943E0
:1097900078E084F8DD38B4F9101003E0B4F9121061
:1097A00084F8DD382C2391FBF3F16BE084F8DD388D
:1097B00094F8DE38224A0133DBB2032B88BF012341
:1097C00082F8DE3842F2107394F8DE1859431F4BCA
:1097D0001B78D80748BF01319A0748BF02315F079D
:1097E000B4F8E03848BF0431DE0748BF0A319807B3
:1097F00048BF14311A0648BF2831DF0548BF283159
:109800005E0748BF6431180748BFC8319A0548BF92
:1098100001F5C8719F0648BF01F57A71DE0648BFA1
:1098200001F5FA61580648BF01F57A614FF480608E
:1098300000F052FD024B002283F8DC28F7E600BF5F
:10984000940F0020909E0108D0BD0108002E00203A
:10985000D4F81818404F11F0200684F8DD3817D0DE
:1098600097F81C2812F0020F14BF4FF47A710021F0
:1098700012F0010F14BF4FF4FA6300230B4494F865
:109880002218194400F028FD002384F8DC38CEE6C5
:10989000D7F8003819067FF5CAAE314600F01CFD36
:1098A00087F8DC68C3E684F8DD38D4F818382A4E27
:1098B0009A067FF5BCAE96F81C389B077FF5B7AECD
:1098C000B6F820386421594300F006FD002386F8DD
:1098D000DC38ACE684F8DD383AE0B37823B1C5F87B
:1098E0009C7886F80280ADE5D5F89C38FB1AB3F574
:1098F0007A6FFFF4A7AD0123D5F8A008B37001F08B
:1099000085F80646D5F8A00801F080F872067FF4C5
:1099100099AD8A2802D08E280DD093E5D5F8183855
:109920009B067FF58FAD95F89A38002B7FF48AADB2
:1099300005F6690306E095F89A38002B7FF482ADAE
:1099400005F63403C5F8A4382D2385F8A83879E541
:1099500004B0BDE8F08700BF940F00202D4B2E4AC5
:109960001B68126810B51A602C4A1168596051685A
:1099700092689960DA602A4A1168196151689268A0
:1099800059619A61274A1168D961516892681962D0
:109990005A62254A11881985518859859188D2883B
:1099A0009985DA85214A11881986518859869288C5
:1099B0009A861F4A1188D986518892881987194634
:1099C00021F83A2F1B4A10780022824206DA1A4CFC
:1099D00034F81240013221F8024FF6E7174A128894
:1099E000A3F86420164A1288A3F86620154A118845
:1099F000A3F8681051889288A3F86A10A3F86C2025
:109A0000114A1288A3F86E20104A5289A3F85E20EA
:109A100010BD00BF0C290020E02D0020BC26002036
:109A2000C8260020D4260020AC0F0020C40E002041
:109A3000A20F002044190020E40E0020E42500209D
:109A4000840E0020CA0E0020000F0020D00E00203F
:109A5000A0F17D03012B70B504460D460A4E05D8D2
:109A600030687D2100F0D8FF84F020043068214662
:109A700000F0D2FF35B12B881C4404EB142404F011
:109A8000FF042C8070BD00BF641800202DE9F8434E
:109A900005460E460D4B002493E88003B44213DACA
:109AA0007B1933F9140008EB050333F9142009EB93
:109AB000050333F9143001341344022293FBF2F30B
:109AC000C01A09F05FFFE9E7BDE8F8830C29002020
:109AD00010B5134B014693F8D437012B19D1114B14
:109AE000114C1878421CD2B21A70120644BF0022E0
:109AF0001A700E4A1B7812782154934236BFC2F175
:109B000080029B1A9B183F2B09D9BDE8104005F035
:109B1000A1BE074BBDE81040186800F07DBF10BD26
:109B2000B40F0020282800202A28002029280020FF
:109B3000F428002070B54720FFF7CAFF174B1B68B9
:109B40001B0307D5164B174A5B6810681B68C01AC1
:109B500009F008FF144E154C154D307809F002FF3E
:109B600023682868C01A09F00DFF63686868C01A86
:109B700009F008FF0F4B188809F0F4FE0E4B188807
:109B800009F0F0FE0D4B188809F0ECFE33782374D1
:109B90002B68A3606B68E36070BD00BF6C2A002077
:109BA0000C290020E02D0020B6170020F828002006
:109BB000B8170020B4170020B2170020080F0020AB
:109BC0007FB5264C264E274D2749284A284B20B1E1
:109BD00028480088B0F5805F31D2308891F8201095
:109BE0001278ADF8040028781C4D1B788DF806001B
:109BF0008DF807108DF8082001A8294606228DF857
:109C000009300EF04BFF30B30198BDF808302860E2
:109C1000AB805320FFF75CFF208809F0A3FEA078FB
:109C200009F0A0FEE37801A80193237902936379F8
:109C3000039309F007FE0F4B00221A800BE03088D7
:109C400091F820102080127828781B78A070E1709D
:109C500022716371DDE704B070BD00BF7818002089
:109C600074180020B01700208C2D0020000D00205B
:109C7000660D00208C2A00202DE9F04FBC4B8BB0E4
:109C80001A880193BB4F002A40F09D8042F20103E5
:109C9000B7F8D207B84EC41A60426041FFF790FF90
:109CA000FFF75CFE346849202546FFF711FFB34BF0
:109CB00004F11C09186809F055FE55F8040B09F069
:109CC00051FE28460AF040FE04F110000AF03CFE66
:109CD0004FF01008AA4D01232A6803FA08F3134233
:109CE00003D0D9F8000009F04DFE08F10108B8F1E1
:109CF000130F09F10409EDD104F128000AF014FE54
:109D0000B7F84031B4F92E00C01A09F02BFE2B68C9
:109D1000D90408D59B4BB4F864001B88181AC0F30B
:109D20000D0009F01FFE2B689A0403D5B4F86600F5
:109D300009F018FE2B685B0503D504F168000AF0F2
:109D4000F3FD2B68180403D5B4F86E0009F00AFE81
:109D5000A04604F130000AF0E7FD04F136000AF0F5
:109D6000E3FDB7F8403138F93C0F0127C01A09F07C
:109D7000F9FD854B1B789F4208DA38F9020FB4F9D8
:109D80003C300137C01A09F0FDFDF2E72B68990558
:109D900005D5B4F95E00A0F2DC5009F0F3FD32689D
:109DA0007A487260B260121A1111794A4A43531C00
:109DB000032293FBF2F202EB42029A1A702303FB96
:109DC00002033360CAE1734B1C68734B1A689442F8
:109DD0000ED01C60714B1B78083B012B08D8452026
:109DE000FFF776FE0020FFF773FE204609F0BAFD6C
:109DF000019B97F8D2171B8897F8D3070B44013BB8
:109E0000B3FBF0F200FB12338B4280F072815A4FA9
:109E10000120FFF7D5FEFFF7A1FD50203E687D68C9
:109E2000FFF756FEBA683B6810681B687A680344FF
:109E3000106806F11C0BA3EB400009F0A3FD6A6853
:109E4000736802A89B1A0293AA68B36805F11C08FC
:109E50009B1A0393EA68F36810249B1A04930AF090
:109E600073FD2A69336902A89B1A02936A697369B0
:109E70009B1A0393AA69B3699B1A049309F0E2FC45
:109E80003F4901220B68A2401A428A4606D0DBF8FD
:109E90000000D8F80030C01A09F074FD0134132C0A
:109EA0000BF1040B08F10408EAD106F1260005F1D4
:109EB0002601002331F9024F30F9022F121B02ACA8
:109EC00044F823200133042BF4D103214FF000097F
:109ED0004FEA89035FFA83F902AB53F821206AB194
:109EE00002F108000F2802D849F0010906E080328B
:109EF000FF2A94BF49F0020949F0030911F1FF312B
:109F0000E6D248460024FFF7E3FDA0460DF1080B1A
:109F100009F00302022A16D0032A1DD0012A50D1CB
:109F2000B8F1000F05D1DBF8004090462401E4B2FF
:109F300047E0DBF800004FF0000800F00F0020437E
:109F4000FFF7C6FD3DE0B8F1000F0CD0DBF80000D4
:109F5000C0F3031020432EE0B8F1000F20D19BF88E
:109F60000100FFF7B5FD9BF80000FFF7B1FD28E009
:109F7000782A0020B40F00200C290020742A002029
:109F80006C2A0020682A002044190020182900208B
:109F9000B76DDBB6802A00207C2A0020A81800209C
:109FA000DBF80000C0F303302043FFF791FDDBF83E
:109FB0000000C0F30710FFF78BFDDBF80040240121
:109FC000E4B20BF1040B06AB9B454FEA99099FD114
:109FD000B8F1010F02D12046FFF77AFDDAF8001040
:109FE00011F480541FBFB6F86430B5F86420012422
:109FF0009B1A18BF02938A040AD50AAB03EB8402AA
:10A00000B5F86600B6F8663001341B1A42F8203CF9
:10A010004B0513D502AB03EB840C06F1660E05F17C
:10A02000660000233EF9022F30F9028FC8EB0202CE
:10A030004CF823200133032BF4D1033408040BD54F
:10A040000AAB03EB8402B5F86E10B6F86E3001343B
:10A050005B1A42F8203C00E0FCB1012C03D10298CD
:10A0600009F090FC19E0631E002002AA52F8232098
:10A070004000C0B20AB140F00100013BF5D5FFF746
:10A0800027FD4FF0000802AB53F8280008B109F093
:10A0900079FC08F10108A045F5DB30200321FFF72A
:10A0A000F5FC36200321FFF7F1FC2F4B3C201978FB
:10A0B000FFF7ECFCDAF80030990506D5B6F95E003A
:10A0C000B5F95E30C01A09F05DFC3A6827487B6834
:10A0D0007A60121A1111264ABB604A43531C0322AC
:10A0E00093FBF2F202EB42029A1A702303FB020383
:10A0F0003B60204B1B681A0630D51F4C1F4D226851
:10A100002B689A420BD162686B689A4207D1019B17
:10A110001B88102B11D11A4B1B885B060DD14820D0
:10A12000FFF7D6FC206809F02DFC606809F02AFCD6
:10A1300023682B6063686B600EE0124A0F4B117846
:10A140002A7C914208D1104A99681068884203D14C
:10A150005268DB689A4201D0FFF7ECFC09F060FB23
:10A160000BB0BDE8F08F00BF441900201829002073
:10A17000B76DDBB6941700200C0F0020F8280020E4
:10A180007A2A0020B6170020B81700200A4A138840
:10A1900001331380094A136801331360084A138896
:10A1A00001339BB2202B01BF00231380054A138883
:10A1B00008BF0133138070478C2A0020742A0020C6
:10A1C000782A00207A2A00202DE9F84F0C9EC2EB55
:10A1D000030B394C0B9B002914BF4FF0060A4FF0BC
:10A1E000040AF61A636805460133904613D12368C2
:10A1F00053455ED2314A032B98BF294652F823209B
:10A200002F4809F02DFC63680022013363602D4B59
:10A2100005469A7113E0002511E02B4A1278954209
:10A2200040DA0B9BE3B109FB06F2995C01228A40FC
:10A23000264909680A4213D1636801336360D4F880
:10A2400004900A9B1C4F9945E7DB2BD10A20FFF7AE
:10A250003FFC3B6801333B604FF0FF337B6021E004
:10A26000184A917921B12C20FFF732FC013501E029
:10A270000121917109FB0BF3226808EB030752B926
:10A2800058F8030009F082FB97F9041005444B1CB1
:10A29000D2D00F4802E03A440E48117909F0E0FBB1
:10A2A0000544C9E7206850452CBF00200120BDE8C7
:10A2B000F88F0020BDE8F88F842A0020A89E0108AE
:10A2C000F0BD010878180020F00000206C2A002062
:10A2D000FFBD010873C6010830B585B004AC002588
:10A2E00024F8025D0091ADF8060021461020FFF72A
:10A2F000AFFB9DF806002146FFF7AAFB9DF807007B
:10A300002146FFF7A5FB9DF800002146FFF7A0FBC3
:10A310009DF801002146FFF79BFB9DF802002146B6
:10A32000FFF796FB9DF803002146FFF791FB9DF890
:10A330000E002946C043C0B2FFF78AFB05B030BD0E
:10A3400010B5054C206800F064FB18B1206800F0DF
:10A350005DFBF6E710BD00BF3418002013B50446BE
:10A3600001A9006803F0ACFF132003F0E5FFBDF97D
:10A37000040003F0CFFF1B2003F0DEFFBDF9060051
:10A3800003F0C8FF232003F0D7FF2368002BB4BFDE
:10A3900053204E2003F0BEFF01A9606803F090FF38
:10A3A000122003F0C9FFBDF9040003F0B3FF1A2027
:10A3B00003F0C2FFBDF9060003F0ACFF222003F05A
:10A3C000BBFF6368002BB4BF5720452003F0A2FFFA
:10A3D00002B010BD034B4FF4004208B11A61704740
:10A3E0005A61704700080140034B4FF4004208B126
:10A3F0005A6170471A6170470008014010B5084B58
:10A400000022196801EBC20393F90240844201D192
:10A41000981C10BD0132042AF4D1002010BD00BFE9
:10A42000A02B002038B1438811EA030003D08B42EF
:10A430000CBF01200220704730B50A4B0A491C6846
:10A440000A78032A0AD81346551C04EBC303EAB260
:10A450009D882842F5D00A70981C30BD0A700020F3
:10A4600030BD00BFA02B002080180020014B00222F
:10A470001A70E1E7801800202DE9F047877890F8FE
:10A4800003C0BBB2C7F1640E03EB83065C42C3F1A9
:10A4900078001C4D5FFA8EFE7600CCF16408A4B201
:10A4A00080B2A3B20FFA83F9B9F1000F04DC002BDC
:10A4B00014BF3B46012300E0734609FB09F25B43EE
:10A4C00002FB0CF292FBF3F3434403FB09F30A2271
:10A4D00093FBF2F333449BB225F8023FB1F80090AE
:10A4E0004A880A34C9EB020A1AB202FB0AF24FF494
:10A4F0007A7392FBF3F3A4B24B4484422B80D0D105
:10A50000BDE8F0878018002010B54478007800225C
:10A5100040F6C41102FB02F3193B634303F6C41374
:10A520005343434393FBF1F3034921F812300132C3
:10A53000072AEDD110BD00BF9A180020104B04303F
:10A5400033F91000B0F5617F05DB40F63303984224
:10A55000A8BF184601E04FF461700A7819235A43E6
:10A5600002F28332824208DA4A78534303F2833399
:10A570008342B4BF0020012070470020704700BF15
:10A58000602D002010B500F1500302788A4203D1FB
:10A590008478C278944204D304309842F5D10020E4
:10A5A00010BD012010BD0B4B1B6813F4805F0A4BDC
:10A5B000B3F9063005D0C089421A934207DD08443A
:10A5C00000E0008A8342B4BF0020012070470120D0
:10A5D000704700BF94170020602D002038B5134B42
:10A5E00005461B680C461B031FD5114B93F82830FA
:10A5F000083B012B19D84520FFF76AFA0D20FFF719
:10A6000067FA85F08000FFF763FAE0B2FFF760FABF
:10A61000C4F30720FFF75CFAC4F30740FFF758FACA
:10A62000200EBDE83840FFF753BA38BD941700201C
:10A630008018002038B50D4B05461B680C461B03DF
:10A6400013D50B4B93F82830083B012B0DD8452030
:10A65000FFF73EFA0D20FFF73BFA2846FFF738FADE
:10A660002046BDE8384009F08DB938BD9417002068
:10A670008018002010B50A4A0A4B11689B6800BF79
:10A6800012689142F7D1084A4FF47A70D46A00FBFD
:10A6900004F2D31AB3FBF4F300FB013010BD00BF8A
:10A6A000980F002010E000E08018002038B5044624
:10A6B000FFF7E0FF0546FFF7DDFF401BA042FAD39E
:10A6C00038BD10B504462CB14FF47A70FFF7EEFF99
:10A6D000013CF8E710BD2DE9F04F064687B08846EB
:10A6E0009DF8407011461A469DF8443000250C2014
:10A6F00068435A4C00EB040E0057A146B04205D106
:10A700009EF808A0BAF1000F04D0A3E00135042D93
:10A71000EDD19FE0022E00F08D8005DC002E40F090
:10A72000998000934E4887E0142E0BD01E2E40F0E7
:10A730009180504600F0E8FD036839465B690446A5
:10A7400098477EE0474F484CBB69032243F004031F
:10A75000BB614FF4805B204605A98DF8162003925B
:10A76000ADF814B08DF8176006F008FEC4F814B008
:10A77000C820FFF7A6FFC4F810B0BB69039A43F0E6
:10A780000403BB614FF4C053204605A9ADF8143053
:10A790001C23364C8DF816208DF8173006F0EEFD90
:10A7A000334A4FF4802353614FF0010BA36704F148
:10A7B0007800082384F87D3084F87EB00AF05AFDD2
:10A7C0002C4B2D4AC3F800A0FB6905A843F40003F5
:10A7D000FB612A4BDA6002238DF815308DF8146086
:10A7E0008DF816A08DF817B00AF026FD2A238DF8F3
:10A7F00014309DF817308DF815B08DF816A01BB1E8
:10A8000005A80AF019FD04E01D4B4FF48062C3F85F
:10A8100084201C4B1C4A1D49136002221A721C4BD7
:10A820001C4A13601C4A1B68116098471B4B23632A
:10A830001B4C06E01B4800933B4605F079FA0446A2
:10A8400040B10C2303FB05952671204685F808804E
:10A850006C6000E0002007B0BDE8F08FA42B002062
:10A86000003801400010024000080140801800201C
:10A8700000040140D80042420005FA0500ED00E066
:10A8800000E100E09C2A0020982A00201800002007
:10A89000B00000200C28002008280020C09E0108DD
:10A8A000B018002000480040024A136801331360CA
:10A8B000704700BF980F0020024BD3F8803003B1DF
:10A8C0001847704780180020014B1B68184700BFCD
:10A8D000E42D002010B50020FFF7F6FF074B002401
:10A8E0001C700AF085FC064B83F88440C3F888404E
:10A8F000A3F88C40C3F8904010BD00BFB02D0020DD
:10A900008018002010B510B9BDE81040E2E7002320
:10A910000C225A430C4C1119125D824203D00133B0
:10A92000102BF5D110BD094BD3F8900018B14A781F
:10A930004078824206D20022C3F89010A3F88C20FF
:10A94000C3F8882010BD00BF88A901088018002026
:10A9500010B540001428A8BF14200023074A022184
:10A9600099540B4499181424834201F8014CF5DBE7
:10A97000FF21D1540F20BDE81040C3E7D8280020A4
:10A980002DE9F84381460B26013E2DD0194B0822B4
:10A990001A6109F101074FF032080524154D012015
:10A9A000EB6883F00803EB60FFF78EFF4046FFF78C
:10A9B00088FEEB68002083F00803EB60FFF784FF5C
:10A9C0004046FFF77EFE44B1013CE7D14FF4FA70F8
:10A9D000FFF777FE4FF0FA08E0E7013FDED14FF4D2
:10A9E0007A70FFF76EFECFE7034A044BDA60BDE8EA
:10A9F000F88300BF000C01400400FA0500ED00E000
:10AA000003681B6918470368DB68184703689B687D
:10AA1000184703685B68184703681B681847B0F954
:10AA200002302DE9F74F93421CBF0023037090F8CA
:10AA300000A004460E469146BAF1000F40F0B480E3
:10AA400010460BF039F88B490BF08AF88A490BF065
:10AA500087F84FF07C510BF083F8074602F0EEFACE
:10AA60000546384602F05CFB014628460BF02CF9FF
:10AA7000014605460BF074F88049834628460BF0E2
:10AA80006FF803465846194601930AF061FF4FF0EC
:10AA90007E510AF05DFF01464FF07E500BF014F935
:10AAA000294680460BF05CF829460BF059F807461A
:10AAB000014660600AF04CFFE7604FF07E57294680
:10AAC000A060276128460AF043FF29460BF048F8AA
:10AAD0004FF080410AF03AFF014640460BF040F843
:10AAE000019B6061194658460AF030FF39460AF06A
:10AAF0002FFF014640460BF033F840F2DC53A046EE
:10AB00002746554663651023A4F852301823A061E8
:10AB1000A4F850304FF09741D8F810000BF020F80F
:10AB2000002182460BF0BAF928B150464FF07C5113
:10AB30000AF00CFF04E050464FF07C510AF008FF89
:10AB40000BF036FAC7E90E014FF09741D8F8040030
:10AB50000BF006F8002182460BF0A0F928B1504610
:10AB60004FF07C510AF0F2FE04E050464FF07C5169
:10AB70000AF0EEFE0BF01CFA0135032DC7E90801BF
:10AB800008F1040807F10807C4D1A6F2DC531B043E
:10AB90002367E3676367C4F88030A367C4F8843031
:10ABA0000123A4F802902370D4F85490B4F9528091
:10ABB000C9EB0606636A06FA08F67343276A4FEA8A
:10ABC000E67B206F07FB0B332667A7FB0667E26F68
:10ABD0001F44636CD4F840C053434FEAE27B0CFB44
:10ABE0000B3ED4F88010C4F88020ACFB02237344E1
:10ABF000B61A67EB0307E36AA26A43434FEAE07BB6
:10AC000002FB0B3EA2FB00237344B6185F41E36CCA
:10AC1000656F4B436067A06C4FEAE17B00FB0B3331
:10AC2000C4F88410A0FB01011944636B361A05FBBC
:10AC300003F3206B4FEAE57B00FB0B3367EB010767
:10AC4000A0FB0501801919447941B4F95020A5678A
:10AC50000AF062FC08F1FF3201239340E067C0185C
:10AC600041EBE37142460AF057FC484403B0BDE8AB
:10AC7000F08F00BF6F12833ADB0F4940F404B53FF9
:10AC80002DE9F8430024254BE0B293F8C460B042AC
:10AC90000DD203EB8003224AD3F8943032F810101F
:10ACA0001BB10B2801D8DB6898470134EBE71D4B3B
:10ACB0001B685B032FD500242346E2B2B2422AD29E
:10ACC000DFF858904FEA840809F1940757F82420D8
:10ACD00055689D4217D0284604F08EFFEFF312838B
:10ACE000502282F312882821AA8C01FB009092B294
:10ACF0000132C0F8EC20AA8ADBB292B242F0010223
:10AD0000AA8283F3118857F8083000221B680134A7
:10AD10001A802B46D1E7BDE8F88300BF80180020D9
:10AD2000E40E00209417002008B50E4B1B6813F4A6
:10AD3000805F0D4B14BFD3F86821D3F86C2193F8D2
:10AD4000C41092880023D8B2884204D2074820F861
:10AD500013200133F7E7FFF793FFBDE808403220E7
:10AD6000AFE400BF9417002080180020E40E0020FC
:10AD70000A4B30B51A680A4B02F48052D3F8684186
:10AD8000D3F86C5100230AB1A18800E0A9880548D6
:10AD900020F8131001330C2BF5D130BD941700208F
:10ADA00080180020AE28002070B5124D00242146E6
:10ADB00005F27110702285F870410DF08AFE21466F
:10ADC000D5F8E4310B4A0B4493F9020088B11E68B0
:10ADD00002F271140E5108199C88073184809B7906
:10ADE0007029837192F8703103F1010382F8703198
:10ADF000E6D170BD80180020426A806A131A58425A
:10AE0000584170474171704743799B070AD5436A9F
:10AE10008269D154436A01690133B3FBF1F201FB4A
:10AE2000123343627047437913F001031FBFC368B5
:10AE300003F1FF32C369006A1DBF181A1040C0B287
:10AE400018467047437910B513F0010304460DD03E
:10AE5000FFF7E9FF58B1236A6269E168D05C01330A
:10AE6000B3FBF1F201FB1233236210BD184610BD93
:10AE700090F83B3210B57BB990F83A3290F83942ED
:10AE8000A34209D2B0F8401201229A400A4301338A
:10AE9000A0F84022DBB2F3E710BD8379DB0748BF9F
:10AEA000B1FA81F1D0F8343148BF49095A681B8999
:10AEB00009B1136170475361704710F80A3C0133C0
:10AEC000DBB20A2B84BF10F8131C054A00F80A3CB9
:10AED00082BF002322F8113000F80A3C704700BFFF
:10AEE000B42C0020354A70B5136C90681944344B6B
:10AEF0001B78D94040F68C23081A98429160D060A4
:10AF0000516013463BD9127893F9451010468A4296
:10AF10000BD1111F082908D893F84610182901D819
:10AF2000013103E083F8442002E0002183F8461059
:10AF300093F944402149A24219D191F84740B4B154
:10AF40000C310024944206DA51F8046F1D4D25F8A7
:10AF500014600134F6E70C2805D01A49002421F8C2
:10AF600010400130F7E7184801780131017083F88B
:10AF70004520002201211A7083F8471070BD92F815
:10AF80004710C9B140F2DA51A0F2EF248C4208D840
:10AF900011780B2905D80B1D0131117042F82300DF
:10AFA00070BD002283F84720084B03F130020021D6
:10AFB00043F8041F9342FAD170BD00BF88010020FE
:10AFC00087010020B42C002064060020940100209A
:10AFD000024A136C01331944116470478801002040
:10AFE000024B53F820301B68198070471419002059
:10AFF000074BA1F57A7153F820301A681B89594321
:10B000004FF47A7391FBF3F189B21180704700BF5E
:10B01000141900201FB50123ADF80830ADF8041055
:10B02000002301A9ADF80A30ADF80C30ADF80620C8
:10B0300006F091F805B05DF804FB38B5A0F513747F
:10B040006379A579DB0745D594F8383205F0010519
:10B05000F3B1226B1068838DC3F34E03838494F89D
:10B060003C3223B1B4F842320133A4F84232917A2F
:10B070006A00FFF7CFFF012384F83B32002384F8F6
:10B08000393284F83A3284F83832A4F8403238BD84
:10B0900094F83B322046012B04BF94F8393284F8EF
:10B0A0003A32FFF7E5FE94F83B22236B3AB90122CE
:10B0B00084F83B221868997A05FA02F207E0002228
:10B0C00084F83B2295421868997A08BF0222BDE8AD
:10B0D00038409FE738BD10B5A0F5127494F83C22B3
:10B0E000BAB9A36A616A994228D0591CA069A162C1
:10B0F000C35C2069DBB25B0043F400738142A4F8B7
:10B100003E324FF00A0384F83D3228BFA262012389
:10B1100012E094F93D327BB1B4F83E1220464B0860
:10B12000A4F83E3201F00101FFF7B7FE94F83D327A
:10B13000013B84F83D3201E084F83C3294F8383227
:10B14000002B4ED194F839320133DBB2092B84F84D
:10B15000393203D12046BDE8104089E60A2B40D1A0
:10B1600094F83B322BB9B4F8403243F00103A4F811
:10B1700040326379D9071CD5B4F84002820501D466
:10B18000C30705D4B4F844320133A4F8443210E0C4
:10B19000E36AC0F347000BB198470AE0E3696269CC
:10B1A000D054E369E1680133B3FBF1F201FB1233E0
:10B1B000E361012284F8382294F83B220023012A1B
:10B1C00084F839320DD1A27984F83B32236B12F026
:10B1D000010F1868997A0CBF02220022BDE81040C6
:10B1E00018E710BDF0B5046D8279A389467923F480
:10B1F000005312F0020F4FEA03434FEA13430CBF10
:10B2000000214FF4005112F0040FA38114BF4FF43A
:10B21000806E4FF0000E16F0010F8768054614BFD0
:10B2200004200020B307238A48BF40F008029BB2E5
:10B2300023F4405343EA01032382A18948BF90B21B
:10B2400089B221F4B05121F00C014EEA010140EA2B
:10B250000102A281A38A87B023F440731B041B0C54
:10B26000A38201A805F01CFF039B049E254A94427B
:10B2700018BF1E46A389192272431BB2002BB4BF0C
:10B280007E00BE00B2FBF6F66427B6FBF7F00001C5
:10B29000010907FB1163A28912B2002AB7BFD900C6
:10B2A0001A013231B1FBF7F2A7BF3232B2FBF7F32A
:10B2B00002F007021043A8BF03F00F03AA79A8BF4A
:10B2C000184380B212F0010F20812B6D06D00D497A
:10B2D0008B4202BF0420A1F53051086112F0080F23
:10B2E0009A8A0BBF22F0080292B2120442F00802BE
:10B2F00008BF120C9A829A8992B242F400529A8143
:10B3000007B0F0BD003801402DE9F04F4E4C4FF42E
:10B31000147585B0804691461E4605FB00452746BC
:10B3200020B94A4B2B63103BC5F834314FF41473EA
:10B3300003FB08F3464AFC18FA50032262712246C6
:10B3400003F59C733B44E162A36100214FF48070DC
:10B35000D4F8343134324FF0010B62612162E16183
:10B36000A162616284F83C1284F83912A4F8421296
:10B37000A4F84412C4F80890A671E060206184F833
:10B3800038B284F8468258681B890222ADF80C3026
:10B3900003A910238DF80E308DF80F20019207F0CD
:10B3A00063FD236B019A597B58681B898DF80E1039
:10B3B00003A9ADF80C308DF80F2007F055FD284695
:10B3C0005946FFF76AFD3220FFF77BF9214BD4F88D
:10B3D00034A11B681A46B2FBF9F1B1F5803F03D3E3
:10B3E000012AF8D95208F6E71B4A5046B3FBF2F29D
:10B3F00089B2D2B204F0D6FB4FF4147000FB08F00F
:10B40000164B07EB000800F512703C180022C8F834
:10B4100048325046214604F00DFCD8F8307016F042
:10B42000010F0CBF022200223868B97AFFF7F2FD43
:10B430000B4B3846C8F84C32211D002204F0FAFBB1
:10B44000284605B0BDE8F08F681A0020BCB8010896
:10B45000E09E0108EC00002040420F00D7B0000839
:10B460003BB0000803460A4690F84602D96A9B7929
:10B470004AE71FB50123ADF808300023ADF80C30C2
:10B48000ADF80A30084BADF804101B7801A9012B68
:10B4900008BF0323ADF8062008BFADF80C3005F057
:10B4A0005AFE05B05DF804FB8401002038B510F8A1
:10B4B0000E2C044650F8043C52B9012200F80E2C20
:10B4C00020F80C1C997A18680222BDE83840D0E7B1
:10B4D00030F80C2C20F80A1C891A89B220F8081CB4
:10B4E000074A10F80F0C002522F8101004F80E5C23
:10B4F0001868997A2A46FFF7BCFF04F8065C38BD45
:10B50000B42C0020044B53F820301BB107289CBFFB
:10B510001B681980704700BFB00200202DE9F74377
:10B520008E460546DFF8A092114699F85042006811
:10B53000164698467246631C89F8503204F0DEFACB
:10B540002B8901A9ADF8043018238DF806306868FE
:10B5500002238DF8073007F087FCAB7A09F51577E1
:10B56000240127442A6849460C2B00F2F680DFE8C4
:10B5700013F00D00F400F400F4005100F400F400A6
:10B58000F4008A00F400F400F400C200138CDFF829
:10B590003CC223F001031B041B0C1384138CB2F870
:10B5A00004E0108B624520F073004FEA00404FEA40
:10B5B00010409BB21FFA8EFE40F0700014D00CF5C4
:10B5C000006C624510D00CF5406C62450CD00CF557
:10B5D000806C624508D00CF5806C624504D023F085
:10B5E000020343F0030307E023F00E032EF4407E32
:10B5F00043F003034EF4807EA2F804E01083A2F827
:10B6000034801384138B23F008031B041B0C43F0BA
:10B61000080336E0138CDFF8B4C123F010031B04D9
:10B620001B0C1384138CB2F804E0108B624520F4D9
:10B63000E6404FEA00404FEA10409BB21FFA8EFEF0
:10B6400040F4E04008D00CF5006C624504D023F0D3
:10B65000200343F0300307E023F0E0032EF4406EB4
:10B6600043F030034EF4806EA2F804E01083A2F899
:10B6700038801384138B23F400631B041B0C43F4E6
:10B680000063138369E0138CDFF840C123F48073F7
:10B690001B041B0C1384138CB2F804E0908B6245DE
:10B6A00020F073004FEA00404FEA10409BB21FFAAF
:10B6B0008EFE40F0700008D00CF5006C624504D09E
:10B6C00023F4007343F4407307E023F460632EF423
:10B6D000405E43F440734EF4805EA2F804E0908331
:10B6E000A2F83C801384938B23F008031B041B0CEB
:10B6F00043F0080330E0138CDFF8D0C023F480530C
:10B700001B041B0C1384108CB2F804E0938B20F400
:10B71000005023F4E6431B0400041B0C000C62459C
:10B720001FFA8EFE43F4E04340F4405003D00CF582
:10B73000006C624503D12EF4804E4EF4804EA2F888
:10B7400004E09383A2F840801084938B23F4006379
:10B750001B041B0C43F4006393832B7B43B1B2F8AF
:10B7600044306FEA43436FEA53439BB2A2F844303C
:10B7700013889BB243F001031380AB7A0C2B19D8CA
:10B78000DFE803F0071818180B1818180F18181806
:10B7900013000B1902F134000AE00B1902F1380012
:10B7A00006E00B1902F13C0002E00B1902F1400027
:10B7B000C3F8540238460C44A4F85C62C4F858221A
:10B7C00003B0BDE8F08300BF681A0020002C0140E0
:10B7D000084A13689B020BD5074B002119704FF6DE
:10B7E000FE730649086803400B604FF40013536072
:10B7F000704700BF00000240FF2D00206C00024097
:10B800002DE9F04F054690F850008DB00A9107924F
:10B810000B9318B13228A8BF322000E001200AF0B3
:10B820004BF90146A1480AF04FFAA14B044618888B
:10B83000002808BF01200AF03FF99E4908900AF04D
:10B840008FF90190019920460AF082F8014601988B
:10B850000AF03AFA984B09901B889A0724D5974921
:10B86000B1F90030B1F9020083EAE37280EAE071D5
:10B87000A2EBE372A1EBE07191420C46B8BF144613
:10B88000B4F5E17F12DA914203DD0028D8BF4042CF
:10B8900003E0002BCCBF184658420AF00DF9884946
:10B8A0000AF012FA064603E0002601E04FF07E5649
:10B8B0004FF0000903950024CDF80890630006932B
:10B8C000804B33F814300593BDF914000AF0F4F8F6
:10B8D0007D490AF045F90AF009FB0AF0EDF87B49C9
:10B8E0000AF03EF9754B804633F914000AF0E4F88B
:10B8F000714B07461B8804939B076CD001460AF0E6
:10B9000027F8734B814633F914000AF0D5F8014645
:10B9100048460AF01DF80AF0E9FA079B5B42984294
:10B9200003DB079B8342A8BF03460699694A885EEA
:10B930000B9A1B1A32F9140018440AF0BDF882461B
:10B94000287F0AF0B5F864490AF00AF98346287A94
:10B950000AF0AEF8014650460AF002F95F490AF0D3
:10B96000FFF80AF0C3FA81460BF100400AF0BEFA74
:10B97000814505DB58460AF0B9FA4845A8BF484654
:10B980000AF09AF8DFF878910290019950460AF08F
:10B99000E7F859F8241009F0DBFF51494FEA840B0E
:10B9A00082460AF07BFA38B950464E490AF094FABA
:10B9B00020B1DFF830A101E0DFF824A149F80BA0A5
:10B9C000A87C0AF075F8014650460AF0C9F84649C5
:10B9D0000AF0C6F88146049BD90700F19380BDF9AF
:10B9E00014304FEA840A002BB8BF5B42B3F5206FD6
:10B9F000DFF804B103DD00234BF8243029E03B4994
:10BA000038460AF0ADF8039B059058780AF050F8D4
:10BA1000059B014618460AF057F9414609F096FF82
:10BA200001990AF09DF85BF8241009F091FF304964
:10BA300083460AF033FA38B958462E490AF04CFAD0
:10BA400020B1DFF8B0B001E0DFF8A4B02A4B43F832
:10BA50000AB0039BD87A0AF02BF8274B53F824102E
:10BA60000AF07EF825490AF07BF8049A034692070B
:10BA70004AD504900299384609F068FF01463046DD
:10BA80000AF06EF80146029809F062FF049B4946ED
:10BA90000746184609F05AFF014630460AF060F89A
:10BAA0000146484609F054FF03462DE083F9223E43
:10BAB000A00E0020BD37863574180020AC0F002082
:10BAC0000000E143C40E00200000A03ECDCC4C405D
:10BAD000F82D0020FC0E00200000A0406F12033C57
:10BAE0000000F0C10000F0410AD7A33D0000A043D0
:10BAF000000040C300004043841D00200AD7233CBF
:10BB00007C1D00204B46029FDFF82CA204931AF8FC
:10BB1000040009F0D1FF014640460AF021F87B49B4
:10BB20000AF01EF80146384609F010FF0AF1040B2E
:10BB30005BF824100746404609F008FF01990AF017
:10BB4000C3F84BF824800AF10C0B5BF824800AF14F
:10BB5000140A414609F0FAFE014609980AF000F875
:10BB60000146404609F0F4FE80464BF824001AF8DE
:10BB7000040009F0A1FF0146404609F0F1FF6449C5
:10BB800009F0EEFF8046049B3846194609F0E0FEB6
:10BB9000414609F0DBFE0DF0A9F95E4A069B0592CD
:10BBA000D05238460AF0A2F9DFF890B1049B4BF866
:10BBB000240018460AF09AF9DFF884A1564B4AF897
:10BBC000240008F1004004930AF090F9039A049BC2
:10BBD00001320392059A43F82400174698460CB99F
:10BBE00001246BE60A9A4D4B9479B3F90430640052
:10BBF00028345C434A4B6411B3F9040009F05CFF3C
:10BC00004FF07A5109F0ACFF0DF070F9201A09F0ED
:10BC100053FF002CB8BF6442322C0646414C02DD73
:10BC20000023A36025E008980AF060F920F00300E3
:10BC300009F042FF0190687B09F03AFF0146304667
:10BC400009F08EFF019B8146374918460AF03CF8FF
:10BC50000146484609F084FF0AF048F9A3681844F1
:10BC6000324B9842A8BF1846314B9842ACBFA060F7
:10BC7000A360A3686FF0FF005B13B3F5807FA8BFDC
:10BC80004FF480739842B8BF184609F015FF8146FB
:10BC900030460AF02BF9EB785843801109F00CFF7D
:10BCA000244B04461B78032B11D9B5F84E50B5F53B
:10BCB000FA7F0CD20AF01AF96B42984203DBA842D1
:10BCC0000346A8BF2B46184609F0F6FE044649462F
:10BCD000204609F03DFE0AF009F980B2B88000B2B2
:10BCE00009F0EAFE0DF002F9B88020460AF0FEF8ED
:10BCF000CBF8080048460AF0F9F80023CAF8080013
:10BD0000C8F808300DB0BDE8F08F00BFA69B443BDB
:10BD1000F7CC9238B4260020D4260020AC0F0020A7
:10BD2000C40E00208426002000803B45FEFFFF0F4C
:10BD3000020000F044190020901D0020BC260020C5
:10BD4000C82600202DE9F04F89B00693AA4B0026A3
:10BD5000B3F90270B3F90030002FB8BF7F42002B57
:10BD6000B8BF5B429F42B8BF1F468046B346B2464B
:10BD70003446B7F5FA7F05910392A8BF4FF4FA77DE
:10BD8000019002969D4B198811F0030541D09A4B02
:10BD9000600033F914209A4B33F9143003EB42025C
:10BDA000039B5B429A4203DB039B9342A8BF13466B
:10BDB000944A6FF0040A805E069A1B1A32F9140046
:10BDC0006422184498F80830434393FBF2F398F840
:10BDD0001C200AFB02FA534504DB02EB820A9A4557
:10BDE000A8BF9A46884A52F82430184442F2107389
:10BDF0009842A8BF1846854B9842B8BF184698F895
:10BE0000123042F824005843012D4FEA20330293A8
:10BE100037D0794B7E4833F914B0019BA60093F8D4
:10BE200001C07C4B50F824E033F9145085EAE573E7
:10BE3000A3EBE573B3F5206F16DC502303FB0BF285
:10BE400092FBFCF3042295FBF2F55D1BAE44BEF5BC
:10BE50007A5F714BA8BF4FF47A5E9E45ACBF40F845
:10BE600024E040F8243002E0002340F824308359D5
:10BE70007D2693FBF6F6019BDB7A7343402693FB0A
:10BE8000F6F68A0711D507FB06F507FB0BF90298B2
:10BE9000C7F5FA7303FB0A9903FB00534FF4FA71D9
:10BEA00099FBF1F293FBF1F505E0CB0759BF35465D
:10BEB0005A465246029D63000493564B042033F8C1
:10BEC00014C056490FFA8CF393FBF0FE14F801905E
:10BED000203109FB0EFE6FF04F099EFBF9F99144EA
:10BEE00031F9142021F814C09B1A98F8502093FBC4
:10BEF000F0F062B1079209F0DFFD4949494B01EBCF
:10BF0000C401079A1B6800F0CDFD09F0EFFF464B16
:10BF1000DFF830E11B5D09EB05025843202390FB5D
:10BF2000F3F30499D21A21F80E20404A5B4242F8FA
:10BF30002430019B3E483F49013341F8245040F8EA
:10BF40002490019375460CB901241BE72A4B042762
:10BF5000B3F90440059B2E4E9B79D6F808E00F33C9
:10BF60005B0063432B4C5B11B4F90440002B94FB42
:10BF7000F7F7A3EB0707B8BF5B42322B98F80D40E9
:10BF80000BDC04FB07E42C4BA342A8BF23462B4C3D
:10BF9000A342ACBFB360B46001E00023B36098F883
:10BFA000034004FB07F3264C9B112478032C0CD987
:10BFB000B8F84E40B4F5FA7F07D26742BB4203DBC4
:10BFC000A342A8BF234600E03B46B4686FF0FF06DB
:10BFD00044F34F34B4F5807FA8BF4FF48074B4426B
:10BFE000B8BF344683601E190023AE808C60936016
:10BFF00009B0BDE8F08F00BFAC0F0020741800201E
:10C00000F82D0020FC0E0020A81D0020F0D8FFFF16
:10C0100084260020C40E002080C1FFFF901D002058
:10C020009C2600207C260020A41D0020D426002071
:10C03000BC260020C8260020FEFFFF0F020000F0F3
:10C0400044190020B42600202DE9F04F85B0039359
:10C050009A4B07461C88029104F00204A4B293464E
:10C0600094B1974BB3F90240B3F90030002CB8BF3C
:10C070006442002BB8BF5B429C42B8BF1C46B4F57B
:10C08000007FA8BF4FF40074BA4600258C4B4FF0D8
:10C09000040C33F915108B4B8B4833F815304FEAED
:10C0A00045090093BDF90020490092FBFCF3019380
:10C0B00082EAE273A3EBE273B3F5206F4FEA8508DF
:10C0C00050F825600FDC019BCB1A3344B3F57A5F3F
:10C0D0007E4EA8BF4FF47A53B342ACBF40F8253030
:10C0E00040F8256002E0002340F8253050F8086051
:10C0F0009AF80B30F6115E439AF801306F484B43C3
:10C100000088B61180074FEAA31341D0704839F96F
:10C1100000000144CBF10000814203DB5945A8BF78
:10C120005946084642F2107C6A49DFF8D4E139F9F1
:10C130000110401A039931F91510084458F80E10EF
:10C1400001446145A8BF6146DFF8B8C16145B8BF89
:10C15000614648F80E1097F808E00EFB00F097F8DB
:10C160001CE0C0110EEB8E0ECEF1000C604503DB1F
:10C170007045A8BF70468446B87CCCEB03034143AE
:10C180000913761A6643634301EB66260CEB6323BF
:10C190005149019811F805C024310CFB00FC39F914
:10C1A0000100A3EBAC1C121A042092FBF0F0BDF8C6
:10C1B000003097F8502029F8013082B1CDF800C046
:10C1C000019209F079FC4549454B01EBC501019A03
:10C1D0001B6800F067FC09F089FEDDF800C0414BE8
:10C1E000DFF824E15B5D0CEB060243435B11D21ADE
:10C1F00029F80E203C483D493D4A5B4248F8016021
:10C2000048F800C048F802300AF1010A76460DB934
:10C2100001253BE72A4B4FF0040EB3F90440029B83
:10C22000294D9B79D5F808C00F335B006343254C3B
:10C230005B11B4F90440002B94FBFEFECEEB030E21
:10C24000B8BF5B42322B7C7B0BDC04FB0EC4294B5A
:10C25000A342A8BF2346284CA342ACBFAB60AC604E
:10C2600001E00023AB60FC7804FB0EF3234C9B1130
:10C270002478032C0CD9B7F84E40B4F5FA7F07D2D6
:10C280006742BB4203DBA342A8BF234600E03B4614
:10C29000AC686FF0FF0544F34F34B4F5807FA8BF5E
:10C2A0004FF48074AC42B8BF2C4683601D19002344
:10C2B000B5808C60936005B0BDE8F08F74180020E5
:10C2C000AC0F0020C40E00208426002080C1FFFF98
:10C2D000F82D0020FC0E0020901D00209C26002040
:10C2E0007C260020A41D0020BC260020C82600209B
:10C2F000D4260020FEFFFF0F020000F044190020AA
:10C30000A81D0020F0D8FFFFB42600202DE9F04F33
:10C3100087B00393934B0026B3F90280B3F9003042
:10C32000B8F1000FB8BFC8F10008002BB8BF5B42DE
:10C330009845B8BF98468346B246B1463446B8F5EC
:10C34000FA7F0292A8BF4FF4FA7800900196864BCC
:10C35000198811F0030044D0022C42D0814B6500B3
:10C3600033F91420814B33F9143003EB4202029B62
:10C370005B429A4203DB029B9342A8BF13467C4A6E
:10C380006FF00409AD5E039A5B1B32F9145064220E
:10C390001D449BF808306B4393FBF2F39BF81C2081
:10C3A00009FB02F94B4504DB02EB82099945A8BF62
:10C3B0009946704A52F824302B4442F21075AB4231
:10C3C000A8BF2B466C4DAB42B8BF2B4642F8243079
:10C3D0009BF81220012802FB03F34FEA2333019359
:10C3E0003DD0604B654D33F914A0009BA00093F83D
:10C3F00001E0634B55F8247033F9146086EAE67364
:10C40000A3EBE673B3F5206F1CDC022C14D0502391
:10C4100003FB0AF292FBFEF3042296FBF2F69E1B4C
:10C420003744B7F57A5F574BA8BF4FF47A579F420E
:10C43000ACBF2F502B5007E08AEAEA73A3EBEA73F4
:10C44000642BE4DD00232B504C4B7D26C35893FB1B
:10C45000F6F6009BDB7A7343402693FBF6F68A07D9
:10C4600013D5022C11D008FB06F508FB0AF701983A
:10C47000C8F5FA7303FB097703FB00534FF4FA7214
:10C4800097FBF2F193FBF2F508E0CB0704D5022C01
:10C4900002D0019D494601E035465146384B0427FC
:10C4A00033F91430384A93FBF7F3A25C6FF04F076F
:10C4B000534393FBF7F3022C4FEA440C01EB0307C1
:10C4C0000FD13846CDF810C009F0F6FA2F4B30499D
:10C4D0001E221B6800F0E6FA09F008FD0746DDF8A9
:10C4E00010C0274B2B4A3CF803103CF902000BB25A
:10C4F0002CF802109BF85020181A042390FBF3F03C
:10C5000082B1CDF814C0049209F0D6FA22491F4B2B
:10C5100001EBC401049A1B6800F0C4FA09F0E6FCC0
:10C52000DDF814C01D4B1E4A1B5D5843202390FBB1
:10C53000F3F07B191B1A2CF802301A4B404243F8D7
:10C540002470194B43F82450184B43F82400009BE7
:10C5500001340133032C00937FF4F9AE07B0BDE83A
:10C56000F08F00BFAC0F002074180020F82D0020C1
:10C57000FC0E0020A81D0020F0D8FFFF842600201C
:10C58000C40E002080C1FFFF901D00207C260020EB
:10C5900074260020B81D00209C260020A41D002029
:10C5A000B4260020BC260020C8260020D426002067
:10C5B0002DE9F04F89B006938F4B0C461B888146BE
:10C5C000990703924DD540F2E631129B8B4AD889E8
:10C5D000B2F900301B1A03F2F3158D4203D8002B79
:10C5E000B8BF5B4201E04FF4FA73B2F90220101AAF
:10C5F00040F2E63200F2F311914203D80028B8BFAE
:10C60000404201E04FF4FA7099F84C503DB3984223
:10C61000B8BF1846C0F5FA7009F04EFA784909F02B
:10C6200053FB4FF07E5109F091F90646642090FBD0
:10C63000F5F009F041FA0146304609F091FA4FF061
:10C640007E5109F085F90021074609F027FC30B931
:10C6500038464FF07E5109F03FFC20B101E0002741
:10C6600001E04FF07E57C846E31C04930024049B6E
:10C67000022C13F8015F0493624B09D1B3F9040053
:10C680000A35684309F018FA5F4909F01DFB68E0B4
:10C6900033F914A062005046019209F00DFA0646E3
:10C6A000039809F005FA564909F00EFB0146304699
:10C6B00009F056FA554B064633F9140009F0FCF917
:10C6C0000146304609F044F9039B0646584209F0FA
:10C6D000F3F983463046594609F0E0FB48B9039820
:10C6E00009F0EAF983463046594609F0F5FB00B9EE
:10C6F000B346474A019BD05E09F0DEF90146584631
:10C7000009F024F9069B064633F9140009F0D4F920
:10C710000146304609F01CF93E4909F0D5FA364B7E
:10C7200083461E88F20704D5D9F8441009F018FA98
:10C7300017E005F114000AFB00F009F0BDF93249D9
:10C7400009F0C2FAB30705460CD5D9F84810584687
:10C7500009F006FA394609F003FA0146284609F0BD
:10C76000F7F80546630005932B4B2C4E33F9140064
:10C7700009F0A2F92A4B196909F0F2F90146284695
:10C7800009F0E4F8D8F82010824609F0E9F9254BC1
:10C790000546185D09F090F90146284609F0E0F9D0
:10C7A000214909F091FA022C019005D11F491E225E
:10C7B000336800F077F901903368504619460293C8
:10C7C000DFF874B009F0CCF9D8F82C1009F0C8F9EA
:10C7D000104909F0C5F95BF8241009F0B9F81449BB
:10C7E000A500064609F05AFB40BB3046114909F046
:10C7F00073FB20B30F4E22E074180020602D002040
:10C800000000FA43AC0F002000004842F82D002041
:10C81000FC0E002000002041C40E00207C260020D9
:10C82000E0260020702600200000C8427426002068
:10C8300000007AC300007A43841D0020374E4BF875
:10C840000560DFF804B1504655F80B1009F07EF88A
:10C850000299079045F80BA04FF07E5009F034FA8A
:10C86000079B0146184609F07BF999F850200346CA
:10C8700032B12B49029B01EBC40100F013F90346CE
:10C88000D8F83810184609F06BF9264B8246185D27
:10C8900009F012F90146504609F062F9224909F0FF
:10C8A00013FA2249824609F0F9FA38B9504620496C
:10C8B00009F012FB20B1DFF878A001E0DFF86CA0EE
:10C8C0000198314609F044F8514609F041F80CF05E
:10C8D0000DFB184BB0F57A7FA8BF4FF47A709842E1
:10C8E000B8BF1846059A144B0134D052019809F08C
:10C8F000FDFA124B08F104085851304609F0F6FAD7
:10C900000F4B5851504609F0F1FA0E4B032C585179
:10C910007FF4ADAE09B0BDE8F08F00BF00007AC370
:10C920009C260020702600200000C842000096C30C
:10C930000000964318FCFFFFB4260020BC26002010
:10C94000C8260020D4260020C01D0020034B002252
:10C95000DA621A6300221A605A6070477C1D002058
:10C9600010B50B4C0123E3704FF48060022384F870
:10C97000203000F0EFFB074A074B126D1B6852781E
:10C98000642101FB0233636123880133238010BDDE
:10C990008C2D00207C1D0020980F0020F0B5012474
:10C9A000B0FBF4F58D4201D34C43F9E70026D4B136
:10C9B000B0FBF4F504FB1500B4FBF1F41EB9002D37
:10C9C00001DC002CF3D1092D03F1010EEFB204DDDF
:10C9D000002A14BF3725572500E030253D441D703F
:10C9E00001367346E3E71C70F0BDF0B50124B0FBDF
:10C9F000F4F58D4201D34C43F9E70026D4B1B0FBE6
:10CA0000F4F504FB1500B4FBF1F41EB9002D01DCB4
:10CA1000002CF3D1092D03F1010EEFB204DD002A41
:10CA200014BF3725572500E030253D441D700136E1
:10CA30007346E3E71C70F0BD03685A1C026019706E
:10CA400070472DE9F843089E002B07468846144698
:10CA5000334614BF4FF030094FF0200913F8012B73
:10CA60000AB9254603E0002CFBDD013CF6E7002D6A
:10CA700004DD38464946C047013DF8E7354624EA1B
:10CA8000E474A01B284415F8011B11B13846C047B7
:10CA9000F7E7BDE8F883024B1868FDF7BDBF00BF9C
:10CAA000900E0020F8B507460C4648680021154650
:10CAB0001E4609F0E9F958B1284608F0FDFF104973
:10CAC00009F04EF801464FF07E5009F0FDF8606025
:10CAD0006168304608F03CFF0146304609F0F4F842
:10CAE000256806462946384608F030FF014630469C
:10CAF00009F036F80146284608F02AFF2060F8BD04
:10CB0000DB0FC9402DE9F04102780346202A00F1ED
:10CB10000100F9D0092AF7D02D2A02D10346414D50
:10CB200004E02B2A08BF03464FF07E551C46002622
:10CB3000234614F8012BA2F13007F9B209290DD8C8
:10CB40003949304609F00CF80646384608F0B4FF7B
:10CB50000146304608F0FCFE0646E9E72E2A17D1CA
:10CB6000314F234614F8010B3038C2B2092A0FD8CE
:10CB700008F0A2FF394609F0A7F80146304608F050
:10CB8000E7FE29490646384608F0EAFF0746E8E787
:10CB90001A7802F0DF02452A39D15A782D2A02D1BB
:10CBA0000233012704E02B2A14BF0133023300278C
:10CBB000013B002413F8012F303AD1B2092903D8E0
:10CBC0000A2101FB0424F5E7B4F59A7F28BF4FF44E
:10CBD0009A74A0464FF07E53B8F1070F07D9184654
:10CBE000124908F0BDFFA8F108080346F4E704F075
:10CBF000070434B118460C4908F0B2FF013C034663
:10CC0000F7E719462FB1304609F05EF804E04FF01F
:10CC10007E51304608F0A4FF0146284608F0A0FFE8
:10CC2000BDE8F081000080BF0000204120BCBE4C68
:10CC300030B5054687B00C4603A800210C220BF046
:10CC400048FF2846002109F047F920B12846284925
:10CC500008F07EFE03E02846254908F077FE2549C6
:10CC600008F07EFF09F042F9054680EAE070694667
:10CC7000A0EBE57007F000FF002DACBF20232D23B3
:10CC800068468DF80C300BF068FF012807D130237F
:10CC90008DF80D308DF80E308DF80F300CE0022835
:10CCA00005D130238DF80D308DF80E3004E00328C7
:10CCB00004BF30238DF80D30694603A80BF030FF18
:10CCC00003A80BF04AFF0338C5B22A4603A9204641
:10CCD0000BF06EFF00236355204607490BF020FF41
:10CCE00003AB204659190BF01BFF204607B030BD9F
:10CCF0006F12033A00007A4423BE010870B506465D
:10CD0000B6FBF2F40846154614B12046FFF7F6FFCD
:10CD100005FB1464024B1B5D00F8013B70BD00BFB6
:10CD200025BE01082DE9F04F81468A4616461C466D
:10CD300089B000253178002900F0DB80252902D058
:10CD40000136484674E072784FF00008302A0CBF74
:10CD5000B278B71CA2F1300312BF4FF0000BF71CE2
:10CD60004FF0010B092B19D8A2F13003D9B20929D0
:10CD700005D80A2202FB083817F8012BF4E7A2F1C4
:10CD80006103052B02D8A2F1570305E0A2F141038C
:10CD9000052B03D8A2F137030A2BEADD6C2A30D128
:10CDA0003A787E1C642A00F083800BD8252A3DD077
:10CDB00003D8002A00F09D80BCE7582A0CD0632AD3
:10CDC00019D0B7E7732A22D002D86E2A37D0B1E73C
:10CDD000752A5CD0782AADD1271D2068A2F15804AD
:10CDE00062424FF01001624155E02CD9582A32D0EE
:10CDF000632A2AD13E4648462178271DD04701356F
:10CE00000FE0642A63D00ED9732A14D13E462368FA
:10CE100048460093514642460023FFF712FE271D65
:10CE200005443C4686E7252ADFD13E464846252173
:10CE3000D04701357EE70AD86E2A06D13E462368E0
:10CE400004341D6076E7002A53D03E4672E7752A07
:10CE500026D0782AF9D1A2F1580304F1040C5A42E1
:10CE60002068CDF80CC04FF010015A4105ABFFF718
:10CE700095FDDDF80CC03E46644605AB0093484680
:10CE8000514642465B46FFF7DCFD054452E7206809
:10CE9000271D0A21002205ABFFF7A7FD3C46ECE762
:10CEA00004F1040CCDF80CC020680A210022DDE753
:10CEB0002068271D002808DA2D238DF81430404201
:10CEC0000DF115030A210022E6E705ABFAE7206819
:10CED00004F1040C00280ADA2D238DF814304042A6
:10CEE0000DF11503CDF80CC00A210022BFE705ABF8
:10CEF000F8E7284609B0BDE8F08F0FB413B50B4929
:10CF000004AB08680A4953F8042B09680193FFF73A
:10CF100009FF0446074B1868FDF772FD0028F9D099
:10CF2000204602B0BDE8104004B070476401002004
:10CF300060010020900E00202DE9F84321F000450B
:10CF400020F00046074688462846314608F0C4FFD0
:10CF500008B9344600E02C462046002108F094FF32
:10CF600060B92846314608F099FF08B9304600E01C
:10CF70002846214608F0A8FE044600E0002420468A
:10CF8000254908F0EDFD254908F0E0FC214608F0B0
:10CF9000E7FD234908F0DAFC214608F0E1FD2149CC
:10CFA00008F0D4FC214608F0DBFD1F4908F0CEFC58
:10CFB0001E4900F10049204608F0D2FD1C4908F046
:10CFC000C7FC214608F0CCFD4FF07E5108F0C0FCB4
:10CFD0000146484608F078FE29460446304608F0E7
:10CFE0007BFF20B12146134808F0B0FC04464046C0
:10CFF000002108F053FF20B121460F4808F0A6FC9D
:10D0000004463846002108F049FF08B104F1004405
:10D010002046BDE8F88300BF39094E3DE3B59E3E8A
:10D0200088FA163E45FE7F3FA7DFA83499FB243FD0
:10D0300069A2163EDB0FC93FDB0F494070B50446BD
:10D0400008F054FF2030402857D820462C4908F0DB
:10D0500043FF28B120462B4908F078FC0446F4E74A
:10D060002046294908F01AFF28B12046254908F032
:10D070006FFC0446F4E72046244908F02DFF30B148
:10D080002249204608F062FC014620480AE020467A
:10D090001F4908F003FF40B11C49204608F058FC26
:10D0A00001461B4808F052FC04462146204608F081
:10D0B00057FD05462046294608F052FD0021064648
:10D0C000284608F04DFD134908F040FC014628466B
:10D0D00008F046FD104908F03BFC0146284608F0E0
:10D0E0003FFD0E4908F032FC0146304608F038FD9D
:10D0F0000146204608F02CFC70BD002070BD00BF2A
:10D10000DB0F4940DB0FC940DB0F49C0DB0FC93FD4
:10D11000DB0FC9BF92E741399730083C15A82A3E7A
:10D1200008B5034908F014FCBDE8084086E700BFD5
:10D13000DB0FC93F064B10B51A881C4622EA0000D7
:10D140009042188002D00120FDF702FC208810BD1B
:10D1500074180020064B10B51A881C4610439042E4
:10D16000188002D00120FDF7F3FB208810BD00BF1E
:10D1700074180020024A936823EA00009060704708
:10D18000B40F002008B5104B1A780023D9B2914291
:10D1900007D20E49002051F8231001330968088096
:10D1A000F4E73220FDF78DFA094B1B685A0309D5C5
:10D1B000084B9B685B0305D4BDE8084040F2DC5097
:10D1C000FDF77FBA08BD00BF4419002014190020E4
:10D1D00094170020B40F00202DE9F34107F0F2FF6F
:10D1E0004B4A6C2313704FF4FC635380BE231371BE
:10D1F000EF2382F8DC3700231946164682F8DD3724
:10D20000F25C0133B3F5FC6F81EA0201F8D1404BC7
:10D21000404A83F8DD17404B04275A6002F18832F8
:10D220005A600020013F17F0FF075ED03A4B3422CE
:10D230003A4CDA6004F17848A8F5FC38C8F30903E1
:10D2400053B100234FF4005056F80880019303F0C7
:10D2500071FF0428E6D11CE04FF4302003F06AFF90
:10D260000428DFD12C4D4FF430202B6943F002030A
:10D270002B616C612B6943F040032B6103F05AFF73
:10D2800041F6FD732A69042803EA02032B61D8D012
:10D29000C8E7214D4FF400502B6943F001032B6187
:10D2A0001FFA88F3238003F045FF042813D1A31C41
:10D2B0000193019B4FEA1848A3F800804FF40050F7
:10D2C00003F038FF41F6FE732A69042803EA0203DB
:10D2D0002B6106D0A6E741F6FE732A6913402B6145
:10D2E000A0E70F4B04349C42A4D10B4A04281369D5
:10D2F00043F08003136102D106F003F810B9052052
:10D30000FDF73EFB07F048FF02B0BDE8F08100BF2B
:10D31000B40F0020230167450020024000F80108F7
:10D32000E0FF010810B50E4C2068FDF7EDF820680D
:10D330000022047A02FB02F3193B634303F6C41391
:10D340005343192193FBF1F3064921F812300132BE
:10D35000072AEFD1BDE810400349FDF78DB800BFA3
:10D36000040F0020600E0020F41000202DE9F04191
:10D3700005F0C7FF10B90420FDF702FBB04C07F021
:10D3800021FFB0494FF4FC6220460BF097FB94F864
:10D39000AC374FF4CC71022B84BF002384F8AC3738
:10D3A00094F8AC27A84D01FB02F3E01800F53970A2
:10D3B0002344286093F8380301FB0242022803F556
:10D3C0004C7384BF0020187292F838339F4A137050
:10D3D0000C2202FB03439E4A03F2AE73136046F233
:10D3E0000902A3681A401AB9954A43F4005393609E
:10D3F000A368DE0703D54FF40050FFF7BBFEA36818
:10D40000580409D50820FFF7B5FE4FF40050FFF788
:10D41000B1FE0120FFF7AEFEA368190706D54FF451
:10D420000050FFF7A7FE0120FFF7A4FEA3689A04AF
:10D4300013D54FF40040FFF79DFE814B93F88431E4
:10D44000012B03D14FF40060FFF794FE4FF48030BE
:10D45000FFF790FE4020FFF78DFEA3685B0603D523
:10D460004FF48030FFF786FE94F8DE21744B2AB12A
:10D4700093F8E22112B1002283F8E2214FF0000C70
:10D480006746744E744B1E6004EB0C03B3F8F6E170
:10D490004FEA5E0101F077314FEA9E0303F0333328
:10D4A000C1EB0E00C11A4FEADE0303F01133CB1AB1
:10D4B00003EB231303F00F32FF2392FBF3F31EF071
:10D4C0000108C3EB032318BF0137A2EB030318BF06
:10D4D000FFB2012B0ADD022B40F0AE80B8F1000F45
:10D4E00000F0AA801EF0BC0F00F0A6800CF1080C22
:10D4F000BCF1200FC8D1013F012F00F29D80FFF742
:10D5000011FF3022002155480BF0E3FADFF8A48127
:10D51000534B2F68C3F80080524B002107F179006C
:10D520001F60FDF72FF8504B80F0010018704F4B33
:10D5300008F128021A604E4B08F1D4021A603878BC
:10D5400004F066FF28684B4B00F5C5721A6001F0C5
:10D55000FBFF494B94F8D61108F196021A60642239
:10D560004A43464BC8325A6000229A60DA601A6118
:10D570005A619A61DA6183F8202083F82120404BB8
:10D580002F6808F12E021A603E4B07F219121A603A
:10D590003D4B07F289121A603C4B08F108021A60F1
:10D5A0003B4B3C4DC3F800803B4B08F1A2021A6094
:10D5B00008F1AC032B60394BB4F864011E6008F02D
:10D5C00077FAA860B4F8660108F072FA97F85C3050
:10D5D0002A1D2B7197F87830E8606B7194F8E1316F
:10D5E000386E2B742E4B6F611A6007F16403AB61C8
:10D5F0002C4908F0B5FA01464FF07C5008F064FB66
:10D60000B7F81641E861204608F056FA0146264868
:10D6100008F05AFB254908F0A3FA254B2F62186041
:10D6200007F1680307F211176B62AF62C5F82C802F
:10D63000BDE8F04107F0B0BD07F0D4F95FE700BFE7
:10D64000B40F002000F80108E00E0020AC280020F4
:10D65000040F00203C1100205C2D0020900D0020C4
:10D66000C40D0020C80D002002000020F826002074
:10D6700030060020D40D0020CC1D00208C2D002071
:10D680006027002050250020F4070020E819002022
:10D69000EC190020D01D002008070020CC07002036
:10D6A000D8270020DB0F4940000061444C3D0F4467
:10D6B00004070020F410002008B5FFF78DFDFFF7E8
:10D6C00055FEBDE808400120FDF742B9F8B5044613
:10D6D0000E4617460025204620210BF030FA04465E
:10D6E000D0B1013420460BF08DFAB0F5617F05DB37
:10D6F00040F634039842A8BF184601E04FF4617029
:10D70000A0F56170192390FBF3F00DB9307000E0C3
:10D7100070703B7801333B700DB90125DBE7204683
:10D72000F8BD30B505460C46134629462246BDE8ED
:10D7300030400148FFF7E1BB1CBF01087FB504780A
:10D740000646E4B9354B1921186800EB840090F8BF
:10D750007B5090F879204D4305F5617590F87A304B
:10D76000009590F87C00414301F5617101912C48CE
:10D7700021460134FFF7C1FB142CE3D14BE00BF041
:10D7800041FA1328054641DC244B701C1C682021FB
:10D7900000238DF80F300BF0D2F91E35064670B11C
:10D7A000013630460BF02EFA1A289FBF04EB850392
:10D7B00058709DF80F30013398BF8DF80F30304608
:10D7C00020210BF0BCF9064670B1013630460BF053
:10D7D00019FA0D289FBF04EB850398709DF80F3050
:10D7E000013398BF8DF80F3004EB85043046E11CFF
:10D7F0000DF10F02FFF76AFF9DF80F30042B0AD0DE
:10D80000601C002104220BF064F904E005480021AB
:10D810001322FFF786FF04B070BD00BFE00E0020AA
:10D820003BBF010850BF0108014806F021BB00BF03
:10D8300056BF01082DE9F04304788FB00546002C4F
:10D8400059D17B4B0021142209A807AED3F80080E0
:10D850000BF03FF90722304600210BF03AF9002384
:10D860001A46A70005A8059308EB070583807149B0
:10D87000B5F802E031F813C01CEA0E0F0AD00E31E1
:10D880000DF1380C595C02F1010E624402F81C1CC7
:10D890005FFA8EF20133072BE9D100210B46664A6D
:10D8A000B5F802E011F802C01CEA0E0F0AD00632E9
:10D8B0000DF1380C8A5C03F1010E634403F8242C4B
:10D8C0005FFA8EF301310629E9D118F807308DE8A7
:10D8D00041006A785949029209A81A0903F00F0316
:10D8E00007F0F8FD2146564809AA0134FFF705FB69
:10D8F000202CA6D198E00BF085F91F28044600F3F0
:10D90000868028462021E4B20BF019F91F2C02D999
:10D91000FFF78AFF88E0464B451C1B68002103EB9C
:10D920008404204604220BF0D4F80027454B09AEAE
:10D93000304600210A2217F803905FFA87F80BF0AF
:10D94000C8F8002315F8012B32B10A2B04D04A4540
:10D9500002D0F2540133F5E74A455ED108F1FF33B6
:10D96000032B09D8DFE803F01005023F0DF1230176
:10D9700034E00DF123011EE030460BF043F923782B
:10D98000C0B243EA001006E030460BF03BF92378C2
:10D9900000F00F001843207031E00133062B0AD04D
:10D9A000244800F11B069E5D9642F6D103445A7D41
:10D9B00063881343638011F8012F02B30023EFE75C
:10D9C0000133072B0AD01B4800F10E069E5D9642DC
:10D9D000F6D130F8132063881343638011F8012FC8
:10D9E0006AB10023EFE730460BF00CF90F2804DC96
:10D9F00030460BF007F9607001E0002363700137D7
:10DA0000052F93D1012400F017FE6CB980E70E4872
:10DA100000211F22FFF785FE06E020460021042298
:10DA20000BF057F80024EEE70FB0BDE8F08300BF1D
:10DA3000001E0020009F0108159F010864BF010817
:10DA400073BF0108219F010850BF0108F8B5047891
:10DA5000064674B9304D2146B5F8C421B5F8C63133
:10DA60002E480134FFF749FA042C05F10405F2D1E0
:10DA7000F8BD2B490BF036F8A8B9274B4FF47A7153
:10DA80004FF4FA62A3F8C411A3F8C621A3F8C81191
:10DA9000A3F8CA21A3F8CC11A3F8CE21A3F8D01182
:10DAA000A3F8D221F8BD30460BF0ACF803280546A8
:10DAB0002BD8304620210BF042F8044630B1013417
:10DAC00020460BF09FF80126074600E00646204658
:10DAD00020210BF034F810B9BDE8F840A4E601307D
:10DAE0000BF090F8012EF7D140F2DC53A7F2EE22B2
:10DAF0009A42F1D8A0F2EE229A42EDD8064B703548
:10DB000003EB85039F80D880F8BD064800210322DF
:10DB1000BDE8F84005E600BFB40F00207FBF010854
:10DB200092BF0108DDC801082DE9FF4104780546D0
:10DB3000002C34D16D4806F09BF96D4D2869002109
:10DB400008F0A2F9002840F0CE8021466948FFF78E
:10DB5000D4F928696946FFF76BF801466648FFF774
:10DB6000CCF968696946FFF763F801466248FFF738
:10DB7000C4F9A8696946FFF75BF801465E48FFF7FC
:10DB8000BCF9E8696946FFF753F8013401465B4880
:10DB9000FFF7B3F90C2C05F11005CFD1A3E05849DC
:10DBA00005220AF0E3FF38B9514B0022034410303C
:10DBB000C0281A61F8D196E02846524904220AF09A
:10DBC000D5FF04462846002C3FD120210AF0B7FF9C
:10DBD000002800F08880451C28460AF0BEFF074652
:10DBE000494B53F824601EB9484806F041F97AE0E1
:10DBF00028463146FAB20AF0B9FF01340028EFD1C5
:10DC00003B4B0021C2181030C02811619E46F7D14D
:10DC10003F4B03EBC402D2F804C09846BCF1000F9E
:10DC200004D131463B48FFF768F953E0002718F864
:10DC300034309F42F5DA3B010EEB030510356344A7
:10DC40000FCB013785E80F00F1E70AF0DBFF0B2867
:10DC5000064643DC284620210AF071FF054648B1FC
:10DC600001352846FEF74EFF214B012403EB061336
:10DC7000186100E00446284620210AF060FF0546AE
:10DC800040B101352846FEF73DFF194B013403EB47
:10DC900006135861284620210AF051FF054640B17D
:10DCA00001352846FEF72EFF114B013403EB061316
:10DCB0009861284620210AF042FF10B9FFF7B4FD11
:10DCC00011E00130FEF71EFF094B032C03EB061693
:10DCD000F061F3D11048FFF727FF04E00F4801215E
:10DCE0000C22FFF71EFD04B0BDE8F08198BF0108CB
:10DCF000B40F0020B3BF0108B9BF01085BC601081B
:10DD000092BF0108BDBF0108F0A50108C2BF01080C
:10DD10004CBE0108D1BF0108B1BC010850BF0108C9
:10DD2000F0B5047887B0064614BB514B192019682A
:10DD3000062303FB041191F8CA5091F8CE20454305
:10DD400005F5617591F8C930009591F8CB50C8314F
:10DD5000684300F56170019008790290497945485F
:10DD6000039121460134FFF7C8F80C2CDDD17CE08B
:10DD70000AF048FF0B28044672DC3D4B701C1D68FE
:10DD8000202100238DF817300AF0D9FE064680B115
:10DD9000013630460AF036FF03289FBF062303FBF7
:10DDA000045383F8CE009DF817309CBF01338DF8E3
:10DDB0001730304620210AF0C2FE074680B10137F5
:10DDC00038460AF01FFF0D289FBF062303FB0453AC
:10DDD00083F8C9009DF817309CBF01338DF81730C8
:10DDE00006266643A9193846CA310DF11702FFF716
:10DDF0006DFC20210AF0A3FE074670B101373846BA
:10DE00000AF000FF14289FBF9DF8173076190133E0
:10DE100086F8CC0098BF8DF81730384620210AF0DC
:10DE20008EFE78B101300AF0EDFE0D289FBF06236B
:10DE300003FB045383F8CD009DF817309CBF0133DA
:10DE40008DF817309DF81730062B0ED0062202FBF6
:10DE500004500021C9300AF03CFEFFF7E5FC04E065
:10DE6000054800210B22FFF75CFC07B0F0BD00BFA6
:10DE7000E00E0020DDBF010850BF0108F0B50278B8
:10DE800087B08AB94A4C04F1200694F8F4210023A3
:10DE9000484950B2595681426DD00C33302BF7D1DE
:10DEA0000834B442F1D180E0002204920592451C6E
:10DEB0000AF0A8FEC4B260B2FCF7A0FA074618B197
:10DEC0008DF81040012400E00446284620210AF085
:10DED00036FE054638B1013528460AF093FE013476
:10DEE000ADF81200E4B20026284620210AF027FEF1
:10DEF000B0B3451C28460AF085FE00222E495FFA81
:10DF000082FE51F82230834204D00132082AF5D132
:10DF1000002300E0734651F82320824220D1022ED4
:10DF20000FD0032E12D05A1E012ED2B204D0042AD2
:10DF300013D88DF814300EE0042A0ED88DF8153061
:10DF400009E0052B09D88DF8173004E09A1E052A40
:10DF500003D88DF816300134E4B20136042EC3D153
:10DF6000052C03D807B0BDE8F0405DE404AB03CB5B
:10DF70003860796019E094F8F9010F4B94F8F85182
:10DF800053F82000B4F8F621009094F8FB0153F800
:10DF90002000019094F8FA0153F8200053F825303E
:10DFA00002900648FEF7A9FF7AE707B0F0BD00BF70
:10DFB000B40F0020A42B0020DCB70108FDBF01082E
:10DFC0002DE9F347047807464CB9204601A906F02D
:10DFD00053FD0134FFF7F4FF122CF6D17DE00AF077
:10DFE00011FEC5B2112D73D8781C20210AF0A7FDAF
:10DFF0003B4C05F1D00614F816800346394F30B972
:10E00000A8F10202D2F1000848EB020846E007F14D
:10E01000260800F1010A597840460AF090FD68B1DF
:10E02000032D8CBF03230023C8EB0000C0B23B4488
:10E03000184490F82A90B9F1030F02D1FFF7F4FBCE
:10E040004BE0A9F10203D3F1000850464FF0200144
:10E0500048EB03080AF073FDD8B1B8F1000FEDD01A
:10E0600001300AF0CFFD40F2ED2380B2984205DD89
:10E0700040F6CA039842A8BF184601E040F2EE20DD
:10E08000A0F2EE20192290FBF2F004EB4603587048
:10E0900002E0B8F1000FD1D104F8169014F8163050
:10E0A0001F4497F82620B8F1000F0CD00C4B0E48F7
:10E0B00003EB4606717819234B43294603F2EE23FE
:10E0C000FEF71BFF09E029460848FEF716FF04E0AB
:10E0D000074800211122FFF724FB02B0BDE8F087BA
:10E0E000B40F0020009F01081CC001082EC00108C9
:10E0F000DDC8010807B50123ADF8041001A98DF8AA
:10E1000006208DF8073004F0AFFE03B05DF804FB85
:10E110002DE9F041044672B63E4E4FF400614FF4D3
:10E1200080677161304648227761FFF7E3FF304630
:10E1300039461022FFF7DEFF374B03EBC40250686D
:10E1400053F834504FEAD00E344B05EB8E025A6030
:10E1500055F82E2000F007019A608900DA600F223E
:10E160008A40D2439846DC681440DC609C682240B8
:10E170009A60DC6808228A402243DA609A680124A7
:10E1800004FA01F10A439A609A68844045F82E2007
:10E190002C613761B3681905FCD440F60557D8F8EF
:10E1A0000820D8F804301A601A4B4FF480626C6172
:10E1B0005A6108221A61174EB3681A0503D4002F5A
:10E1C000F9D0013FF7E72C612846A1B24822FFF7BA
:10E1D00091FF7FB10F4A93681B05DED5AB684FF402
:10E1E00080611C424FF0080315BF1161516113613A
:10E1F0005361EFE74FF480610823316130463361AA
:10E200001822FFF777FF62B6BDE8F0410A20FCF75D
:10E2100058BA00BF000C014040C00108001E002099
:10E2200010B504462046FCF7EBFB18B90A20FCF7B2
:10E2300048FAF7E710BD002207490C2303FB02133D
:10E240005968814204D10022C2621A725A60704732
:10E250000132042AF0D17047A42B0020022803D0F9
:10E26000431E584258417047064B1B681B7823B128
:10E27000054B1868C0F3C0407047044B1878C0F3D2
:10E280008000704730060020A40E0020002E0020E1
:10E2900010B50A4C5E280146206805D15D21FCF7C7
:10E2A000BBFB20683E2105E05D2903D1FCF7B4FBF0
:10E2B00020683D21BDE81040FCF7AEBB101E0020D9
:10E2C0000028114AB8BF404290FBF2F330B50F4C22
:10E2D0003C2504FB030068430D4D90FBF2F22D68D2
:10E2E0002D7B25B903EB830303EB830301E0C3EB31
:10E2F000031302EB830304FB02020B804FF47A73D7
:10E3000092FBF3F24A8030BD80969800806967FFE7
:10E31000A017002010B50446C0B2FFF7B9FFC4F340
:10E320000720BDE81040B3E7024B5E211868FCF7F8
:10E3300073BB00BF101E002038B50546054C5E219A
:10E340002068FCF769FB20682946BDE83840FCF7E7
:10E3500063BB00BF101E0020674B73B51878FFF732
:10E360007DFF664D04462B78834220D0C8B1644BB4
:10E370001B68E3B193F9000002230093614B042171
:10E380001B6800225B78003318BF012301934FF410
:10E390001653FCF7A0F95C4B186040B101232B70B9
:10E3A00005E0594E3068FFF746FF34602C70574B3C
:10E3B000574D1878FFF752FF2B780446834218D048
:10E3C00088B1544B1B68A3B10022012493F90000CB
:10E3D00008214FF4964300940192FCF77CF94E4BD0
:10E3E000186028B905E04C4E3068FFF724FF346010
:10E3F0002C704A4B4A4D1878FFF730FF2B780446B3
:10E4000083422E4643D0002838D0464B1A68002A53
:10E410003DD0D37992F90000002B4FF00202424C1C
:10E4200008BF02230092002254F8233001921021E9
:10E43000FCF751F93D4B0546186040B33C4C94F84D
:10E440004A30022B0BD094F89620022A01D14C348A
:10E4500005E023B1002A04F14C0418BF0024354B19
:10E460001C6044B1204600214C220AF032FB0223FA
:10E47000256084F84A300123337008E02B4E306861
:10E4800005F000FC3068FFF7D6FE34602C702A4B94
:10E490002A4D1878FFF7E2FE2B780446834229D0F4
:10E4A00000B3274B1B682BB3264A93F90000126870
:10E4B000032352782021002A0CBF0822092200934E
:10E4C00001924FF461430022FCF705F91E4B1860DE
:10E4D00080B11E4A012313702B701D4B1A681D4B0F
:10E4E0001A6007E0184E3068FFF7A5FE174B34603E
:10E4F0001C702C7002B070BD38060020940F0020F4
:10E5000034060020A0170020101E0020390600202D
:10E51000C0170020441800203418002044060020B2
:10E520004A18002040060020DCB701084C180020E3
:10E53000FC2A0020501800205006002060180020FF
:10E540004C060020480600206418002068180020AF
:10E55000980F00206C18002010B54B88DC0641BFD6
:10E560002F4B14791B6853F8244044BF2D4B43F8BC
:10E5700020404B889B0641BF294B54791B6853F8B8
:10E58000244044BF274B43F820404B881C070ED53E
:10E59000254B0C781B78B3EB141FA1BF204BD4780C
:10E5A0001B6853F82440A4BF1E4B43F820404B88FF
:10E5B0009B070ED51D4B0C781B78B3EB141FDFBFE8
:10E5C000174B54781B6853F82440DCBF154B43F8B5
:10E5D00020404B88DC070FD5154C0B78247803F0CE
:10E5E0000F03A342DFBF0E4B14781B6853F824407F
:10E5F000DCBF0C4B43F820404B885B070FD50B78F2
:10E600000C4903F00F0309788B42A1BF044B9278A9
:10E610001B6853F82220A4BF024B43F8202010BDF2
:10E620004C2500203A0C0020D30C0020D10C0020F7
:10E63000D00C0020D20C0020254A0023F0B515682C
:10E640001C461A462348244903700B712E197688FC
:10E650004EB92F5D3FB9037000230A714B710778E3
:10E660001C461A460CE0360548BF013204F104048A
:10E6700003F1010348BFD2B2802CDBB2E6D1EAE756
:10E68000E0B2B8420CD215F82400013406099E42CB
:10E6900000F00F00A8BF731C9042A8BF421CEFE718
:10E6A0008A714B71C2F3470102F001020A444C1E09
:10E6B0000A490B480A70C3F3470203F001031344ED
:10E6C00004700849501E084A08701370F0BD00BF5E
:10E6D000001E0020C80C0020101E0020D20C0020BC
:10E6E000D00C0020D30C0020D10C0020924B2DE93F
:10E6F000F04FDA68914D1A612A6891B0DA60904A59
:10E700000295136843F0200313608E4B1A78012A98
:10E710000CBF002201221A708B4B1A78910740F12E
:10E720004D838A490978042940F248838849097849
:10E7300001F0040101F0FF0011B922F001021A708A
:10E740001B78DB0702D408B100F04EFF8149CA797B
:10E75000531C052293FBF2F202EB82029A1A7E4BC3
:10E76000CA711F7892000023DFF81082DFF8109240
:10E7700058F82310794C91FBF9FE04F1080040F899
:10E7800023E0774844F8231000FB0E1142F210708A
:10E7900091FBF0F004F1100680B226F813004FF060
:10E7A000140C04F114060CFB036C04F13C0A5AF837
:10E7B00023605CF802504CF80210761B31440526A9
:10E7C0004AF8231091FBF6F109FB0E114434012F96
:10E7D00044F823104FEA830B444605D10238B0F5C4
:10E7E000797F98BF4BF808100BB90123BCE7594E4D
:10E7F000029BB2461868736DC01A07F059F959495F
:10E8000007F062FA029B4FF07E511B680746736562
:10E8100007F044FB08B94FF07E574B4BCAF85870CD
:10E820001B78514E13F00103504D12D00DAA0092E7
:10E830004F4B0EAA01920CCB94E8030000F0EAFDC6
:10E840000D9A6421B2FBF1F20E9B328093FBF1F33F
:10E8500000E033802B809AF85C303E4D002B35D0A1
:10E86000A96D4FF07E5007F02FFA07462B6E2068F7
:10E87000C01A07F021F9394607F072F907F036FBA4
:10E880006B6E86B2606836B2C01A07F015F9394B64
:10E89000196807F065F9394607F062F907F026FBB9
:10E8A000B5F96A2000B28118B5F968200220B318C2
:10E8B00091FBF0F193FBF0F389B29BB2A5F86E10D7
:10E8C000A5F86C30A5F86A10A5F8683001238AF81D
:10E8D0005C30294B61681B88206803F030031D4EB3
:10E8E000264DCAF86410CAF86000002B00F066825A
:10E8F00006F17803009306F17C030193326F736F86
:10E9000000F088FD6B68706FC01A07F0D5F8194BDE
:10E91000196807F025F907F0E9FA336F2A68C6F895
:10E9200084009B1AC6F880300B4B1B78012B29D032
:10E93000022B00F0E58041E294060020980F0020B1
:10E94000AC1700200A0F0020B0170020B6170020D7
:10E95000002E0020101E0020D00D0020181E0020C8
:10E96000806967FF00007A442A1800202C180020D4
:10E970000C0F00203C00002074180020B817002065
:10E9800080969800D6F88830D6F8A4400293D6F83E
:10E99000983004F100400393D6F89C30B76D05938E
:10E9A00007F0A4FA8146204607F0A0FAD6F8A03076
:10E9B000BB4C0493BB4B06901B684FF0000B0793B6
:10E9C000B94E4FEA4B0356F82B80A6F1140240468D
:10E9D00032F81B50089307F06FF8029907F0C0F85F
:10E9E00007F084FA401B1FFA80FA283626F81BA08D
:10E9F0000FFA8AFA504607F05FF8039907F0B0F86B
:10EA000007F074FA86B20AEB080007F055F805998A
:10EA100007F0A6F8394607F0A3F8216806F098FF3A
:10EA200007F064FA484504DB069B9842A8BF1846E5
:10EA300000E0484607F040F8206007F057FA079BCF
:10EA4000304486B2987807F033F8984907F088F890
:10EA500001464FF07E5007F037F9394606F078FF4F
:10EA60000146384607F030F909906068D4F808A0EC
:10EA7000C0EB080007F020F8394607F025F95146A9
:10EA800006F064FF099A0146104607F069F801464E
:10EA9000504606F05DFF3135ADB2622D0146206172
:10EAA000C4F80480A0600ED9049807F059F807F064
:10EAB0001DFA7F4AB0F5FA6FA8BF4FF4FA60904292
:10EAC000B8BF104600E0002040F6B832064436B227
:10EAD0009642A8BF1646774A089B9642B8BF16468C
:10EAE000754A54F8140B9E52142202FB0BF2734920
:10EAF0005050BBF1000F40F061814FF0010B5FE718
:10EB0000684BB6F8AC401F68B36F3D8902935B0851
:10EB10009D4228BF1D4623B29D4202DC1FFA85F9A3
:10EB20000AE06749B06D07F01BF807F0DFF92044F1
:10EB30001FFA80F9A6F8AC90DAF87C60DAF8B040F9
:10EB4000341B204600F0A8FC41F293130028D8BFE4
:10EB500040429842CCBF0020012078B3204606F006
:10EB6000ABFF584906F0FCFFFEF768FA044602982E
:10EB700006F09EFF0146204606F0F2FF07F0B6F9C8
:10EB800040F6B83380B2AAF8B40000B29842A8BFE9
:10EB90001846484B9842ACBF3018F01848F6A043CE
:10EBA000984203DDA0F50C40A03804E00028BCBF6B
:10EBB00000F50C40A030CAF8B80001E0CAF8B8600F
:10EBC000DAF8B8300026C3F50C502830039306F06D
:10EBD00073FF3C4906F0C4FF0446FEF7A1FA0F900C
:10EBE0002046FEF72BFADAF8BC30DAF8C840059375
:10EBF000DAF8C0300E9004F10040089307F076F97F
:10EC00000490204607F072F9DAF8C430DAF8588038
:10EC10002A4C09900793730048460A9306F04CFF6C
:10EC20000EAB53F8261006F09BFFDFF8A0A00546B8
:10EC30003AF9160006F040FF0146284606F086FE27
:10EC400007F054F905B2204BB5F57A7FA8BF4FF411
:10EC50007A759D42B8BF1D460AF13C0AA8B22AF84F
:10EC6000160000B206F028FF0599824606F078FFEC
:10EC700007F03CF9089983B25046069306F070FFFE
:10EC8000414606F06DFF216806F062FE07F02EF99E
:10EC9000049B98421CDB099B9842A8BF184618E0C9
:10ECA0000C0E0020D40D0020901E0020DB0FC94068
:10ECB00030F8FFFF48F4FFFFDE0D0020340E002087
:10ECC0000000C842D302373918FCFFFF7C1E002029
:10ECD000049806F0F1FE20608346B87806F0E8FE5E
:10ECE000384906F03DFF01464FF07E5006F0ECFF3C
:10ECF000414606F02DFE0146404606F0E5FF0B902A
:10ED00006068D4F808A0281A06F0D6FE414606F03E
:10ED1000DBFF514606F01AFEDDF82CC001466046C6
:10ED200006F01EFF0146504606F012FE65600146E1
:10ED30002061A060079806F013FF07F0D7F8069B44
:10ED40001434034458469A4607F0D0F840F6B832D7
:10ED5000504400B29042A8BF10461B4A0A9B904202
:10ED6000B8BF1046194A1A4998521422724342F801
:10ED700001B00EB901264EE73B792BB1039A64230B
:10ED800092FBF3F3134A13803B88029A124C9A4287
:10ED90000DD9D4F8B030E06FC01A00F07DFB42F21C
:10EDA000107380EAE072A2EBE0729A4206DD0B4B30
:10EDB00001221A70B4F8CC20064B1A8011B0BDE8BD
:10EDC000F08F00BFDB0FC94048F4FFFFDE0D0020CD
:10EDD0000C0E0020CC0D0020101E0020D00D0020B5
:10EDE00010B506F069FE0021044607F075F808B179
:10EDF000204601E004F10040054906F065FF0549A1
:10EE000006F0AEFEFEF78CF9034B186010BD00BF94
:10EE10008096184B35FA8E3C3C000020F8B59A4B92
:10EE200005461B68187818B1012800F06281D6E207
:10EE3000242D964C0CD006D80A2D00F0D7800D2D2D
:10EE400000F0D48040E12A2D06D02C2D04D03BE1E7
:10EE500020706070A07048E18D4B617827780020A9
:10EE60008A4A58542FBB1978D770472921D159782D
:10EE700050291ED19978472907D1D978472904D13B
:10EE80001979412901D10121D1709978804A5229FB
:10EE900003D1D1784D2900F0A48299787C4A472982
:10EEA00007D1D178532904D11279562A04BF0322FD
:10EEB000E270E278754E022A38D0032A4BD0012A3C
:10EEC00040F08380BA1E072A7FD8DFE802F00408EA
:10EED0000F131A257E2A06F079FA606075E01B7818
:10EEE000532B72D163685B4263606EE006F06EFA8A
:10EEF000A0606AE01B78572B67D1A3685B42A360D0
:10EF000063E01B78302B634B1A788CBF42F002020F
:10EF100022F002021A7058E0002006F0B7FA2073BF
:10EF200053E0002006F0B2FAE0814EE0072F06D051
:10EF3000082F4AD1012006F0A9FA708245E001208D
:10EF400006F0A4FA41F2184358434FF47A73B0FB29
:10EF5000F3F0308239E0022F07D0032F0AD10020CE
:10EF600006F094FA4C4B18702FE0002006F08EFA51
:10EF700030752AE029D93A1F9210337D0132D2B27E
:10EF8000013B02EB8303DBB2102B1ED8F91EC2F14A
:10EF9000010201EB8202D2B2012A0BD0042A11D164
:10EFA00000205E1E06F072FA3C4B002298553C4B46
:10EFB0009A5507E03B4A5E1E0020935506F066FA1C
:10EFC000394B9855A3690133A361304B2A2D18BFE3
:10EFD0009A7807F101074FF000000CBF012255405D
:10EFE000277060700CBF1A779D707EE0207F00282C
:10EFF00047D02E4B13F8012D2D495A708B42F9D171
:10F00000234A224D13785278402B85BF373B1B0192
:10F010001B01DBB298BF03F0F003402A8CBF373AE4
:10F02000303AD2B21344A278DBB29A4226D12123DD
:10F030000B70E8782B6A012803F101031C4A2B624C
:10F040000AD002281CD1722313702A8A194B1A8005
:10F050006A8A194B1A8013E0672313700D4B1B78D3
:10F060009F070ED5154B6A681A60AA685A602A7BFA
:10F07000134B1A70EA89134B1A8002E03F230B707E
:10F0800000200023237730E0B4060020E01E00209B
:10F09000CC2D0020B0170020200F0020510F0020A1
:10F0A000410F0020210F0020310F00200403002019
:10F0B000F0020020B2170020080F0020B81700202F
:10F0C000B6170020B41700206378207F0E2B9FBF57
:10F0D000A84A591C5170A84A98BFD554A54A18B9D6
:10F0E00093785D40957000E00020003018BF01204B
:10F0F000F8BDA04B002293F82410082900F26F817C
:10F10000DFE801F0050C101A2B3B5E788500B52D69
:10F1100040F0658183F8252001224EE0622D08BF72
:10F1200002224AE0032283F8242083F8265083F841
:10F13000275083F8285052E1042283F8242093F8C2
:10F14000272093F828102A44D2B283F827200A44B3
:10F1500083F8282083F8295041E1052283F82420F0
:10F1600093F8272093F828102A44D2B283F8272056
:10F170000A4483F828205D8531E1062283F82420A3
:10F1800093F8272093F828102A44D2B283F8272036
:10F190000A4483F828205A8D02EB0525ADB2B5F557
:10F1A000AC7F82BF734A012182F8251000225D8561
:10F1B0009A85002D40F01381072283F824200EE168
:10F1C00093F8272093F828102A44D2B283F82720F6
:10F1D0000A4483F828209A8DB2F5AC7F3EBF65497A
:10F1E000891881F830500132598D92B291429A8536
:10F1F000E2D9F4E0082283F8242093F82730AB42C8
:10F2000000F0ED805B4B012283F825200FE05B4C82
:10F2100083F8242014F8012D6270594A9442F9D1E0
:10F2200093F82810534AA94206D03F232370554A29
:10F23000536801335360D2E0116A92F8250001311E
:10F24000116210B13E232370C9E02121217092F890
:10F250002910062941D004D8022907D0032923D038
:10F26000F8BD122959D0302967D0F8BD502121703E
:10F270004549546B4C60946B0C60116C4FF47A747C
:10F2800091FBF4F1414C218092F88811404A19B168
:10F29000117841F0020102E0117821F002011170B1
:10F2A000012283F889218CE05321217092F83510D6
:10F2B000CE0705D592F83420D51E6A426A4100E097
:10F2C000024602F0010183F88811002A79D1304901
:10F2D0000A7822F002020A7073E04F21217092F83E
:10F2E0003B10CC0705D592F83A20D11E4A424A413C
:10F2F00000E0024602F0010183F8881122B9244996
:10F300000A7822F002020A7093F85F10214A117005
:10F31000B3F85C10204A118053E056212170546CE0
:10F320001E490C8042F21074916C91FBF4F11C4C5C
:10F330002180012182F88A1143E04921217092F84D
:10F340003410184A102988BF1021117016491478FA
:10F350000022A24232D20E7A144D56554E7A144DE6
:10F360005655CE7A134D565511F80C6F124D565511
:10F370000132EEE7E01E0020CC2D00200403002027
:10F38000F002002094060020B8170020B4170020D7
:10F39000B0170020B6170020E2000020B2170020AE
:10F3A000080F0020200F0020101F0020210F002038
:10F3B000310F0020410F0020510F00209A690132C7
:10F3C0009A6193F889310B4A93B192F88A317BB1F3
:10F3D000002182F8891182F88A111846F8BD0020B0
:10F3E000F8BD1279432A7FF458AD0222E27054E549
:10F3F000F8BD00BFE01E00200449054B096800224B
:10F4000018705A6199611A77704700BF980F0020F1
:10F4100094060020F8B5101A0D461F4606F04CFB66
:10F420000446781B06F048FB174B079E196806F048
:10F4300097FB21460546204606F092FB29460746E3
:10F44000284606F08DFB0146384606F081FA09F0A1
:10F45000DDFD0E4906F084FB06F06EFD069B294695
:10F46000186004F10040FDF767FD094906F078FBDC
:10F47000084906F06DFA06F039FD0028BCBF00F51A
:10F480000C40A0303060F8BD3C0000202C7D8E3F49
:10F49000A00CB34500A00C4644F25063984203DD33
:10F4A000A0F50C40A0387047034B9842BCBF00F554
:10F4B0000C40A030704700BFB0B9FFFFF7B503683C
:10F4C000174C184D23600B68174E63600068FFF7F8
:10F4D00087FC95E80300154B0196009394E80C0017
:10F4E000FFF798FF3668124B60681E606B68114F1B
:10F4F000C01A06F0E1FA104B196806F031FB06F06D
:10F50000F5FC2A68236878609B1A3B600B4B1E60F1
:10F510000B4B1B68DA880B4B1A8003B0F0BD00BFA1
:10F52000801E0020B81700208C1E0020881E00209E
:10F53000C81E0020901E00203C000020C01E00209D
:10F54000D40D0020BC1E002070B50446407906F0A2
:10F55000AFFA1E4906F0B8FB1D4D1E4E2860E07B39
:10F5600006F0A6FA194906F0AFFBEE606860A079D4
:10F5700006F09EFA184906F0A7FB184D2860207C7B
:10F5800006F096FA114906F09FFB6860A07E06F02F
:10F590008FFA134906F098FBEE60A860E07906F058
:10F5A00087FA0D4906F090FB0E4D2860607C06F04E
:10F5B0007FFA064906F088FB6860E07E06F078FA7C
:10F5C000074906F081FBEE60A86070BD0000C842EC
:10F5D000981E00200000FA4400002041A81E0020D0
:10F5E00000007A44CC1E002010B50C4C23789B07F9
:10F5F00013D50B4B1B78042B0FD90A4A0A4B106802
:10F60000526818605A60FFF7EBFB084B1A88084BEA
:10F610001A80237843F00103237010BDB017002037
:10F62000B6170020B81700200C0F0020A80F0020EC
:10F63000DC1E0020094A137818441346C0B210F0AB
:10F64000800F18BF80381070054A197813789942D6
:10F6500001BF00231370014A13707047292800204E
:10F660002828002010B50A4B0A4A1B7842609C18D3
:10F67000094A046012789A4225BFD31A0B60C3F17D
:10F68000800300232EBF4B600B604A6010BD00BF9B
:10F69000292800202A280020282800201FB5684695
:10F6A00002A9FFF7DFFF044B02981B68034403988D
:10F6B000184405B05DF804FB540600202DE9F04F16
:10F6C000814689B002930023039104920193049A26
:10F6D000934207DA039A019952F823200133114427
:10F6E0000191F4E7029B019D002B57D103F0AAFC86
:10F6F000002853D102987FE00222414E8DF81C2051
:10F700001A0C4FF480578DF81D2006201A0A8DF828
:10F710001E208DF81F3003F0BDFC776106213948AB
:10F72000F9F74EFA384B01223761C8461A707761F3
:10F7300026463448002107AA0423F9F713FA039F49
:10F740004FF0000A049B9A451DDABC4657F8043B6B
:10F750004FEA8A0B002B48D0B34235D333462948B1
:10F76000002159F80B20CDF814C0F9F7FBF959F82E
:10F770000B30DDF814C0334449F80B30DCF80030AE
:10F780009E1BCCF800601E4B4FF480521A611F4A3A
:10F790002D1B13681C44029B14605BB355B31B4BB9
:10F7A0001B68DCB22A19B2F5807F194A88BFC4F5FC
:10F7B0008074D26898BF2C4693429DD3154A00238B
:10F7C0001370154A137015E0D8F800200D48002179
:10F7D000F9F7C8F957F8043CD8F80020F61A134492
:10F7E000C8F80030002347F8043C0AF1010A08F188
:10F7F0000408A7E7019B581B09B0BDE8F08F00BFC4
:10F80000000C014000380040510600205406002042
:10F8100004000020282800202928002030B50B4CA7
:10F820000B4D22782B7885B09A420CD0684602A9FD
:10F83000FFF718FF0123684602A90222FFF73EFFE7
:10F8400000232B70237005B030BD00BF2928002095
:10F850002828002030B50E4D0E4C2A78237885B02C
:10F860009A4211D0684602A9FFF7FCFE002302A9C4
:10F8700002226846FFF722FFFFF7DCFE20782B7894
:10F880001B1A5842584100E0012005B030BD00BFAE
:10F89000292800202828002070B50F4C0F4E4FF467
:10F8A000805545F2082003F0F5FB062165613046DE
:10F8B000F9F786F90A4B0122256130461A70C721F3
:10F8C0006561F9F77DF9074A002325611370064A3F
:10F8D0001370064A136070BD000C014000380040F0
:10F8E0005106002028280020292800205406002046
:10F8F0000148024900F0BEB800080040C0190020CD
:10F900000148024900F0B6B80004004098190020F0
:10F910004FF08040014900F0ADB800BF70190020E1
:10F920000148024900F0A6B8002C01404819002007
:10F930000148024900F09EB8002C014048190020FF
:10F94000026D70B515880446ADB2A90613D5036BD8
:10F950008BB9C36A1BB1908880B298470BE0E1690C
:10F96000928840694E1CD2B2E6614254E169E26875
:10F97000914228BFE3612B0613D5636AA26A9A42BB
:10F98000236D0AD0511CA069A162825C9A80236910
:10F99000994206D30023A36270BDDA6822F0800288
:10F9A000DA6070BD026B0346C16810B5406942B1B0
:10F9B0001A6C8C1A013A08BF0A46005D1A64C0B27C
:10F9C00010BD1A6A805C01328A4228BF0022C0B290
:10F9D0001A6210BD436B13B190F844007047836AFC
:10F9E000406A1B1A584258417047036B13B15B6859
:10F9F000016C01E0C369016A8B423CBFC2689B187D
:10FA0000581AC0B27047836A8169426B1944D16049
:10FA1000416A994297BF0169CB1ACB1A536096BFCE
:10FA20000023536083624FF0000380F84430136872
:10FA300088BF816243F0010313607047436A8269A3
:10FA4000D154436A02690133934228BF00234362C1
:10FA5000436B1BB11B68DB0705D4D4E7026DD36889
:10FA600043F08003D36070474171FBF7BBBB8160FB
:10FA7000FBF7B8BB2DE9F04105460E46078A83899E
:10FA80009BB21F40002F37D0B7FA87F24FF00043E8
:10FA9000D340DB4399B21F40A2F11B032982042B00
:10FAA000F0D8DFE803F0221F1C190300746A24B1A8
:10FAB000013C0023A4B2736201E0AC8DA4B2D6F87D
:10FAC0002080B8F1000FDDD0D8F800304046214644
:10FAD0009847D8F80480F4E73068A98E08E0706889
:10FAE000298F05E0B068A98F02E0F068B5F84010F2
:10FAF000036889B29847C5E7BDE8F081254B10B58A
:10FB00005A43254B254C1B680139B3FBF2F203889D
:10FB1000013AA04289B292B29BB212D004F50064BD
:10FB2000A0420ED0B0F1804F0BD0A4F59834A04283
:10FB300007D004F58064A04203D004F58064A0429D
:10FB400002D123F070039BB2154CA04206D004F5FD
:10FB50008064A0421CBF23F440739BB203800F4B10
:10FB60008185984202850FD003F5006398420BD03F
:10FB700003F54063984207D003F58063984203D0B1
:10FB800003F58063984201D1002303860123838219
:10FB900010BD00BF40420F00EC000020002C0140CF
:10FBA0000010004073B505460068FFF7A7FF2A68FC
:10FBB0000124138800269BB243F001031380EB7AE3
:10FBC00001A88DF804308DF805408DF806608DF899
:10FBD000074005F031FBEB7A1B2B0BD1192301A851
:10FBE0008DF804308DF805408DF806608DF80740DB
:10FBF00005F022FB02B070BD0C4B800A98420CD07D
:10FC000004D8B0F5801F0CD101207047084B9842F2
:10FC100005D04933984206D003E002207047032004
:10FC20007047FE2070470020704700BF01001000A1
:10FC3000020010002DE9F843046807462046884674
:10FC40009146FFF7D9FF03284BD8BA7A9108B8F14B
:10FC5000000F06D1A589AEB202258D4026EA050522
:10FC6000A5810A2303FB00131F4A42F823800433B3
:10FC700042F82390B8F1000F07D0BD7AA189AD08F2
:10FC80000223AB400B439BB2A3812823434303F1E0
:10FC900020011144EFF31286502585F3128803F1F9
:10FCA0000C051C331544134455F8047F17B10F603D
:10FCB000296804319D42F7D100230B60F3B283F32E
:10FCC0001188282303FB0020036A23B1A3899BB278
:10FCD00043F0010304E0A38923F001031B041B0C80
:10FCE000A381BDE8F88300BF48190020004827E63B
:10FCF0006C200020004823E6C02000200A4B4FF46F
:10FD000000525A604FF6FE730848D0F888201168F8
:10FD10000B401360826FC36F9A4201D0543072E679
:10FD2000012380F898307047000002406C200020CA
:10FD30002DE9F0431E469C4B8DB098428946904673
:10FD40009DF850705ED1994B994AC3F85C805A6512
:10FD500003F1A8029A6603F5D472DA664FF4807252
:10FD60001A665A66934AC3F8A400C3F88820A2F51D
:10FD70004842403AC3F89C208F4B9A6942F4804233
:10FD80009A615A6942F001025A6102238DF80330E8
:10FD90003A074FF40073ADF8003001D51C230FE093
:10FDA000B30706D51823854869468DF8023003F05D
:10FDB0005BF8F5070AD54FF48063ADF800304823AF
:10FDC0007E4869468DF8023003F04EF801240E2378
:10FDD000002501A88DF804308DF805408DF8074006
:10FDE0008DF8065005F028FA252301A88DF8054066
:10FDF0008DF807408DF804308DF80650704C05F0F2
:10FE00001BFA50E06F4B984240F0C980674B684A3C
:10FE1000C3F808801A6003F52A725A6103F56A7202
:10FE20009A614FF48072DA601A61674A18659A64C1
:10FE3000DA64614B3C07DA6942F48022DA619A693C
:10FE400042F008029A614FF002038DF803304FF43C
:10FE50008063ADF8003001D51C230FE0B00706D554
:10FE600018235A4869468DF8023002F0FDFFF10769
:10FE70000AD54FF40063ADF8003048235348694673
:10FE80008DF8023002F0F0FF27238DF804300022B5
:10FE9000012301A88DF805308DF806208DF8073074
:10FEA00005F0CAF9414C0025012384F8443025624D
:10FEB000E561A5626562C4F82C906671C4F808809B
:10FEC000A7712046FBF78EF9F20731D5206B002889
:10FED00026D0E36C039501934FF480530A9380235B
:10FEE0000693E368059504932023099363690795B6
:10FEF000029308950B9501F05BF801A9206B01F0C6
:10FF000039F8226B216D136843F0010313608B8A6B
:10FF10009BB243F040038B8253689BB2236407E09B
:10FF20004FF6DF72236D1A80DA6842F02002DA6041
:10FF3000B3072CD5606B28B3A36C002501934FF455
:10FF400080530A9380230693236902950493102318
:10FF5000039305950795089509950B9501F028F8E9
:10FF6000606B01A901F006F8636B1A6842F00202A7
:10FF70001A60226D5D605D60938A9BB243F08003DE
:10FF8000938204E0226DD36843F08003D360226D36
:10FF9000204693899BB243F40053938100E00020F4
:10FFA0000DB0BDE8F08300BF003801406C20002098
:10FFB000F0A3010844000240001002400008014084
:10FFC000C02000200048004004480040000C0140D0
:10FFD00038B500240B4D6059254403F049FF69688A
:10FFE00011B10948FCF789FFA96811B10748FCF76E
:10FFF00084FF0748103403F03BFFB4F5F07FE9D1EC
:020000040801F1
:1000000038BD00BF10A4010870C0010876C0010807
:10001000B7C7010870B50546284608F09EFD06469C
:1000200058B91A4B1A485A791A4BBDE8704003EB7D
:100030008203D3F8DC11FCF760BF2846164932462C
:1000400008F094FD60B9154803F012FF144C54F801
:10005000041F19B11348FCF750FFF8E7124805E0F8
:100060000024124B53F8241021B91148BDE8704008
:1000700003F0FEBE2846324608F078FD0134002821
:10008000EFD1024B0B4D5C71C6E700BFB40F0020EF
:100090007CC0010810A4010888C001088DC00108B7
:1000A000ECA50108A0C00108B7C70108F0A5010828
:1000B000C2BF0108B1BC0108F0B585B0044608F024
:1000C0004CFD082826D1621EE01D1F4912F8013F91
:1000D00009681944497801F00301022908BF203B4F
:1000E00082421370F1D1254604F1080715F8016B1F
:1000F0001648314608F023FD20B12846314608F065
:100100001EFD10B1FDF790FB1CE0BD42EED1204674
:1001100004F094FC0E4803F0ABFE00230D4A04A942
:100120001A4492F888210A440849595C0133082B83
:1001300002F80C1CF2D10023074801A98DF80C30FD
:10014000FCF7DBFE05B0F0BDF400002014D201087E
:10015000A4C00108B40F00205BC601081D4B1E4C53
:100160001D6880B52068FEF75BF82846FEF758F852
:10017000206841798B0704D4036841F002015B6970
:100180009847164B08221A612068FAF742FC90B192
:10019000124E08237361104B1868FAF737FC0746B4
:1001A000FEF73CFE08B1FEF7A1FA28463946FAF7F9
:1001B00033FC082333612846FAF72BFC0028E3D0F0
:1001C00028462668FAF722FC01463046FAF724FC56
:1001D000DAE700BFC828002014250020000C0140E9
:1001E0002DE9F047054608F0B8FC314E0446D6F834
:1001F000088090B92F4803F03BFE2F4B53F8241092
:1002000049B10123A34013EA080F02D02B48FCF7A1
:1002100074FE0134F1E72A4822E0284629492246A3
:1002200008F0A4FC58B9284803F022FE274C54F8E3
:10023000041F0029EFD02148FCF75FFEF7E72B7879
:100240004FF000092D2B03BF013504F1FF344FF0AF
:10025000010A4FF0000A184B53F8297027B91C48BF
:10026000BDE8F04703F004BE28463946224608F0B0
:100270007DFCC8B9012000FA09F0830501D51548B5
:10028000EEE7BAF1000F03D0FCF774FF124803E069
:1002900040EA0800B060114803F0EAFD3946BDE8C5
:1002A000F0470F48FCF729BE09F10109D3E700BF69
:1002B000B40F0020AAC0010858A60108A0C0010878
:1002C000B7C7010888C00108B4C0010854A60108D6
:1002D000C2BF0108C0C00108CEC00108D7C00108D4
:1002E0005AC6010810B5084803F0C2FD074B0024A8
:1002F0001C715C63064B1C70FAF73AFD03F05EFF5D
:10030000044B1C6010BD00BFDFC001081425002095
:10031000012E0020C828002070B5064600240B4B93
:10032000E518AA8816420AD0E1580948FCF7E5FD0D
:100330002846002103F02DFD064803F099FD40F604
:10034000584314349C42EAD170BD00BF28AB010869
:100350000BC10108B7C7010808B50848FCF7CDFD77
:10036000FFF79AFA02F06EFE18B96420FAF7A9F9BD
:10037000F8E70348BDE80840FCF7BFBD15C1010818
:1003800022C101082DE9FF410A4806888568448892
:10039000B0F80480C768FFF781F9CDF800800290BB
:1003A000019731462A4623460348FCF7A6FD04B0D0
:1003B000BDE8F081040000202AC10108F0B50478EE
:1003C0008BB005460CB1002436E04B4B19680E2368
:1003D00003FB0411B1F91D51B1F91921B1F91B3118
:1003E000009591F8205101F58C70019591F82151FB
:1003F00001F59071029590F90700039091F90210B0
:100400003E48049121460134FCF777FD082CDCD1ED
:1004100070E02D2B14D1072C1BDC284608F0F2FBD2
:100420000AAB661C03EB440424F8100C15F8013FDA
:10043000303B092BFAD934462B78002BE9D104E064
:10044000A3F13002092A09D8E5E7082CBDF81820E5
:1004500009D00BB0BDE8F040FDF7E6B9202BF8D18C
:1004600001352646E7E7072AF3D840F2DC55BDF808
:100470001A00214BA0F2EE2189B2A9421B68E8D8EC
:10048000BDF81C10A1F2EE24A4B2AC42E1D8BDF834
:100490001E6004B237B2A742DBDB0DB2AF42D8DC3C
:1004A000A542D6DBBDF8247007F16404A4B2C82CC1
:1004B000CFD8BDF826E00FFA8EF4112CC9DCBDF8B8
:1004C0002050B42DC5D8BDF82240B42CC1D812B2EA
:1004D0004FF00E0C0CFB0233A3F81901A3F81B110B
:1004E000A3F81D6183F8205183F8214183F81F711F
:1004F00083F822E10BB0F0BDE00E002087C10108B7
:10050000F0B504468FB0204608F027FBC5B21DBBEE
:10051000AE4803F0ADFCAE4C94F8D21009B9AD482A
:1005200053E049B294F8D02094F8D130009194F877
:10053000D310A948019194F9D4100734029194F989
:10054000CE10039194F8CF10049129460135FCF7A1
:10055000D4FC102DE0D1E2E72046A049052208F0A6
:1005600005FB0546B8B929469D48702208F0B1FA46
:1005700028469C4B19680E2303FB00130130002210
:10058000082883F8232183F8242183F8252183F880
:100590002621F0D118E120469349042208F0E6FA1A
:1005A00005462046002D4AD1202108F0C8FA00282F
:1005B00000F00A81461C304608F0CFFA2C46074668
:1005C0008A4B53F824502DB989480FB0BDE8F0404C
:1005D000FCF793BC30462946FAB208F0C7FA01345A
:1005E0000028EDD17A4A164602F17001002382F804
:1005F000D63082F8D23082F8D13082F8D03007324B
:100600008A42F3D17B4901EBC40191F8A0229342C5
:1006100010DAD1F8A472C3EBC302B0183A441768D9
:1006200000F1D001C0F8D0709088013388809279B1
:100630008A71E7E729467048FCF75FFC95E06F494F
:10064000072208F093FA05462046002D49D12021C3
:1006500008F075FA064608F080FAC4B26CBB684828
:10066000FCF74BFC214667480134FCF746FC0E2C96
:10067000F8D15848FCF741FC002463482146FCF7B8
:100680003CFC0025574A012311680E2202FB04128C
:10069000D2F82321AB4013425C4B5D495D4808BF53
:1006A00019460135FCF729FC0E2DEBD149480134E0
:1006B000FCF723FC082CE0D186E03046564908F0D0
:1006C000A5FA2C46002852D0022C55D008F09AFAF0
:1006D00006AB43F824005049002008F097FA013493
:1006E000F0E74D4908F092FA002460B1082C3ED0A2
:1006F00008F088FA06AB43F824004749002008F0C8
:1007000085FA0134F1E7082C31D1069B0F2B2ED846
:10071000DDF81CE0BEF1070F29D8089F0D2F26D861
:10072000099E06F16402C82A21D80A9DFF2D1ED811
:100730000B9864281BD80C99642918D8884216DABB
:100740000D9C032C13D8224AC3EBC303134483F834
:10075000D0E083F8D17083F8D26083F8D35083F867
:10076000D40083F8D51083F8D6402C4CCBE60FB0DC
:10077000BDE8F040FDF758B8069B072B20D8079935
:100780000D291DD80278722A0DD06E2A18D1154A6B
:100790000E20126800FB032301228A40D3F82311A4
:1007A00021EA020209E00F4A0E20126800FB03232F
:1007B00001228A40D3F823110A43C3F8232101E020
:1007C000FDF732F80D4C9EE60FB0F0BDAFC1010849
:1007D000B40F0020B7C70108DAC1010892BF0108B1
:1007E00084100020E00E0020BDBF0108F0A5010824
:1007F000C2BF010810A40108D1BF0108A7C10108A8
:100800007AC00108F6C1010873C60108CACA010806
:1008100010CA0108FBC10108FFC10108B1BC0108F1
:100820002DE9F743047805468CB9324D95F8A712A7
:10083000B5F8A42295F8A6322F480091214601343C
:10084000FCF75BFB102C05F10405EFD14EE008F03E
:10085000D9F90F28044636DC2846202108F06FF924
:10086000264EE4B2D6F83880451CA400002728465E
:1008700008F0C8F95FFA87F9B9F1010F83B208D01F
:10088000B9F1020F0BD0B3F5B47F24D2B26B13537E
:100890000AE0FF2B1FD8B36B2344987004E0FF2BB2
:1008A00019D8B36B2344D87028462C2108F047F997
:1008B000054608B1013502E0B9F1020F0BD101374D
:1008C000032FD4D112E00E4800210F2203B0BDE85F
:1008D000F043FCF726BF08EB04000021042208F0D7
:1008E000F8F803B0BDE8F043FCF79EBF03B0BDE8E5
:1008F000F08300BFB40F002001C2010814250020BE
:1009000050BF01082DE9F04FAC498BB0044608F008
:10091000E9F8AB49002820460CBF0125072508F05F
:10092000E1F8A8490028204608BF022508F0DAF8B7
:10093000002808BF0425E90740F1E780A24803F03A
:1009400097FA002003F09EF8A04CA14803F090FA1B
:10095000A04803F08DFA62799F4BA04803EB820315
:10096000D3F8DC11FCF7C9FA9D48FCF7C6FA264615
:100970000027D6F810800021404605F085FA20B106
:100980009848FCF7BAFA002669E039469648D6F846
:1009900014B0D6F818A0D6F81C90FCF7AEFA404672
:1009A000002105F07BFA10B1202003F059FA06A9C6
:1009B0004046FCF73DF901468C48FCF79EFA584644
:1009C000002105F06BFA10B1202003F049FA06A9C6
:1009D0005846FCF72DF901468448FCF78EFA50463C
:1009E000002105F05BFA10B1202003F039FA06A9C6
:1009F0005046FCF71DF901467C48FCF77EFA484654
:100A0000002105F04BFA10B1202003F029FA06A9C5
:100A10004846FCF70DF9013701467548FCF76DFAB9
:100A20000C2F06F11006A4D1AAE749B294F8D02001
:100A300094F8D130009194F8D3106E48019194F954
:100A4000D4100734029194F9CE10039194F8CF108A
:100A5000049131460136FCF750FA102E03D094F879
:100A6000D2100029E1D1644803F002FA574B634CDD
:100A70009F6854F8041F19B16148FCF73EFAF8E783
:100A80000E46604B53F826404CB10123B3403B4225
:100A900003D05D482146FCF730FA0136F1E75B48A8
:100AA00003F0E6F92146494B0AAA0B4493F8883132
:100AB0001344574A8A5C0131082903F8102CF2D1FB
:100AC000002306A953488DF82030FCF716FA524847
:100AD00003F0CEF95148FDF7D1F9514803F0C8F9B8
:100AE0004E48FCF7A7FE4F4803F0C2F94B48FFF70A
:100AF00097FE4D48FCF701FA4020FFF70DFC4B48EC
:100B000003F0B6F94548FDF75BFAAA0739D548481E
:100B100003F0AEF9474803F0ABF9404802F0F2FFAA
:100B2000454803F0A5F93D48FCF708FE434803F0AB
:100B30009FF93A48FDF7F4F84148FCF7DEF93748E9
:100B4000FCF784FF3F4803F093F93448FFF736FC85
:100B500000260E27774300243B4A0123D26BA34093
:100B60003A44D2F80A2013421ED101340E2CF3D19C
:100B70000136082EEDD12C48FCF7BFF98020FFF795
:100B8000CBFB6B0716D5314803F072F9304803F000
:100B90006FF9224802F090FF2348FCF7AEF94FF4BA
:100BA0008070FFF7B9FB05E0314622462948FCF783
:100BB000A4F9DAE70BB0BDE8F08F00BF15C2010859
:100BC00012CE01081CC2010822C20108B40F002085
:100BD00030C2010842C2010810A401084EC2010837
:100BE00059C2010866C2010873C2010879C0010830
:100BF0005BC601088BC201087BC2010854A601082C
:100C0000AAC2010858A60108B8C20108C5C2010855
:100C100014D20108D1C20108DAC20108B1BC01082E
:100C2000E9C20108F5C20108B7C7010803C30108FA
:100C300010C3010823C3010831C301083BC30108E5
:100C40004AC3010858C301081425002064C30108E1
:100C500075C3010887C3010810B5204A18B9136885
:100C600002221A8210BD1E481468002303802178D6
:100C7000024611F07F010DD1637A990644BF02212B
:100C8000017013F0400F037814BF43F0010323F009
:100C9000010314E0012920D002291DD1617901F05E
:100CA0000F039B0003F1804303F5B84311F0800F5D
:100CB0001B6806D003F03003102B07D101231370FB
:100CC00004E003F44053B3F5805FF6E7054B1B687F
:100CD0001B699847024810BD184610BD982A00208D
:100CE000582500200828002010B5064C18B92368A4
:100CF00001221A8210BD044B1B689B68984720682C
:100D00000C3010BD982A00200828002010B5064C91
:100D100018B9236801221A8210BD044B1B681B6896
:100D2000984720680A3010BD982A00200828002023
:100D3000084BDA68D10709D4DA68520708D4DB68AF
:100D400013F0100F14BF03200420704701207047D8
:100D5000022070470020024003788B4283BF034B80
:100D600003EB410148880020704700BF5825002050
:100D700070B50546F9F77EFC324CE369E061C31AB1
:100D8000B3F5FA5F236282BF002384F8243084F82D
:100D9000253094F824302BB9A12D02BF294A012116
:100DA00082F8251094F82510264A31B1D118EDB2F9
:100DB000013381F8265082F8243094F8245094F8B6
:100DC0004730AB423CD11F4B93F84830052B02D043
:100DD000062B03D02FE0002004F06CF994F82730A4
:100DE0001E2B28D100200246C1B26B1E99421ADA8E
:100DF000214491F826300821DBB283EA0206F60787
:100E000044BF83F01803C3F3460301F1FF3154BF1D
:100E10005B0843F0800311F0FF01C2F34702ECD1FD
:100E200001301A46E0E7234493F826309A4202D173
:100E3000032004F03FF9002384F8253084F824309F
:100E400070BD00BF582500202DE9F843324F3D68A2
:100E50002A8A2E7AB2B9042E14D1304C3048237825
:100E6000012B0BD12F4B19682F4B89B20B445B0020
:100E700019681A6030230380227048E01023038031
:100E8000072644E0AC8AAB69A24294BF042602263E
:100E9000944228BF14461FFA84F840469847214AD6
:100EA00004F1010E13684FEA6E0E9BB203F100537A
:100EB00003F540535B001B6800219BB203F1005314
:100EC00003F540535B00714500F1020009D010F8B2
:100ED000019C10F802CC4CEA092C23F821C0013106
:100EE000F1E71268104B92B213445B001A681C6061
:100EF0002B8A3022C8EB03032B826B8A9844084B61
:100F0000A5F812801A80094B4FF440521A803B68B2
:100F10001E72BDE8F88300BF982A0020032E00202F
:100F200002280020505C00400230002000280020F1
:100F30000E4B0F4A1B683E299BB203EBC0000244D4
:100F40004FEA420209D94B09C80604BF03F1FF3337
:100F50009BB29B0243F4004304E04B08C90748BF1F
:100F600001339B0211681360704700BF505C004062
:100F7000063000208A6810B50C6A036814430A69B9
:100F800023F4FF4314434A6923F0700314438A692E
:100F90001443CA6914434A6A14438A6A22431343B6
:100FA0000360CB6843600B6883604B68C36010BD0F
:100FB0004FF6FE7302681340036000230360436032
:100FC0008360C360284B984201D1284A27E0284B10
:100FD000984201D1254A2AE0264B984201D1234A62
:100FE0002DE0254B984201D1204A30E0234B984216
:100FF00001D11E4A33E0224B984204D11B4A536868
:1010000043F470032EE01F4B984204D1174A5368F3
:1010100043F0706326E01C4B984204D11B4A53688E
:1010200043F00F031EE01A4B984204D1174A53684D
:1010300043F0F00316E0174B984204D1134A53686B
:1010400043F470630EE0144B984204D10F4A536886
:1010500043F4704306E0114B984204D10B4A5368A5
:1010600043F47023536070470800024000000240C0
:101070001C00024030000240440002405800024080
:101080006C0002408000024008040240000402405C
:101090001C04024030040240440402405804024050
:1010A0001F4A10B5536803F00C03042B03D0082B20
:1010B00004D01C4B14E01C4B1B6811E053685168B2
:1010C000C3F38343C90303F1020301D4174906E0C4
:1010D000516811F4003F1449096818BF49084B438F
:1010E000036053681249C3F30313CC5C0368E34005
:1010F00043605468C4F302240C5D23FA04F4846052
:101100005468C4F3C2240C5DE340C3605268C2F368
:1011100081320A44127CB3FBF2F3036110BD00BFBD
:101120000010024000127A004000002000093D003B
:1011300040A8010810B50446FFF7FAFD012806D1C2
:101140001CB1FFF7F5FD013CF8E7052010BD002CB0
:1011500008BF052010BD0A88F0B54B888E88B1F80D
:1011600008E0CC88002A3AD1028C43F0010322F037
:1011700001021204120C0284058B078CADB225F01B
:10118000F30545EA0E1189B241EA06027A49BFB277
:10119000884212D001F5006188420ED0B0F1804F34
:1011A0000BD0A1F59831884207D001F580618842C3
:1011B00003D001F58061884202D127F0020701E0E7
:1011C00027F00A071F4302830784038B23F00C03D5
:1011D0001B041B0C0383038B9BB21C4344E0042AB7
:1011E00044D1028C22F010021204120C0284018BF2
:1011F000058C21F440721205120D42EA0E325E494E
:1012000092B242EA06228842ADB292B212D001F501
:10121000006188420ED0B0F1804F0BD0A1F598311B
:10122000884207D001F58061884203D001F58061D2
:10123000884207D125F0200141EA03139BB243F015
:10124000100304E025F0A00143F010030B430283D8
:101250000384038B23F440631B041B0C0383038B65
:101260009BB243EA0424A4B20483F0BD082A028C92
:101270003ED122F480721204120C0284828B3E4D05
:1012800092B222F0F307018C47EA0E1292B2A84202
:1012900089B242EA060212D005F50065A8420ED0D6
:1012A000B0F1804F0BD0A5F59835A84207D005F5D1
:1012B0008065A84203D005F58065A84207D121F4D6
:1012C000007141EA03239BB243F4807304E021F4EC
:1012D000206143F480730B4382830384838B23F068
:1012E0000C031B041B0C8383838B9BB21C4341E0C8
:1012F00022F480521204120C0284858B018C25F496
:1013000040752D052D0D45EA062545EA0E321A4D8C
:1013100089B2A84292B212D005F50065A8420ED05B
:10132000B0F1804F0BD0A5F59835A84207D005F550
:101330008065A84203D005F58065A84207D121F455
:10134000005141EA03339BB243F4805305E047F672
:10135000FF5543F480530D402B4382830384838BDA
:1013600023F440631B041B0C8383838B9BB243EAEF
:101370000424A4B28483F0BD002C0140CA78F0B5E7
:10138000D40648BF8C780D8802F00F0348BF234372
:1013900015F0FF0F1DD0016800240126A64006EAC3
:1013A0000507B74211D14FEA840E0F2606FA0EF652
:1013B00021EA0601282A03FA0EF641EA060101D1C4
:1013C000476102E0482A08BF07610134082CE4D1D4
:1013D0000160FF2D1FD94168002404F10807012690
:1013E000BE4006EA0507B74211D14FEA840E0F2628
:1013F00006FA0EF621EA0601282A03FA0EF641EA59
:10140000060101D1476102E0482A08BF07610134A3
:10141000082CE2D14160F0BD0F4B1A6842F0010286
:101420001A6059680D4A0A405A601A6822F084729C
:1014300022F480321A601A6822F480221A605A68F4
:1014400022F4FE025A604FF41F029A60044B4FF0E0
:1014500000629A60704700BF001002400000FFF871
:1014600000ED00E02DE9F843564C0368013AC4F85A
:101470004A3083880D46A4F84E30072A42D8DFE868
:1014800002F0040A101822292F35B4F84A300B80D4
:10149000B4F84C3013E0B4F84C300B80B4F84A3058
:1014A00005E0B4F84A305B420B80B4F84C305B4244
:1014B00005E0B4F84C305B420B80B4F84A306B80E6
:1014C000B4F84E301DE0B4F84A305B420B80B4F8FB
:1014D0004C3012E0B4F84C300B80B4F84A300CE0D9
:1014E000B4F84A300B80B4F84C3005E0B4F84C3016
:1014F0005B420B80B4F84A305B426B80B4F84E30EC
:101500005B42AB80304B1B79002B59D1B5F9000001
:1015100004F0D2FA8046B5F9020004F0CDFA07468D
:10152000B5F9040004F0C8FA216D0646404604F0FF
:1015300017FBE16D8146384604F012FB0146484630
:1015400004F006FAA16E8146304604F009FB01461C
:10155000484604F0FDF907F0C9FC616D288040465B
:1015600004F0FEFA216E8146384604F0F9FA01468D
:10157000484604F0EDF9E16E8146304604F0F0FA99
:101580000146484604F0E4F907F0B0FCA16D68801C
:10159000404604F0E5FA616E8046384604F0E0FA11
:1015A0000146404604F0D4F9216F0746304604F066
:1015B000D7FA0146384604F0CBF907F097FCA8802B
:1015C000BDE8F883582500204000002044F6FB7158
:1015D000084B1A68137803EB431300FB031350788E
:1015E000C0EB0030B3FBF0F39078B3FBF0F080B2C7
:1015F000704700BF9817002008B50A480A2290F8E3
:10160000753000EB4303B3F88410903089B220F8B2
:10161000041CF9F704FA80B2FFF7D8FF024B1880D8
:1016200008BD00BF582500209C1700202DE9F84F69
:101630004668D1F808A0D0F808904F680D68D0F837
:10164000008051463046144604F08AFA39468346F3
:10165000484604F085FA0146584604F077F92946D1
:101660002060484604F07CFA51468146404604F02A
:1016700077FA0146484604F069F939466060404609
:1016800004F06EFA29460746304604F069FA01462E
:10169000384604F05BF9A060BDE8F88F2DE9F04111
:1016A00006460D4640684968144604F051F9A96899
:1016B0008046B06804F04CF929680746306804F0A9
:1016C00047F9C4F804802060A760BDE8F0812DE9E7
:1016D000F04106460D4608467168144604F040FA8B
:1016E000B1688046284604F03BFA29460746306830
:1016F00004F036FAC4F804802060A760BDE8F081E9
:101700002DE9F04F87B00493834B81461B880392E9
:101710009D0737D540F2E632109B8048DC89B0F94E
:1017200000301B1B03F2F315954203D8002BB8BF02
:101730005B4201E04FF4FA73B0F9022040F2E63068
:10174000121B02F2F314844203D8002AB8BF52429B
:1017500001E04FF4FA729342B8BF13460522C3F575
:10176000FA7393FBF2F30A22643B534399F81C206B
:10177000D2105343642293FBF2F3134423EAE3733E
:10178000DBB200E06423C8460093CB1C0293002523
:10179000029B022D13F8010F614902934FEA450B9A
:1017A00007D1B1F9041000F11B0301FB03F463112D
:1017B00031E05C4B31F9152033F91530039903EB17
:1017C000420349428B4203DB03999942A8BF194661
:1017D000554B33F90B40049B091B33F915404E4B15
:1017E00021441E88F40712D400F11B035343B207AF
:1017F0004FEA23130FD599F8124064224C439DF908
:1018000000104C4394FBF2F203EB221303E099F82F
:10181000083059430B11454A042432F90B2098F83B
:10182000017092FBF4F41C1B414E6743AB5D022D2B
:1018300003FB07F701934FF0640397FBF3F74FEABD
:10184000E7170AD1384604F037F9311D1E22F36834
:10185000FBF728F904F04AFB0746354B98F80B6074
:10186000198A03F1140E01FB04F25EF82500D2126E
:1018700006FB02062F4AB6F5001FA8BF4FF400165C
:101880009642B8BF164603F1200252F8250042F8EE
:1018900025404FF6FF720909B2FBF1F1201A4843C7
:1018A00099F850404EF825604FEA850A761380116A
:1018B0006CB1059304F000F9059B224603F12C015D
:1018C00001EBC501DB68FBF7EDF804F00FFB98F8BE
:1018D0001530194A5843019BB919434318466423EC
:1018E00090FBF3F31B12194422F80B10013502F19F
:1018F00008014AF80170032D02F1140102F12002DF
:101900004AF801604AF8023008F101087FF440AF5C
:1019100007B0BDE8F08F00BF74180020602D0020D4
:10192000AC0F0020F82D0020FC0E0020C40E00207B
:10193000702600200000E0FFB4260020094B1A6842
:101940000E2303FB0020437AFF2B07D0064A1278B0
:101950009A4203D9054A32F8130000E0808800B2A9
:10196000704700BF50250020982B0020602D0020DC
:101970002DE9F04F11F0FD0599B001900391AF4CA6
:1019800006D0AF4B1B689A0700F1BF8000F02CBD5A
:10199000636FAC4898470028F3D0AA4894F8842095
:1019A0000146FFF75FFDA84B1B88002B00F08480E9
:1019B000D4F8883004F18C061B7804F1980802935F
:1019C000A14A4FEA450A1788B7F57A7F02BF00227D
:1019D0003260C8F810209B4A32F915003268024480
:1019E000326004F069F8D8F8101001F1010BBBF176
:1019F000010FC8F810B007D10022C8F80400C8F8D9
:101A00000000C8F808202BE0D8F800C00590614617
:101A1000CDF810C003F09AFF8146584604F04CF808
:101A20000146484604F050F9DDF810C00146604612
:101A300003F08EFF8346059AC8F804005946104605
:101A400003F084FF0146484604F08AF8D8F80810ED
:101A500003F07EFFC8F800B0C8F80C00C8F8080012
:101A60007849DFF8E8B10022012F2AF801202AF88E
:101A70000B20DFF8D4912AD1D8F81000012808DD16
:101A8000013804F019F80146D8F80C0004F01CF9EC
:101A900000E0002007F0BAFA029B7BB104901846E0
:101AA00004F00AF8049A0146104604F015FA28B129
:101AB0004FF47A73A9F80030002319E032684FF42C
:101AC0007A7102F5FA7292FBF1F22BF80A200135D5
:101AD000032D06F1040608F114087FF471AF012FFD
:101AE00002D13846F8F70EFFB9F80030013BE1E7C4
:101AF0005449564831F8132030F81300121A21F8CF
:101B000013200133032BF3D13BE7039B002B00F0A1
:101B10006B844A4C94F8DA70254647B1012F40F0A7
:101B20005A84D4F81C71D4F82061002420E1F8F71D
:101B3000A1FD0646C4F8DC00D4F8E400301A03F036
:101B4000B7FF434904F00CF8424BC4F8E0005B686F
:101B500004F1E800C4F8E460984704F1E8060028BE
:101B600000F0F9803C4B30461A783146FFF77AFC9A
:101B7000B4F8EE30002B42D03B46D4F8F000B5F874
:101B8000EE203649B2F5C87F04BF002241F8232079
:101B90004FEA830C36F913E051F80C20274F7244BA
:101BA00041F80C20002126F8131020F813100133FF
:101BB000032BE4D1B7F8EE30012B1BD1D7F8F4306A
:101BC0004FF4C87EC83393FBFEF20280D7F8F820AA
:101BD000C83292FBFEF24280D7F8FC30204AC8336C
:101BE00093FBFEF312889B1A8380019B1980598016
:101BF000FBF762FDB4F8EE30013BA4F8EE30194B70
:101C00001B685B0740F19380B4F800210B4B322A2C
:101C10002AD1D3F8F0201188A3F8021151889288B4
:101C2000A3F80411A3F80621019A1288A3F8082149
:101C3000019A5288A3F80A2118E000BF70260020FC
:101C4000AC170020C40E0020FC2D002044270020EB
:101C5000BD378635CC280020022E002064270020C6
:101C60001400002094170020002A3FD0D4F8F01070
:101C70000020B5F800314FEA800E322B394B04BFFB
:101C8000002243F8202036F910C053F80E20364FBA
:101C9000624443F80E20002326F8103021F810305B
:101CA000013003281A46E4D1B7F80031012B18D1CE
:101CB0000C2087F8182187F81931F8F723FED7F898
:101CC000F030B7F802211A80B7F804215A80B7F82B
:101CD00006219A80B7F80831019A1380B7F80A31C3
:101CE0005380B4F80031013BA4F8003194F81A3164
:101CF0001D4AE3B1D2F80C31322193FBF1F3D2F853
:101D0000F050002082F81A012B80D2F8103193FB9A
:101D1000F1F36B80D2F81431144A93FBF1F312887B
:101D20009B1AAB80019B18805880FBF7C5FCD4F848
:101D3000F020B4F8E83011885B1AA4F8E830518834
:101D4000B4F8EA305B1AA4F8EA309288B4F8EC30C0
:101D50009B1AA4F8EC3094F8DA30013384F8DA30C6
:101D6000D7E600BF7C27002070260020140000204A
:101D7000DFF8D8B20BF1E80232F81400AF4A0BF5E5
:101D8000927522F8140000B203F096FE394603F073
:101D9000E7FEAB4A45F8240032F9140003F08CFE4C
:101DA000314603F0DDFE0BF5987545F8240001344B
:101DB000032CDDD128462A460BF59E71FFF76EFCF9
:101DC00028460BF5A47106AAFFF768FC06A8024690
:101DD000DBF8E010FFF77BFC06984FF07C5103F036
:101DE000BFFE4FF07C510646079803F0B9FE4FF056
:101DF0007C510546089803F0B3FE31460446304650
:101E000003F0AEFE29460746284603F0A9FE014628
:101E1000384603F09DFD21460746204603F0A0FE0C
:101E20000146384603F094FD4FF07C5103F098FED4
:101E300001464FF07E5003F089FDDBF85891029087
:101E4000494603F08DFEDBF85C8103904146204655
:101E500003F086FE039A0146104603F079FDDBF895
:101E6000607103903946284603F07AFE039A0146D2
:101E7000104603F06BFDDBF854A103905146304649
:101E800003F06EFE039A0146104603F061FD4146E1
:101E90000590029803F064FE39460390304603F043
:101EA0005FFE039A0146104603F052FD514603902F
:101EB000284603F055FE039A0146104603F048FDFC
:101EC00049460390204603F04BFE039A0146104614
:101ED00003F03CFD49460490284603F041FE41468C
:101EE0000390304603F03CFE039A0146104603F08F
:101EF0002DFD39460390029803F032FE039A014605
:101F0000104603F025FD51460390204603F028FEBD
:101F1000039A0146104603F01BFD514603900298B8
:101F200003F01EFE49468246304603F019FE014684
:101F3000504603F00BFD41460646284603F010FECE
:101F40000146304603F002FD39460546204603F0BF
:101F500007FE0146284603F0F9FC059BDDF810C09A
:101F6000039A03F10041CBF85401CBF85CC109A8F6
:101F70000CF1004CCBF8602102F10042CBF8583153
:101F80000991CDF828C001460B920CAAFFF786FBF9
:101F90002C48DBF8541112AAFFF799FB0FAE09A8E1
:101FA000284915AAFFF742FB15A812A93246FFF7E8
:101FB00075FB0CA8314615AAFFF738FB32462148BD
:101FC00015A9FFF76BFB1198DBF8641103F084FF90
:101FD0001D4B1A7810B142F0080201E022F008020D
:101FE0001A4C1A70D4F8683104F5B8771B787BB3B3
:101FF000D4F86C913846494612AAFFF768FBD4F82A
:102000007C8104F59270414615AAFFF760FB12A887
:1020100015A93A46FFF742FB04F5C070494612AADB
:10202000FFF755FB3046414615AAFFF750FB12A8B3
:1020300015A904F5C072FFF731FB15E0A20F0020CF
:10204000C40E002054A80108B017002070260020FC
:1020500004F5927304F5C07593E8070087E807005C
:1020600096E8070085E80700D4F82401D4F8288111
:10207000014603F075FD41460546404603F070FDFC
:102080000146284603F064FCD4F82C710546394615
:10209000384603F065FD0146284603F059FC9A498D
:1020A000074603F019FF994E002520B93846984994
:1020B00003F0F4FE30B1C4F84851C4F84C51C4F8F0
:1020C000505112E006F5A47206F5B87006F5C0711D
:1020D000FFF7ACFAD6F8E0108E4803F0F5FD0146A4
:1020E00006F5A4700246FFF7F2FAB4F88C31874D7A
:1020F00001339BB2B3F57A7FA4F88C314ED1D5F879
:102100005401D5F85891014603F02AFD4946064688
:10211000484603F025FD0146304603F019FCD5F88A
:102120005C8106464146404603F01AFD01463046B2
:1021300003F00EFCD5F8607106463946384603F0C8
:102140000FFD0146304603F003FC06F05FFF014639
:102150004FF07E5003F0B8FDD5F85811064603F055
:10216000FFFCD5F85C118146304603F0F9FCD5F848
:1021700060118046304603F0F3FC31460746D5F83F
:10218000540103F0EDFC0023C5F85401C5F8589143
:10219000C5F85C81C5F86071A5F88C31D4F854811C
:1021A000D4F85C614046314603F0DAFCD4F858714B
:1021B000D4F8605139460446284603F0D1FC014664
:1021C000204603F0C3FB014603F0C2FB4FF07E51F3
:1021D000044603F081FE50B920464F4903F05EFEED
:1021E000E0B920464FF07E5103F076FE08B14FF083
:1021F0007E54204603F002FB06F0B4FE03F052FBCF
:102200000021044603F068FE48B14449204603F02B
:102210009DFB002103F060FE88B923E0404C04F1EF
:1022200000493E49484603F091FB0021824603F0F5
:1022300053FE90B12046002103F04EFE30B12046FF
:10224000364903F083FB4FF0010902E04FF001092A
:102250005046344903F022FE0FE02046002103F0EF
:102260003BFE08B1204600E048462C4903F06EFBD7
:102270002D494FF0010903F02FFE00B981465FFAA6
:1022800089F353B128464146FAF756FE014603F05A
:102290005FFB4FF0000A05467DE03946404603F0FB
:1022A0005FFC29468146304603F05AFC0146484609
:1022B00003F04EFB014603F04BFB314683463046AC
:1022C00003F04EFC81463946384603F049FC494646
:1022D00003F03EFB014603F03BFB01464FF07E500E
:1022E00003F034FB00218246584603F0CDFD20B1B7
:1022F0005046002103F0C8FDC0B951465846FAF7D0
:102300001BFE824614E000BFB81E8D3F70260020E1
:102310003D0A673F6F12833A000080BFDB0FC93F61
:10232000DB0FC9BF35FA0E3C35FA0EBC4FF0000A80
:102330002946404603F014FC31468046384603F0F7
:102340000FFC0146404603F003FB014603F000FB8F
:1023500029460646284603F003FC0146484603F09A
:10236000F7FA014603F0F4FA01464FF07E5003F00D
:10237000EDFA00210546304603F086FD20B12846DF
:10238000002103F081FD28B929463046FAF7D4FD33
:10239000054600E000251949504603F0E1FB06F030
:1023A000A5FD174E15493080204603F0D9FB06F0F5
:1023B0009DFD1449708005F1004003F0D1FB03F04E
:1023C00095FD80B2104B10F4004F18BF00F5B470AB
:1023D0001880002300E001230C4A002182F8DA1063
:1023E000002B7FF496AB06E00023A4F8E830A4F8B5
:1023F000EA30A4F8EC3019B0BDE8F08F4D3D0F4441
:10240000FC0E0020E12E6542A80F0020702600205F
:1024100001380A4B042804D8DFE800F00507090B4F
:102420000D00074A08E0074A06E0074A04E0074AA9
:1024300002E0074A00E0074A1A607047E400002003
:102440000DC3000801170108B1C5000849C0000804
:1024500045BD000801B80008704708B50B4B0020C7
:1024600093F82C10FEF764FD094B1B68187A0828B6
:1024700001BF084B4FF480521A80102208BF5A80C7
:10248000A0F109035842584108BD00BFB000002028
:10249000982A002000280020704770477047FEE708
:1024A000FEE7FEE7704730B50024E3B293420DD259
:1024B000030F092B94BF3033373301F81430002554
:1024C00001EB440300015D700134EEE730BD30B52F
:1024D000002240F60F7102F1805303F5B8539B00C0
:1024E0001D6842F4004444F0800429400132214335
:1024F000042A1960EDD1024B40F08000186030BD15
:102500004C5C00402DE9F347884D894C2B68894E7F
:102510009BB2A380A28831880A40970507D54FF661
:10252000FF53854A2B6013780133DBB21370A38805
:102530000B40180440F100830023ADF802302B68F3
:102540007B4F9AB21804A28040F1F682BB8803F058
:102550000F03BB71002B40F0C182784A13689BB215
:102560003B803B8803F030037B803B8803F440537F
:102570003B804BF6BF7311680B4083F4005383F02C
:10258000200343F4004343F080031360BB88D90663
:1025900021D448F60F7311680B40694913600B682A
:1025A00088461A7A022A01D0042A02D1FEF74CFC8E
:1025B00059E2062A40F06B825A78052A08D11A7827
:1025C000520605D1D878FFF782FFBB681B6A98478F
:1025D000E3689B685AE213689BB2ADF80230BDF81D
:1025E00002301F0540F1CF8140F68F731168544FC0
:1025F0000B40544913600A68534B92B213445B007A
:102600001A683B688846187A092817D092B2520097
:1026100002F1804202F5C042117819705178597068
:102620009188C8B2090A41EA002159801189C8B2CB
:10263000090A41EA002199809289DA8001221A72FE
:10264000DA8893F80190002A40F0DC801A7812F0C2
:102650007F024AD1B9F1090F0FD1DA78012A00F2CD
:10266000B8809978002940F0B4809988002940F01A
:10267000B0809A72A3685B68A9E0B9F1050F10D128
:1026800093F90320002A01DA0823B9E09A78002A96
:10269000FAD19A88002AF7D19B7A002B00F0A28009
:1026A000F2E7B9F1030F0ED1DA78012A40F09180F8
:1026B0009A88002A40F08D805A7A42F020025A729D
:1026C000A368DB6983E0B9F1010F40F08280DA781A
:1026D000012A7ED19A88002A7BD15B7A980678D528
:1026E00006F04AF900287DD073E0012A2ED1B9F115
:1026F0000B0F6ED1E26858799269D97890473B68A0
:102700009A7A002A65D0002863D11A79002A60D10C
:102710009B78002B5DD1064B9B68DB689847084B84
:102720001B685A79DA72DA781A735BE0445C00400D
:1027300000280020D42B0020042E0020005C004044
:10274000982A0020505C004004300020022A40D12A
:10275000B9F1010FC4D0B9F1030F3AD1587920F083
:10276000800E4FEA8E0202F1804101F5B8410968FE
:1027700010F0800F14BF01F0300101F44051BEF1A0
:10278000030F26D8B3F802E0BEF1000F21D101B348
:102790009B7AF3B102F1804202F5B8421368010658
:1027A0004BBF23F4E04323F4804323F0400323F0A2
:1027B00070034BBF9BB29BB283F0100383F4805332
:1027C00043F4004343F080031360A3689B69984778
:1027D00008E0E36848465B69984703280FD0002863
:1027E0007FF452AFD8F80020A14B92B213445B00A3
:1027F0001A6800221A6030236380062300E0092350
:102800003A6847E1B9F1060F12D11A78520677D12A
:102810009B78012B02D1E368DB6966E0022B02D1D1
:10282000E3681B6A61E0032B6AD1E3685B6A5CE0E2
:10283000B9F1000F37D15988002961D15A6822F4C3
:102840007F42B2F5003F5BD11A7812F07F0204D1CB
:102850009B88002B00F0D58152E0012A08D1E26864
:1028600058799269904700284AD13B689B7A16E0D4
:10287000022A45D15A7902F00F018B0003F18043FF
:1028800003F5B8431B6812F0800F14BF03F0300348
:1028900003F44053032933D812F0700F30D1002BCA
:1028A00040F0AF812CE0B9F1080F04D11B785B0632
:1028B00000F0A98124E0B9F10A0F21D11A7802F0C1
:1028C0007F02012A1CD19A7AD2B15988C1B95A68BB
:1028D00022F47F42B2F5803F12D1E26858799269C2
:1028E0009047002800F091810AE04BB13A684FF020
:1028F0000008A2F8128093614046984740460BE0DA
:10290000E3683A681B6950789847032804D1594B0B
:1029100009221B681A72BEE04FF6FF713A68138AEB
:102920008B4201D10923B5E0022800D00BB908235E
:10293000B0E092F9001000291FDAD18801910198C6
:10294000834202D9019B138210E08B420ED2E168D0
:1029500091F82C00834201D2002105E093FBF0F1B5
:1029600000FB113313B90121434B1970E36893F84D
:102970002C309382FEF768FA8DE0032313724FF434
:102980004053238087E0BDF802301BB2002BBFF616
:10299000D6AD40F68F7311680B401360354A176847
:1029A00090463B7A022B72D0042B70D0032B01D0BF
:1029B000052B67D1BB693A8A8BB9398A00293BD08C
:1029C0004FF4405323802D4B1A68294B92B2134485
:1029D0005B001A6800221A60302363802CE0002A12
:1029E000EBD0B7F81490914528BF91461FFA89FAA9
:1029F000504698473B8A4FF0000ECAEB03033B82D8
:102A00007B8A53447B821D4B1A681D4B92B2134440
:102A10005B001B6809F101029BB203F1005303F54F
:102A2000405352105B009645C7D053F82E1020F843
:102A30001E100EF1010EF6E7BB8A8B42D8F800306B
:102A400001D8032201E011B105221A720BE006221F
:102A50001A720A4B1A68064B92B213445B001A684A
:102A6000196030236380D8F800301B7A10E000BF73
:102A700002300020982A0020032E0020505C0040E5
:102A800004300020072B02D1E368DB689847082355
:102A9000D8F800201372FFF7E0FC5E4B1A684BF683
:102AA000BF7313402288D704228848BF83F4805321
:102AB0009004628848BF83F40053D106628848BFFF
:102AC00083F01003920648BF83F0200343F40043D1
:102AD00043F080034F4A9BB213602DE09A0002F14D
:102AE000804202F5B842116889B2ADF80210BDF813
:102AF000021009B2002909DA40F68F711068013B13
:102B000001401160444A52F823309847BDF8023022
:102B10001F067FF514AD48F60F72A1798B0003F103
:102B2000804303F5B843186802401A603A4B03EB40
:102B300081039B69984702E5A288338813405905B1
:102B400005D54FF6FF332B60344B5B689847A2885E
:102B500031880A40920444BF4DF6FF732B60A3886E
:102B60002F4A0B40DB0452D54EF6FF732B60002337
:102B70001374137C052B41D8DFE803F0030D141800
:102B8000222D6369264D1BB902F002F8062300E0EE
:102B900005232B743BE001F0FBFF04232374012386
:102BA000636134E002236374032328E0637C013B08
:102BB000DBB26374637C53BB194B04221A7426E0A6
:102BC000184A13689BB243F0100313600523237463
:102BD0000A2363741BE0637C114A013BDBB263741C
:102BE000637C03F0FF0093B94FF6EF730D490C6857
:102BF00023400B6006231374506108E006232374FE
:102C000005E0094B72E6094B70E6094B6EE602B02F
:102C1000BDE8F087005C004060A80108B00000201B
:102C200000280020405C0040590C01080D0D0108EF
:102C3000E90C010837B50446062103206A4602F074
:102C400089FB70B39DF801309DF80000164D43EAF2
:102C5000002000B202F030FF296802F081FF03F08B
:102C600045F99DF8033020809DF8020043EA0020DA
:102C700000B202F021FFA96802F072FF03F036F9FA
:102C80009DF80530A0809DF8040043EA002000B2C2
:102C900002F012FF696802F063FF03F027F9608019
:102CA000012003B030BD00BF480000202DE9F047EF
:102CB000664D2B686649581C0A788E4602F0FF065E
:102CC0000AB10346F6E737462B60687BAB6895F898
:102CD0000C80AA7B39B2202900F09C80DFF880C1EB
:102CE0000CEB8103DC789B783CF82110C3F1FF03E7
:102CF0009BB2002B65D04FF03C0CB1FBFCF9C3F14B
:102D0000FF0363431B12B9F1050F5DD8DFE809F03B
:102D1000030B1A293A4AE01A4143B1FBFCF0DAB23C
:102D20001044C0B251E0B1FBFCF00CFB101189B2B1
:102D3000DAB2C1F13C01E31A4B43B3FBFCFC204681
:102D400094442CE0B1FBFCF00CFB1011E21A89B2A8
:102D50004A43B2FBFCF25FFA83F84244D2B2204607
:102D600032E0B1FBFCF90CFB191189B2E01AC1F198
:102D70003C014843B0FBFCF05FFA83F84044C0B22A
:102D8000224621E0B1FBFCF80CFB1811D8B289B245
:102D9000E31A01FB03F2B2FBFCFC224684445FFA17
:102DA0008CF412E0B1FBFCF80CFB181189B2D8B21C
:102DB000C1F13C01E31A4B43B3FBFCF20244D2B233
:102DC00003E02246204600E044464FEA042C4CEA49
:102DD000004C4CEA020C17234FF0010808FA03F8E4
:102DE00006F1170118EA0C0FA1EB0301DFF874805C
:102DF00014BF4FF011094FF0090989B213F1FF33E5
:102E000008F80190E8D218360137B6B2BFB2114BBC
:102E1000A0465FE7AB6001238EF8003040F22A3312
:102E2000AA730D4AE9800D4985F80C806873AE805D
:102E3000536000238B840B889BB243F001030B800B
:102E4000136843F001031360BDE8F08718280020E1
:102E5000FF2D0020242800206C00024000040040C8
:102E60003A0C002005030020F0B5B1F800E0002383
:102E70004EFA03F2D50725D58E784FEAD30CF40627
:102E800048BFCC7806F00F0203F0070748BF224383
:102E9000BF0050F82C500F24BC4025EA0404BA406F
:102EA0002243282E40F82C2005D1C46801229A40E4
:102EB00024EA020205E0482E04D1C46801229A40A7
:102EC0002243C2600133102BD2D1F0BD2DE9FF4166
:102ED000574B1B689BB11A681AB15649886902435F
:102EE0008A619A889868ADF8042002228DF807203C
:102EF00004220DEB02018DF80620FFF7B5FF32200A
:102F0000F7F7DFFB1121002002F0E4F96021012036
:102F100002F0E0F96420F7F7D4FB002402A8FFF7E1
:102F200089FE274626460A250121022002F0D2F911
:102F30003220F7F7C6FB02A8FFF77CFEBDF9082098
:102F4000BDF90A1014448A42A8BF0A46BDF90C30E4
:102F50000F4493421E44A8BF134613F5805F04DD5F
:102F6000013DE1D14FF0010801E04FF000080020E1
:102F7000122102F0AFF90A250121022002F0AAF97C
:102F80003220F7F79EFB02A8FFF754FEBDF9082098
:102F9000BDF90A10A41A8A42A8BF0A46BDF90C302E
:102FA0007F1A9342A6EB0306A8BF134613F5805F72
:102FB00002DD013DE0D101E04FF00008204602F0C3
:102FC0007BFD01461C4802F07FFE1C4D20F00040B6
:102FD0002860384602F070FD0146174802F074FE82
:102FE00020F000406860304602F066FD014614485B
:102FF00002F06AFE20F00040A8607021002002F07C
:1030000069F92021012002F065F90220002102F077
:1030100061F96420F7F755FBB8F1000F04D14FF0C8
:103020007E532B606B60AB6004B0BDE8F08100BFE5
:10303000E00200200010024000406F4648000020DF
:1030400001C05E46104B73B518781C46A0B105232D
:103050000E4D8DF800304FF4805600238DF801306E
:103060000B486E6101A96A460223F5F77BFD2E61CC
:103070009DF8050000F0010000F00100207080F0D4
:10308000010002B070BD00BF51060020000C0140DD
:1030900000380040064B70B506461C461D68FFF719
:1030A000D1FF18B923685B1BB342F8D970BD00BFCC
:1030B000980F0020F7B503238DF80430030C8DF82A
:1030C00005308DF80700030A06200F4614468DF8D8
:1030D0000630FFF7DFFF88B1094D4FF4805600211D
:1030E00001AA04236E610748F5F73CFD05483946FF
:1030F00000222346F5F736FD20462E6103B0F0BDD1
:10310000000C014000380040012828BF01202DE9B3
:10311000F04F06464FF0140E0EFB00F36F4FDFF832
:10312000D881F918F8586E4B0A69DE736D4BC8F8F0
:103130000000DC690D892243DA618288B1F80AA0B7
:1031400022F440724C68120489B0120C4AEA050954
:10315000828003A9C4F81090022220460193ADF8A2
:103160000C908DF80F208DF80EE0FFF77DFE019B8F
:1031700000971F464FF0080BA268154203D10A20A2
:10318000F7F794FAF8E70A206561F7F78FFA2561F7
:103190000A20F7F78BFABBF1010BEDD1C4F814A0AC
:1031A0000A20F7F783FA65610A20F7F77FFA2561AD
:1031B0000A20F7F77BFA0222C4F810A0204603A9E0
:1031C0008DF80F201C228DF80E20ADF80C90FFF723
:1031D0004BFED8F80040444A03A894423A690BBF1A
:1031E00042F4001242F480023A613A610BBF3A693C
:1031F0003A6922F4001222F480023A61A38823F48F
:1032000040731B041B0CA38023889BB243F0010373
:103210002380A588FDF744FF0599344B25F03F0531
:10322000B1FBF3F32D042D0C1D43ADB2A580228814
:10323000002522F001021204120C22802C4A03A85D
:10324000B1FBF2F100298AB208BF012242F4004129
:103250004FF4967253434FF47A7293FBF2F30133B7
:103260009BB22384A1832388009A9BB243F001037D
:103270002380238823F4816323F002031B041B0CA7
:1032800023804FF480432381142303FB0626737BA2
:1032900001248DF80C308DF80D508DF80E508DF8FE
:1032A0000F4001F0C9FF337B9DF80F208DF80C30E3
:1032B0008DF80D508DF80E501AB103A801F0BCFF27
:1032C00008E05A0903F01F039C4002F12003094A59
:1032D00042F8234009B0BDE8F08F00BF9CA8010868
:1032E00018280020001002400054004040420F0007
:1032F00080EE360000E100E0C82D00200846F6F719
:10330000E7BB0E4B1A786C2A15D15A88B2F5FC6FC0
:1033100011D11A79BE2A0ED193F8DC270020EF2AAA
:103320000BD113F8012B5040054A9342F9D1B0FA62
:1033300080F04009704700207047704700F801088E
:10334000E0FF01082DE9F04FE84C00214FF4FC624A
:1033500085B0204605F0BDFBE54B04F539721A60D7
:10336000E44B00221A70E44B04F2AE7119606C2336
:103370002370032363714FF48073A3604FF41673BB
:10338000A4F86431FA23A4F866314FF4FA73A4F870
:103390006C31012384F85E3184F8693184F86A3134
:1033A00084F87C3184F88431052384F8233240F298
:1033B000DC53A4F8963140F24C43A4F8983140F223
:1033C0006C73A4F89A3140F27533A4F89C3140F63E
:1033D0004303A4F89E312346202184F868116E210E
:1033E00084F87A110A2184F87B112B2184F87D114D
:1033F000212184F87E11232184F87F114FF4C871B4
:10340000A4F88011032ACCBF0121002102F101029E
:1034100083F8A01114BF1E210521122A83F8A111DF
:1034200003F10203EED140F27E41A4F8401140F2D4
:103430003A71A4F8421140F27E51A4F8481140F2CA
:10344000EA5140F2DC5CA4F84A1140F2B4514FF466
:10345000FA63A4F8C631A4F8CA31A4F8CE31A4F8AE
:10346000D231052384F8E031C82301264FF47A785D
:103470004FF0320BA4F8E431DFF874924FF4C873C4
:103480004FF01E0A1922A4F8E831A4F846C1A4F8A6
:103490004C11A4F8C481A4F8C881A4F8CC81A4F884
:1034A000D08184F8E26184F8E36184F8E661A4F8ED
:1034B0004481A4F84EB184F893A184F8E1210192EB
:1034C000CDF80CC0A4F8503184F8DF6184F8EC61C9
:1034D000A4F852B184F8EF6101F084FAD9F8003011
:1034E0000025019A55212573D9700F215971DA7180
:1034F0002221212299715A740E2153222D201974F0
:10350000DA7635215A222827587399761A720A21B9
:10351000642218754FF0780E4FF4FA7083F80BA000
:1035200083F80CA0997402911A7783F80AE01D7051
:103530005F705F759F709F75DD7583F804B09D7334
:103540001D76DD735D765F729E77A3F84E006B4843
:10355000DFF8CCE19863D8636948C3F82CE0C3F87E
:1035600030E09862DFF8BCE16648C3F848E0586391
:103570004FF07F5A64484FF04B0EC3F820A0C3F8B9
:1035800024A083F84CE0DDF80CC04FF0460E4FF05D
:10359000000A586483F85070C3F840A084F8AFE77D
:1035A0004FF0140E84F8AE2784F8B6E7A4F8B8C735
:1035B00084F8B0B784F8B15784F8B55784F8B25797
:1035C00084F8B35784F8B4571866152083F8680058
:1035D0004E484FF0040E0192A3F85850A3F85A50E9
:1035E000A3F8565083F85CE083F8647083F8657044
:1035F000D866474883F87860186746485867464851
:1036000001F01CFAD9F800304FF44870A3F8160105
:103610001846C82283F8115183F8125183F81371A8
:1036200083F8146183F81851029984F8D721019A1C
:1036300084F8D611A4F8D88184F8DA51A4F8DC21F2
:103640000E2202FB05326FF0170482F819410324A1
:1036500082F81A416FF02F0482F81B41072482F888
:103660001C416FF0230482F81D41052482F81E419D
:1036700001355A2480F8204180F821416422FF243A
:10368000082D80F81F2180F822414FF0000100F141
:103690000E00D5D1C820A3F88A01142083F88C012C
:1036A000A3F890211E204FF4967283F88D01A3F8A1
:1036B00092210120282283F8891183F88E01A3F832
:1036C00094210B46094D5A191033C02BC2F810A093
:1036D000F8D105F529700021402205F0FAF9002300
:1036E0000E4EEA189959043308681DE0B40F002003
:1036F000E00E0020AC280020040F00208FC2F53C13
:10370000000060406666663F0000A0409A99193F3D
:10371000F6287C3F3D0A773FD2C50108C4A80108BE
:10372000CDCCCC3E00004040382B234CC2F8A40244
:10373000D6D104F509700021802205F0CAF906F1FE
:103740003801702204F5097005F0B8F9FAF774FF32
:10375000D9F8006000230125314604F27C404FF483
:10376000CC7284F8D43784F8D25784F8D35705F054
:10377000A5F904F2146031464FF4CC7205F09EF9BD
:103780000E4B1B681A68C4F8BA275A68C4F8BE27DB
:103790009A68C4F8C2271A68C4F8C6275A68C4F8D9
:1037A000CA279A680223C4F8CE2784F8D05484F834
:1037B000683605B0BDE8F08FB40F0020040F00207C
:1037C000074B93F8D437012B08D1064A064BD06833
:1037D0001B68834234BF00200120704700207047DF
:1037E000B40F0020040000205406002038B5094B17
:1037F00093F8D45765B9084C2068FAF71CFD074BBD
:1038000025601B78022B03D1BDE8384001F0A9B830
:1038100038BD00BFB40F0020F4280020F02800209D
:10382000064B93F8D4371BB1012B05D1FCF712B826
:10383000034B1868F7F7E4B800207047B40F002076
:10384000F4280020F8B5011F06460023083051F87F
:10385000042F02F120043F2C3BD802F108040F2C66
:1038600006D80232032A04D9002B08BF012300E046
:1038700002238142EBD1012B30680ED0022B1AD0EB
:10388000736800F0030003F003039B0043EA001099
:10389000B36803F00303184317E000F00F0040F093
:1038A0004000F6F715F9B068736800F00F0040EAC1
:1038B0000310C0B209E000F03F0040F08000F6F7CE
:1038C00007F93079F6F704F9307ABDE8F840F6F7F1
:1038D000FFB806F10C0734463A46002552F8043D7D
:1038E000AD0003F18001FF2910D903F50041B1F5C6
:1038F000803F02D245F0010508E003F50003B3F173
:10390000807F34BF45F0020545F00305B242E5D1A2
:1039100065F03F00C0B2F6F7DBF805F00303022BB9
:10392000207807D0032B0CD0012B13D1F6F7D0F859
:1039300060780FE0F6F7CCF86078F6F7C9F8A07871
:1039400008E0F6F7C5F86078F6F7C2F8A078F6F761
:10395000BFF8E0780434F6F7BBF8BC424FEAA5059F
:10396000DBD1F8BD10B504467F2C06D964F07F008A
:10397000C0B2F6F7ADF8E409F6E7E0B2BDE81040F2
:10398000F6F7A6B8430083EAE070EBE72DE9F047CD
:10399000304B86B093F8D4370746012B01D004464C
:1039A0004AE005F0DAF80546064603A96846FBF743
:1039B00059FE039B049A029713442B443F2B059511
:1039C00019D90023684603A90322FBF777FE039B5E
:1039D0003BB9049B2BB9204A13705370059BABB3C2
:1039E00001E0FBF727FE039B049A059E1344334432
:1039F0007F2B2BD8029FDFF860903946CA461AF811
:103A0000024BC4F18008B04528BFB0460AEB040061
:103A10004444E4B2424605F051F8802C89F8004055
:103A200014D1C8EB0606504607EB0801324605F0F4
:103A300045F889F8006009E0254614F8011B21B11A
:103A4000064B1868F6F7E8FFF6E7ED1B284606B0C8
:103A5000BDE8F087B40F002028280020F4280020BB
:103A60000FB407B504AB53F8042B054900200193AC
:103A7000F9F758F903B05DF804EB04B0704700BFE4
:103A8000FD32010807B5064B06490093064B074A6D
:103A900001930748074BF9F730FA03B05DF804FBD0
:103AA000C0B90108FEC5010895B9010803C601089F
:103AB000DBC50108B4B9010808B5037833B90C4B6C
:103AC0000C481978BDE80840F9F717BA05F09AF8DC
:103AD00002280CD8064B0C221870074B02FB003052
:103AE000064B06301860F9F71DFC0548E5E708BDF0
:103AF000AC2800200AC601085C170020040F002033
:103B0000B1BC010808B503783BB90B4B0B4893F8DF
:103B1000AC17BDE80840F9F7F0B905F073F80228D2
:103B200008D8054B83F8AC07F9F756FBF9F71EFCEC
:103B30000348E8E708BD00BFB40F00200EC6010827
:103B4000B1BC010838B5037803BB214B1B680133B6
:103B50000F2B07D81F490C2202FB031295681C4645
:103B60002DBB00E01C4601340F2C01DD002400E0D9
:103B700005D818490C2202FB04129568BDB99C4275
:103B8000F1D11548BDE83840F9F7B7B905F03AF872
:103B90000F28044605D80F4A0C2303FB00239D6819
:103BA0002DB92146BDE838400C48F9F7A6B9084BB5
:103BB0001C60F6F78FFE21462A460948F9F79DF961
:103BC0000C235C43034B185DBDE83840F6F79ABE02
:103BD0005400002088A901081BC6010831C601084D
:103BE00049C6010873B5037813B9F9F71DFE3DE026
:103BF0001F4901AA05F067F800240146264625461C
:103C000099B134B1012C08D1084604F0FBFF0646F7
:103C100003E0084604F0F6FF05461549002001AA16
:103C200005F051F801340146EAE70B2D02D911489D
:103C30000C220BE0022C10D1A6F57A73B3F57A7F33
:103C400007D90D484FF47A714FF4FA62F9F769FD1C
:103C50000CE00A4B03EB45035E80084B084803EB7E
:103C600045032946B3F90220F9F747F902B070BDC0
:103C7000FFC1010850BF010853CD0108AC28002046
:103C800060C6010838B50D4C05462368834206D14D
:103C9000FAF7D1FA204600214C2204F01AFFE36C17
:103CA000AB4209D12846FAF7C6FABDE838400448C5
:103CB00000214C2204F00DBF38BD00BFFC2A0020BB
:103CC000482B0020034B1A68D379591C1344D17137
:103CD000187A70475418002010B5FFF7F3FF84B22C
:103CE000FFF7F0FF04EB002080B210BD10B5FFF726
:103CF000F3FF0446FFF7F0FF04EB004010BD10B5E2
:103D00000446054B21461868F6F786FE034B1B68F0
:103D100098796040987110BD581800205418002000
:103D2000014B1B689879EAE75418002038B504461F
:103D30000D462420FFF7E3FF4D20FFF7E0FF002CA6
:103D4000084C14BF21203E20FFF7D9FF2368002232
:103D500028469A71FFF7D3FF236893F84900BDE81E
:103D60003840CCE75418002001460020DEE710B5AB
:103D70000446C0B2FFF7C3FF200ABDE81040BEE70B
:103D800010B5044680B2FFF7F2FF200CBDE81040EA
:103D9000EDE737B582888368044610060D4641BFBB
:103DA00029494FF4CC7091F8AC1700FB0133D105D1
:103DB00042BF26490C20097802F03F0248BF00FBB1
:103DC0000133042A12D006D8012A0DD0022A2FD19D
:103DD00093F900102DE0102A0AD0202A0AD0082AD0
:103DE00026D1B3F9001024E0197822E0198820E0E8
:103DF00019681EE069461868F8F71AFF014614486A
:103E0000F9F77BF8F5B1E06801F056FE6946F8F77E
:103E10000FFF01460F48F9F770F8206901F04CFEDA
:103E20006946F8F705FF01460A48F9F766F809E020
:103E300000210948F9F761F825B10848E1682269CD
:103E4000F9F75BF803B030BDB40F0020AC280020B8
:103E500079C0010872C0010873C601086FC6010865
:103E6000024B0146D869F6F7D7BD00BFAC28002049
:103E700010B5441E14F8011F21B1034BD869F6F7A1
:103E8000CBFDF7E710BD00BFAC28002010B50378CC
:103E90001BB9BDE810400948EAE704F0B3FE044648
:103EA000062899BF2146064806480621F9F725F855
:103EB000601EC0B2BDE81040FAF72AB976C6010804
:103EC000BDC60108E9C60108F7B52A492A4B08789A
:103ED0002A4D1C682A4B05EB80001A88D0F8C010C8
:103EE000284B29481B7800914FF47A71B4FBF1F10B
:103EF000F9F703F8254B26481968264B0026B1FB35
:103F0000F3F1F8F7FAFF244B1F68F3B205EB8302D5
:103F1000D2F8D010E9B101249C403C4217D02207CE
:103F200015D01E4A0B20D25C00FB0323134A1C4809
:103F300002EB8303D3F8F020F8F7DFFF022C06D161
:103F4000184B93F8281011B11748F8F7D6FF01362F
:103F5000DBE71648FFF78CFF154B16481A88164BFF
:103F600092B219884FF4FC6303B0BDE8F040F8F753
:103F7000C4BF00BFFC170020980F002088A90108CB
:103F80009C170020E000002014C70108EC0000206E
:103F900057C7010840420F00AC170020E80000207E
:103FA00067C70108AC2800206FC70108B7C7010820
:103FB000A20E002073C70108A00E00202DE9F041D9
:103FC0000024804625460F4E4146A759384604F046
:103FD00001FE58B139460C48F8F78FFF301900211F
:103FE000FFF7D7FE0948FFF743FF013540F6584376
:103FF00014349C42E7D11DB9BDE8F041044837E7CD
:10400000BDE8F08128AB01080FC10108B7C701085E
:10401000C2BF01082DE9F74F824604F09EFD054618
:1040200028B1012819D19AF800302A2B15D1594806
:10403000FFF71EFF0024584E5848A159F8F75DFFBE
:1040400030192946FFF7A5FE5548FFF711FF40F646
:10405000584314349C42EED198E050463D2104F080
:104060006EFD002800F08D8003461D4613F8012DDB
:10407000202AFAD0441C204604F0C4FD8146204684
:10408000F8F740FD0746CAEB05054FF0000B142476
:1040900004FB0BF4DFF8208108F5D073E658019398
:1040A000304604F05AFD8446314662465046CDF80B
:1040B00000C004F05BFDDDF800C0019B002856D174
:1040C000EAB2624553D11D194444D4F8AC0101F061
:1040D000F3FC0146384601F0F5FE002845D0D4F83F
:1040E000B00101F0E9FC0146384601F0E1FE00288C
:1040F0003BD0B4F8A4319A0658BF4F46142202FBB5
:104100000B881C0648BF2748D8F8A82142BF90F862
:10411000AC074FF4CC7404FB0022D80542BF224800
:104120000C24007803F03F0348BF04FB0022042B5B
:1041300039460BD004D8013B012B0CD817700AE08C
:10414000102B05D0202B05D0082B04D1118002E0C4
:10415000176000E0176031461448F8F7CEFE284695
:10416000002103B0BDE8F04F13E6114805E00BF164
:10417000010BBBF19E0F8AD10E4803B0BDE8F04F92
:1041800076E6504603B0BDE8F04F17E703B0BDE850
:10419000F08F00BFA5C7010828AB01080FC10108B7
:1041A000B7C70108B40F0020AC280020BAC7010827
:1041B000C5C70108C2BF010888A9010808B507489A
:1041C000FFF756FE064BD869FAF72AF8F6F7ACFD6A
:1041D000F8F7D8FF034A044BDA6008BDE5C70108C9
:1041E000AC2800200400FA0500ED00E008B5054801
:1041F000FFF73EFEFFF7A6F8F8F7EEFFBDE8084030
:10420000DCE700BFF1C7010808B50448FFF730FE3E
:10421000F8F7E2FFBDE80840D0E700BF07C8010893
:104220002DE9F04F9B498BB00B7813F0010F03F091
:10423000040200F08E81002A40F0988196480768B9
:1042400017F0806740F09281980700F1828143F077
:1042500004030B70914B1A88914B1A80914B1A688A
:10426000994612F4002F00F055818F4B80201F706B
:1042700000F05CFC08B1FFF705FD8C4C2678012EA0
:1042800040F048818A4D95F8D22722B195F8D3376E
:104290000BB19A4203D3012385F8D2370FE01846B9
:1042A000114630B191FBF0FE00FB1E1E0146704628
:1042B000F7E792FBF1F293FBF1F385F8D22785F84B
:1042C000D33795F8D437012B82BF794B002283F87E
:1042D000D42741F66902774B95F8D4871B6803EB26
:1042E000C303934284BF40F2E242B3FBF2F3724A4B
:1042F0008CBFDBB204231370B8F1000F03D0B8F108
:10430000010F23D028E08020F6F7B0F8834618B3D9
:104310008021F6F787F89BF80620684BDFF8A4A108
:1043200053F822300221B3F5613F0CBF0222002274
:104330008AF800009BF900008DE8060080214246C3
:10434000F6F7C9F9CAF8040048B905E05C4BDB6828
:1043500013B1FFF735FA10B100232370DAE0594C9E
:104360000021142204F1080004F0B3FB04F1280337
:10437000E36104F1980395F88411236204F58473D2
:104380006362514B049195F892111B880029697959
:10439000A4F87831D9F80030A1F1190E03F40062C5
:1043A000C3F3400CC3F3C03318BF0123DEF1000098
:1043B00040EB0E00012914BF0146012195F8D207F8
:1043C000039195F8D317059388422CBF0021012152
:1043D00006913E493E4B8A463E481B680078D1F81C
:1043E00000B0C3F3C003029006F1FF385FFA88F80B
:1043F00008F1FF31132943D8DFE801F00C0C0C0C55
:104400000C0C0C0C0AB246B433463D1212123F4655
:104410000399A8E002994145B4BF002501252EE08B
:104420009BF80010022915D1A8F102015BF82100C8
:1044300000210992CDF820C0079301F025FD4FF02F
:104440000105079BDDF820C0099A08B14FF000056F
:10445000EDB214E00BEB08014D79003518BF0125D2
:104460000DE022B10499481E4142414100E011464D
:1044700001F0010177E0059975E0069973E01DB13F
:10448000012101FA08F10F43142E25D80136F6B2A6
:10449000AAE700BF002E0020A40E0020A80F0020D5
:1044A000CE0D0020941700209D2B0020A81800207E
:1044B000B40F002080260020F0000020DCB70108A7
:1044C00004000020F0280020E4250020E00E002059
:1044D000AC17002044190020DAF8000019217930C7
:1044E000C4F87C71F6F74EF80023C4F88431A4F8C0
:1044F0008831A4F88A31C4F894311E4BD4F8902145
:104500001B68C4F88C21C4F898311B4B022284F834
:1045100080011A70174B194A1B6892F8E0214FF47A
:104520007A7101FB0233164A1360D9F800301A067B
:1045300009D5144B1B789B0705D5134B1B78042B0F
:1045400001D9062000E005200BB0BDE8F04FF6F7DA
:10455000D9B95AB901200BB0BDE8F04FF6F7F8B958
:10456000194600E0614600298AD18FE70BB0BDE80B
:10457000F08F00BF980F0020A8180020B40F002073
:10458000880D0020B0170020B617002010B51A4A79
:10459000137859072ED523F004031370174B1B68AB
:1045A0001B0322D5164C2378A3F10802012A14D844
:1045B0004520F5F78DFAFF20F5F78AFA1148FFF745
:1045C000E5F90020F5F784FA0F4B1A680F4BC3F892
:1045D0009821FFF725F90A2306E0012B05D90A2BBC
:1045E00003D0FFF703F9012323700420BDE8104036
:1045F000F6F788B910BD00BF002E002094170020E8
:10460000A8180020F3D10108980F0020F0280020FE
:10461000012380F8453070472DE9F04390F84410AD
:10462000002380F84430002953D02E4C2268002A01
:1046300052D02268052A52D10D462B4C202928BF82
:1046400020256E1C27687610DFF8A8E0DEF8003021
:104650009BBB3246DFF8A0C000F1320313F8019C87
:1046600013F8028C013A48EA09282CF8048C03F16B
:1046700002030CF1040CF1D11C4B1A681C4B92B2D2
:1046800013445B00D3F800C01D60DEF800302A46FA
:104690002B44CEF80030DFF864E0DEF8003023F47D
:1046A000E04323F040039BB283F0300343F4004324
:1046B00043F08003CEF8003000E000228A4203D0AD
:1046C0002368DB1B312BBFD9531A58425841BDE830
:1046D000F0830120BDE8F0831046BDE8F083184662
:1046E000BDE8F083E82D0020980F0020505C0040CA
:1046F0000A300020902A002084610040045C0040C1
:10470000002280F8452087E790F84420531CDBB254
:10471000024480F8443082F8301090F845200AB105
:10472000132B00D978E77047014B5868C0B2704727
:10473000902A0020012070477047704720B9034B32
:1047400008229B681A82704701487047902A00200F
:104750005800002020B9034B08229B681A8270473A
:1047600001487047902A00205800002021B90128F4
:104770008CBF0220002070470220704710B5094B03
:104780009A68D378042B0BD8074CDB00518A23445A
:1047900018B99B895B1A138210BD9B68581810BD0D
:1047A000002010BD902A002058000020054B996879
:1047B000054B4A8A18B99B8D9B1A0B827047986AE1
:1047C00010447047902A002058000020054B99683B
:1047D000054B4A8A18B99B8E9B1A0B827047186B3F
:1047E00010447047902A002058000020074B9B6817
:1047F0001B7803F07F03212B06D100F0DF00022895
:1048000014BF02200020704702207047902A002029
:10481000212810B508D1114B9B681B7803F07F034A
:10482000212B10D0022010BD2028FBD10B4B0C4AAD
:104830009B6810701B7803F07F03212B094B18BF76
:1048400000230BB9EEE7084B044A00249268204687
:10485000936154829847204610BD00BF902A0020E3
:10486000052E00203D470108554701087047034BBE
:104870001A78202A04BF00221A707047052E0020E3
:10488000014B04221A607047E82D0020034B9B7DEA
:1048900013B1034B05221A60704700BF902A002015
:1048A000E82D0020F7B51E4B5A681D460AB95C6812
:1048B00000E0012493F828000021CAB2A24201F1CD
:1048C000010108D202AE2F1816443A4492F829206A
:1048D00006F8042CF1E75A68121B5A6093F8282056
:1048E0005D68224483F82820A5B903204021FCF705
:1048F0001FFB0C4A136823F4804323F070039BB220
:1049000083F4405343F4004343F080031360044BAB
:1049100083F82850002CC6D09DF8040003B0F0BDE9
:10492000902A00200C5C004010B50446B0F900004D
:10493000FFF728F8B4F90200FFF724F8B4F90400EF
:10494000BDE81040FFF71EB810B504460068FFF739
:1049500019F86068FFF716F8A068BDE81040FFF787
:1049600011B82DE9F74F0120F5F780FD002488B339
:10497000012C2FD84FF04C0909FB04FA174E06EB17
:104980000A0808F1B407BD7815B10134E4B2EEE7C6
:1049900090F9003090F804E01846114B03228DE89E
:1049A000240001212A4653F82E30F5F794FE834661
:1049B00060B106F16C00504429464A4604F089F87B
:1049C00001231C44C8F86CB0BB70E4B20120F5F7B9
:1049D00033FDCCE703B0BDE8F08F00BF902A002084
:1049E000DCB701080021222210B5114804F071F84B
:1049F000104B0022194610480424105C013283F841
:104A0000F40183F8F94105200024042A83F8F80111
:104A100083F8FB4183F8FA0103F10803EBD101238A
:104A2000A1F8F631A1F8FE31522381F8F23110BD20
:104A3000A6110020B40F002010D2010870B5064660
:104A4000441E14F8011F89B1094D284604F077F877
:104A50000028F6D005F1080398423FBF054B401BE4
:104A6000C018A31B38BF80F88831EAE770BD00BFCB
:104A700014D20108B40F0020031EB8BF2D2210B5B8
:104A8000B8BF58420C46B8BF01F8012B0A22F8F70C
:104A900035F900230370204610BD07B51C4B03F504
:104AA0008472C3F804211B4A92F890215AB1012A5A
:104AB00014D1032183F80A11072183F80C2183F80C
:104AC0000B110C2208E0022183F80A11032183F85C
:104AD0000C2183F80B11072283F808210E4A0F4B93
:104AE00040209A63F5F7C2FC70B10122002390F9CF
:104AF000000040218DE80C00094A4FF4E133F5F73E
:104B0000EAFD003018BF012003B05DF804FB00BFD0
:104B1000902A0020B40F00206D4E0108580000209C
:104B2000214F010801200021FFF700B9174AF0B515
:104B3000164692F80D31D2F810E1032B10D85C1C08
:104B40000EEBC3039D1CE4B208D09A88D10705D5AB
:104B5000104203D008E00131042907D12346ECE7D5
:104B600086F80D310020F0BD9F7800210C2202FB59
:104B700001F3064D05F58A7C1CF803209742EAD123
:104B80002B4485F80D41D3F81801F0BD902A002080
:104B90004FF6FB72094B10B519681C460A401A60A3
:104BA000074A084B927D0AB1052200E001221A60F3
:104BB000FCF732FC4FF43643236010BD405C0040EC
:104BC000902A0020E82D00200D4B10B51A680D4BDF
:104BD00092B213445B001B680B4AC3F309031360D2
:104BE00013680A499BB201335B1000229A4206D037
:104BF00051F8044B064820F812400132F6E710BD88
